:100000000C94080A0C94270A0C94270A0C94E30B0E
:100010000C941D0C0C94270A0C94270A0C94270AA4
:100020000C94270A0C94270A0C94270A0C94270A8C
:100030000C94270A0C94270A0C94270A0C94370F67
:100040000C94270A0C94270A0C94270A0C94270A6C
:100050000C94D7730C94856B0C94270A0C94270A84
:100060000C94270A0C94586C0C94270A0C944C6C32
:100070000C94270A0C94270A0C94270A0C94270A3C
:100080000C94087F0C94270A0C94270A0C94270AD6
:100090000C94966C0C94270A0C948A6C0C94270A86
:1000A0000C94270A0C94270A0C94270A0C94270A0C
:1000B0000C94270A0C94270A0C94270A0C94270AFC
:1000C0000C94270A0C94270A0C94270A0C94270AEC
:1000D0000C94270A0C94270A0C94270A0C94270ADC
:1000E0000C94270A0C9490730C949A730C94867356
:1000F0000C9446730C94CB730C94BC730C94B07337
:100100000C94A4730C94270A0C94270A0C94270AC5
:100110000C94270A0C94270A0C94270A0C94270A9B
:100120003D885C88D688C889E889088A108ABD8994
:10013000084AD73B3BCE016E84BCBFFDC12F3D6C4E
:1001400074319ABD56833DDA3D00C77F11BED9E4B4
:10015000BB4C3E916BAAAABE000000803F076342E1
:1001600036B79BD8A71A39685618AEBAAB558C1D4E
:100170003CB7CC5763BD6DEDFD753EF6177231BFD0
:10018000000000803F08000000BE922449123EABF0
:10019000AAAA2ABECDCCCC4C3E00000080BEABAAA1
:1001A000AAAA3E00000000BF000000803F0000003F
:1001B0000000084178D3BB4387D1133D190E3CC3DF
:1001C000BD4282AD2B3E68EC8276BED98FE1A93E5E
:1001D0004C80EFFFBE01C4FF7F3F00000000000025
:1001E00025630025630025730A005854414C5F5471
:1001F00052494D3D25640025730A0025730A0054B9
:1002000065737420362025730A0054657374203595
:100210002025730A005465737420342025730A0066
:100220005465737420332025730A00546573742059
:10023000322025730A005465737420312025730A17
:10024000006368616E3D25640A0074787077723DC2
:1002500025640A003530306B0A003235306B0A00F5
:100260003131356B0A0035366B0A0033386B0A00C2
:1002700025730A00765F6C6F773D252D332E32662D
:100280000A0025730A0073656E743D252D75206480
:1002900075703D252D752069676E6F7265643D250B
:1002A0002D752074746C5F7A65726F3D252D750A0B
:1002B0000025372E33662025372E33660025352E50
:1002C000326620004572726F72203020566F6C7457
:1002D000004E6F7420737570706F727465640A00DD
:1002E0004572726F72203020566F6C7400457272C6
:1002F0006F72203020566F6C740062756C6B5F6497
:10030000656C61793D252D750062756C6B3D252D01
:10031000750056616C7565206E6F7420616C6C6F32
:100320007765640062756C6B3A206D61783D257568
:100330002073746172743D25752C20656E643D25B3
:10034000752C20696E5F7573653D25750A007062B6
:10035000323D25730A007062313D25730A00256C19
:100360007500416C6C6F77656420737065656420FF
:10037000312F31302F3130302F343030206B6269E3
:10038000742F730025630074746C3D252D64200068
:1003900074746C3D252D6420004E65772074746C58
:1003A0003D252D6420002563004D53353631312025
:1003B000503D252D372E326620252D372E32666D85
:1003C0000A00424D5030383520256C6420506120A1
:1003D00020252D372E32666D00256300545F484579
:1003E00041545F4944583D252D352E326620005436
:1003F0005F4445573D252D352E3266200041483D4E
:10040000252D352E32662000545F53485432583D16
:10041000252D352E3266200052485F5348543258FD
:100420003D252D352E32662000545F52483D252D46
:10043000342E3166200052483D252D342E31662061
:100440000025630025630025630025630025630004
:100450007265706F72745F616C6C3D007265706F75
:1004600072743D0025630025630025630025630049
:10047000204F534343414C3D256420002046757373
:10048000653A2065653D253032782068663D253027
:100490003278206C663D25303278206C623D253004
:1004A0003278004D43553D2530366C780025630089
:1004B00074785F6C656E3D252D6C752C765F6C6F66
:1004C000773D252D6C752C73687432783D252D6C25
:1004D000752C62756C6B3D252D6C75002563004F86
:1004E0004B0A002563002563002563002563002572
:1004F00063002563002563002563006465627567FA
:100500005F616C6C3D0064656275673D00646562A7
:1005100075673D0025730A00646565700A006E6F9B
:100520006E650A00707772733D007062323D25730C
:100530000A007062313D25730A00696E74725F7340
:1005400065635F70313D252D372E33660A00696E75
:1005500074725F70313D252D6C640A00696E74728F
:100560005F7365635F70303D252D372E33660A005B
:10057000696E74725F70303D252D6C640A00765F81
:100580006D63753D252D352E32660A00745F6D63EF
:10059000753D252D352E32660A00707077723D2527
:1005A000730A0064656275673D0072636D643D2582
:1005B000730A0025730A006175746F0A006C6F6717
:1005C0005F6D6F64653D007573625F7077723D2586
:1005D000730A0072656C61793D25730A0074746C4E
:1005E0003D252D640A0052494D455F616464723DAA
:1005F000252D642E252D640A006E65696768626F7B
:10060000725F7461626C655F73697A653D25640A27
:1006100000765F6C6F773D252D332E32660A0074AD
:100620007870773D25640A006368616E3D25640A31
:100630000069643D006932635F6275733D00693231
:10064000635F73706565643D252D6C750A00747871
:10065000743D25730A0053797374656D2053756D6D
:100660006D6172790A002530366C780041744D65F1
:100670006761323536524652320041744D656761CA
:10068000313238524652320041744D65676136341A
:10069000524652320041744D6567613132385246DC
:1006A0004131004D43553D006D61736B3D002C00A1
:1006B000696E74657276616C3D252D750023252D5C
:1006C000642C00745F686561745F69647800745FAE
:1006D00064657700616800705F6D73353631310095
:1006E00072685F736874327800745F73687432780C
:1006F0000070610070006164340061643300616403
:100700003200616431006133006132006131007692
:100710005F696E0072680065727200757074696D51
:10072000650070315F6C73740070315F74007031FC
:100730000070305F6C73740070305F740070300054
:10074000765F6D637500745F6D637500743100745E
:100750000069640065363400747874002D002B0045
:100760006175746F006E6F6E650062756C6B007002
:100770006F7765725F736176655F6C65647279002F
:1007800072656C61795F6C65647900636F6D70612F
:10079000737300616363656C007072657300705FF2
:1007A000707772006165730070315F6C6564790009
:1007B00070305F6C656472006576656E74006C65A0
:1007C00064006F7700706B740074785F6C65647997
:1007D0000072785F6C656472006F706572006E6F96
:1007E0006E65002530327800765F6164343D252DDA
:1007F000382E3666002000765F6164333D252D3843
:100800002E3666002000765F6164323D252D382E3D
:100810003666002000765F6164313D252D382E3626
:1008200066002000765F6C696768743D252D382E60
:100830003666002000765F61323D252D372E336607
:10084000002000765F61313D252D372E3366002074
:1008500000765F696E3D252D352E326600204E658F
:100860007665722D7573656420737461636B203EC9
:100870002025642062797465730A00757074696D4F
:10088000653D252D642D646179732D253032643AE0
:10089000253032643A253032642D686F7572730AE0
:1008A0000074657374205B6F66667C317C327C33C8
:1008B0007C347C355D20202020202020202D2074B9
:1008C000657374206D6F6465730A0D007478205B26
:1008D000706B74207061796C6F61645D20202020E2
:1008E00020202020202020202D2073656E6420727F
:1008F0006164696F20706B74206B6579626F6172DF
:10090000640A0D00776474205B6F6E7C6F66667C92
:10091000746573745D20202020202020202020205A
:100920002D207761746368646F670A0D00765F6CD1
:100930006F77205B765F6C6F775D20202020202012
:100940002020202020202020202D206C6F77657310
:1009500074207265706F727420766F6C7461676555
:100960000A0D007570677220202020202020202092
:100970002020202020202020202020202020202D6A
:10098000207265626F6F742076696120626F6F7488
:100990006C6F616465720A0D0075617274205B335F
:1009A000386B7C35366B7C3131356B7C3235306B56
:1009B0007C3530306B5D202D20736574207465723A
:1009C0006D2F756172742073706565640A0D006225
:1009D0006F6F742020202020202020202020202025
:1009E00020202020202020202020202D2072656221
:1009F0006F6F740A0D0070777273205B64656570A9
:100A00007C6E6F6E655D202020202020202020201D
:100A100020202D206D637520736C656570206D6FCF
:100A200064650A0D007265737420656570726F6D80
:100A300020202020202020202020202020202020B6
:100A4000202D20726573746F726520656570726FFA
:100A50006D0A0D0070707772205B6F6E7C6F66663A
:100A60005D20202020202020202020202020202049
:100A70002D2070726F6772616D6D61626C652070A0
:100A800077720A0D0070623220205B6F6E7C6F6699
:100A9000665D2020202020202020202020202020D3
:100AA000202D2070726F6772616D6D61626C6520C0
:100AB00070696E2062320A0D0070623120205B6F17
:100AC0006E7C6F66665D2020202020202020202064
:100AD00020202020202D2062756C6B204750494F2C
:100AE0002070696E0A0D00747874205B73747269EB
:100AF0006E675D2020202020202020202020202024
:100B00002020202D20536574207265706F72742030
:100B10007465787420737472696E670A0D00747856
:100B20007077205B31352D305D2020202020202063
:100B3000202020202020202020202D20545820500C
:100B400077722E20486967686573742030202833D7
:100B500064426D290A0D0074746C205B302D3135B0
:100B60005D20202020202020202020202020202048
:100B70002020202D2074696D652D746F2D6C697691
:100B80006520666F72207061636B6574730A0D0077
:100B900073732020202020202020202020202020AF
:100BA0002020202020202020202020202D2073798C
:100BB0007374656D2073756D6D6172790A0D0072C5
:100BC00073202020202020202020202020202020D2
:100BD00020202020202020202020202D2072616431
:100BE000696F2073746174730A0D007269205B234E
:100BF0006E5D205B696E745D202020202020202007
:100C0000202020202020202D207265706F727420FB
:100C1000696E74657276616C0A0D0072636D642092
:100C20005B6F6E7C6F66665D202020202020202078
:100C3000202020202020202D20616C6C6F772063E5
:100C40006D642066726F6D206E65746F726B0A0D35
:100C5000007265205B236E5D205B2B7C2D5D205B2D
:100C60006D61736B7C6175746F2C6D61736B5D204E
:100C70002D206D6F7465207265706F7274207365BE
:100C8000742F6D6F646966790A0D006F77202020DC
:100C90002020202020202020202020202020202054
:100CA000202020202020202D206F6E652D77697256
:100CB000652073656E736F72730A0D006C6F672029
:100CC0005B6175746F7C6F6E7C6F66665D20202043
:100CD00020202020202020202D206D6F746573207F
:100CE00064617461206F6E205553420A0D006E6579
:100CF000205B666C7573685D2020202020202020FA
:100D0000202020202020202020202D206E656967B3
:100D100068626F72207461626C650A0D00657272A0
:100D200020202020202020202020202020202020C3
:100D30002020202020202020202D206572726F721C
:100D40002073746174730A0D006D63752020202078
:100D50002020202020202020202020202020202093
:100D600020202020202D206D637520696E666F0A7B
:100D70000D00693263205B70726F62657C73706511
:100D8000656420236E5D20202020202020202D203F
:100D90006932632070726F6265206275737C73655F
:100DA00074206275732073706565640A0D00696450
:100DB000205B72657365745D202020202020202038
:100DC000202020202020202020202D206964206841
:100DD000616E646C696E670A0D0068756D20202075
:100DE0002020202020202020202020202020202003
:100DF0002020202020202D2068756D696469747979
:100E00002073656E736F720A0D0072656C617920D4
:100E10005B6F6E7C6F66667C73746174735D20209B
:100E20002020202020202D2072656C6179206E65A5
:100E300074776F726B207265706F7274730A0D0035
:100E40006465205B6D61736B5D2020202020202075
:100E50002020202020202020202020202D206465FC
:100E60006275670A0D006368616E205B31312D3257
:100E7000365D20202020202020202020202020201F
:100E800020202D206368616E2031312D32362028DC
:100E9000322E3430352D32343830204D687A290ADC
:100EA0000D0063616C69205B5B765F696E7C61310C
:100EB0007C61325D20766F6C747C72657365747CC6
:100EC0006E6F6E655D202D2063616C696272617466
:100ED000650A0D0062756C6B205B5B73686F777CD5
:100EE000666C7573685D205B7365742074687273DB
:100EF000682064656C61795D5D20202D2062756CD1
:100F00006B696E67207061636B657473200A0D00F6
:100F10006164632020202020202020202020202009
:100F20002020202020202020202020202D20736819
:100F30006F7720765F696E2C2061312C2061322022
:100F4000766F6C74616765730A0D00752020202030
:100F50002020202020202020202020202020202091
:100F6000202020202020202D20757074696D650AB6
:100F70000D0076202020202020202020202020204E
:100F800020202020202020202020202020202D2054
:100F900076657273696F6E0A0D006820202020202C
:100FA0002020202020202020202020202020202041
:100FB0002020202020202D2068656C700A0D00253F
:100FC0006300756E6B6E6F776E20636D640A004808
:100FD0004D433538383300257300257300202573C1
:100FE000002025362E3266200025303278007465C8
:100FF0006D705F65787465726E3D252D362E326694
:1010000000202573002025362E3266204F6E2D429B
:101010006F61726400253032780074656D705F62B4
:101020006F6172643D252D362E3266000A004275CE
:101030006C6B2072656D3A2073746172743D257516
:101040002C20656E643D25752C20696E5F75736577
:101050003D25750A0042756C6B206164643A20730B
:10106000746172743D25752C20656E643D25752C68
:1010700020696E5F7573653D25750A0042756C6B5E
:10108000207468726573683A2074696D65723D25D5
:10109000750A00503A20256C642050612020252DCF
:1010A000372E3266206D0A004932433A200045202F
:1010B00025642E256420636C6F636B20256C75207E
:1010C00063707520256C75206C706D20256C752003
:1010D00069727120256C7520676C656420256C75BC
:1010E00020796C656420256C7520726C6564202500
:1010F0006C7520747820256C75206C697374656E2E
:1011000020256C752073656E736F727320256C7566
:101110002073657269616C20256C750A0053202567
:10112000642E256420636C6F636B20256C752074BE
:101130007820256C7520727820256C752072747863
:1011400020256C752072727820256C752072657868
:101150006D697420256C752061636B747820256C33
:1011600075206E6F61636B747820256C75206163E8
:101170006B727820256C752074696D65646F757469
:1011800020256C752062616461636B727820256C28
:101190007520746F6F6C6F6E6720256C7520746F8F
:1011A0006F73686F727420256C7520626164737947
:1011B0006E636820256C752062616463726320250C
:1011C0006C7520636F6E74656E74696F6E64726F98
:1011D0007020256C752073656E64696E6764726F2C
:1011E0007020256C75206C6C747820256C75206CD3
:1011F0006C727820256C750A00257325730A004FE0
:101200006E6C696E650A000A002C20636865636B6A
:10121000207261746520257520487A002573202589
:10122000732C206368616E6E656C20257520706F6D
:10123000776572202575000A0025783A004D4143F4
:101240002061646472657373200052616E646F6D17
:101250002045554936342061646472657373206794
:10126000656E6572617465640A000A2A2A2A2A2A50
:101270002A2A426F6F74696E672025732A2A2A2AE8
:101280002A2A2A0A00454550524F4D20697320638F
:101290006F72727570742C20726577726974696EE2
:1012A0006720776974682064656661756C74732E55
:1012B0000A006C6F63616C686F73740041544D4534
:1012C00047413132387266613100020000FFFE0092
:1012D00000016E616E00696E660000407A10F35A7C
:1012E00000A0724E18090010A5D4E80000E8764866
:1012F000170000E40B54020000CA9A3B000000E112
:10130000F505000080969800000040420F000000A4
:10131000A08601000000102700000000E803000084
:1013200000006400000000000A000000000001004E
:10133000000000002C76D888DC674F0823DFC1DF6F
:10134000AE59E1B1B796E5E3E453C63AE651997672
:1013500096E8E6C28426EB898C9B62ED407C6FFCAC
:10136000EFBC9C9F40F2BAA56FA5F490055A2AF7EE
:101370005C936B6CF9676DC11BFCE0E40D47FEF5F7
:1013800020E6B500D0ED902E03009435770500805F
:10139000841E080000204E0A000000C80C333333BE
:1013A000330F986E12831141EF8D2114893BE6555E
:1013B00016CFFEE6DB18D1844B381BF77C1D901D41
:1013C000A4BBE424203284725E228100C9F124ECA3
:1013D000A1E53D274E414E494E495459494E46CD0F
:1013E000CCCC3D0AD7233C17B7D13877CC2B3295DC
:1013F00095E6241FB14F0A000020410000C84200BA
:10140000401C4620BCBE4CCA1B0E5AAEC59D740083
:1014100011241FBECFEFD1E4DEBFCDBF1AE0A0E0A4
:10142000B2E0E8EDFAE301E00BBF02C007900D92D5
:10143000A633B107D9F72DE3A6E3BAE001C01D92A8
:10144000A036B207E1F70E94DF8A0C946A9D0C94E3
:1014500000008115910511F00197F1F7089584E2DC
:1014600095E09F938F930E94499A80916202909198
:101470006302A0916402B09165020F900F9093FFF8
:1014800003C08EE195E002C088E195E09F938F93C1
:101490000E94499A0F900F900895E091FD1BEF7301
:1014A000F0E0E25BF34E80838091FD1B8F5F8093C1
:1014B000FD1B80919E34886080939E3448E452E006
:1014C00061E1CA010E94445B80E090E00895CF93FF
:1014D000DF93EC018091410A9091420AA091430A66
:1014E000B091440A86FF1DC08E811F928F938D811B
:1014F0001F928F938C811F928F938B811F928F935A
:101500008A811F928F9381E793E09F938F930E942C
:10151000359A8DB79EB70C960FB6F8949EBF0FBE46
:101520008DBFBE0182E89AE00E94785CBE0184E033
:1015300092E0DF91CF910C94EC5B52985A981DBACF
:10154000E9E6F0E0808180628083EA9A53985B98B4
:10155000EB9A808180688083E8E6F0E0808181609A
:1015600080830895E3EBFCE11182128210820895DA
:10157000CF92DF92EF92FF920F931F93CF93DF935F
:10158000EC019B018091B31C843108F0BBC08091B9
:10159000B51C64E10E9427939093B51CC090D02F96
:1015A000D090D12FE090D22FF090D32F092F10E0C0
:1015B0008DE8989FD0011124AD54B34E1396CD926F
:1015C000DD92ED92FC9216974115510559F0FA0102
:1015D0008081FD01EA57FF4F8083FA018181A9577D
:1015E000BF4F8C932097A9F089819DE8909FF001CF
:1015F000919FF00D1124ED54F34EDF01A657BF4F1C
:101600008C93E557FF4F88818F70808388818F701E
:10161000808321153105E1F1D90116964C91169779
:101620005DE8509FC001519F900D11248D54934E41
:10163000FC01E757FF4F408315964C911597319762
:10164000408334961B964D915D916D917C911E97D0
:10165000452F562F672F7727518340837C01BEE8A3
:10166000EB0EF11CF9012385348545855685A4E6EA
:10167000B0E00E94CA93672F782F892F992724E61C
:1016800030E040E050E00E945B93D7016D937C9383
:101690008DE8809FD001819FB00D1124A654B34ED8
:1016A000FE0132968FE701900D928A95E1F78091C5
:1016B000B51C8F5F8093B51C9091B31C9F5F909376
:1016C000B31C4091410A5091420A6091430A7091C3
:1016D000440A60FF2DC01F929F931F928F938091A9
:1016E000B41C1F928F9385E590E19F938F930E9486
:1016F000499AEDB7FEB738960FB6F894FEBF0FBE05
:10170000EDBF16C08091E02F9091E12FA091E22FC4
:10171000B091E32F0196A11DB11D8093E02F90930E
:10172000E12FA093E22FB093E32F80E090E002C07E
:1017300081E090E0DF91CF911F910F91FF90EF90AA
:10174000DF90CF9008952091B31C222361F1809106
:10175000B41C8F5F21502093B31C64E10E94279337
:101760009093B41C4091410A5091420A6091430AFF
:101770007091440A60FF1AC01F922F938091B51C8C
:101780001F928F931F929F938EE290E19F938F936E
:101790000E94499A8DB79EB708960FB6F8949EBFDF
:1017A0000FBE8DBF03C080E090E0089581E090E01F
:1017B000089581110C949D0A109269005A9AEA9832
:1017C0005B9AEB9808951F920F920FB60F92112417
:1017D0008F939F93AF93BF938091680080FF24C045
:1017E0008091793490917A34A0917B34B0917C349B
:1017F0000196A11DB11D8093793490937A34A09302
:101800007B34B0937C348091410A9091420AA0913C
:10181000430AB091440A87FF07C0749882E090E0C1
:1018200090938F0280938E02BF91AF919F918F9181
:101830000F900FBE0F901F9018951F920F920FB62A
:101840000F9211248F939F93AF93BF938091680061
:1018500080FF24C080917D3490917E34A0917F34AC
:10186000B09180340196A11DB11D80937D34909379
:101870007E34A0937F34B09380348091410A90915C
:10188000420AA091430AB091440A90FF07C073989E
:1018900082E090E090938F0280938E02BF91AF918F
:1018A0009F918F910F900FBE0F901F90189580936E
:1018B0007C0080917B00877F80937B0080917C00FF
:1018C000806C80937C0085E080937A0080917A0020
:1018D000806880937A0080917B0087FFFCCF8091A5
:1018E0007B0085FFFCCF80917A00806480937A0032
:1018F00080917A0086FDFCCF1092790010927800DA
:1019000084E090E060E070E020917A002064209311
:101910007A0020917A0026FDFCCF2091780030914A
:101920007900620F731F019779F710927C00809104
:101930007A008F7780937A0076956795769567958C
:1019400080E090E00E944E90089580E00E94570C45
:10195000209186023091870240918802509189023D
:101960000E94489221EE3AE744E95EE30E94B98E74
:1019700008950F931F93CF93DF930FE110E0CBE512
:10198000DEE00093510187EC90E00E94290A8091EB
:10199000510185FD0DC00031110521F02CF0CB5413
:1019A000D10903C0C4ECD9E0E29701501109E9CF95
:1019B000BE0180E090E00E944E9020E030E04AE7D7
:1019C00054E40E949C8FDF91CF911F910F91089555
:1019D000CF93DF93EC0188819981009799F08B3D3B
:1019E000914121F01982188283E011C0623171F4B3
:1019F0000E94B90C6093CC2F7093CD2F8093CE2F83
:101A00009093CF2F8BED91E19983888381E0DF91D3
:101A1000CF91089580917B00886080937B0089EC52
:101A200080937C0085E080937A0080917A008068C2
:101A300080937A0080917B0087FFFCCF80917B00B0
:101A400085FFFCCF80917A00806480937A0080913A
:101A50007A0086FDFCCF80917A00806480937A00C2
:101A600080917A0086FDFCCF6091780070917900BA
:101A700080917A008F7780937A0080E090E00E94D6
:101A80004E9027ED33EA40E95FE30E94489226E654
:101A900036E648E853E40E94B88E0895CF92DF926C
:101AA000EF92FF921F93CF93DF93CDB7DEB72997C5
:101AB0000FB6F894DEBF0FBECDBF6C0110923A0A8C
:101AC0008FEF898786E0E82E8CE1F82E10E089857B
:101AD0008823E9F11830D9F1BE016F5F7F4FCE0145
:101AE00009960E94C76499859F3F11F09E3F19F4A3
:101AF00090933A0A2CC0CE010196C114D10481F40E
:101B00000E94E16480939B34A3E9B4E3FE01319623
:101B100088E08E0F91919D938E13FCCF81E018C0C9
:101B20000E94E164F7018087FE01319620E030E0F9
:101B30008191D701A20FB31F8C932F5F3F4F2830A5
:101B40003105B1F71F5FF9E0EF0EF11CC0CF812F17
:101B500029960FB6F894DEBF0FBECDBFDF91CF91AF
:101B60001F91FF90EF90DF90CF9008958CE290E16D
:101B70009F938F930E94499A0F900F9008952F92F0
:101B80003F924F925F926F927F928F929F92AF920D
:101B9000BF92CF92DF92EF92FF920F931F93CF935A
:101BA000DF93EC015B01009711F427E003C001977C
:101BB00049F426E04AE250E06BE270E089E290E00E
:101BC0000E94A163CE010E944E0D9E01255C354FFF
:101BD0006901D9018C93CD2B69F0C6E0DCE1E12CE1
:101BE000F12C81EE282E8FE0382E9DED892E9FE07E
:101BF000992E9EC083E994E30E941066BC01990F60
:101C0000880B990B0E9450906B017C01AB2869F006
:101C100020E030E048EC52E40E949C8F9F938F9329
:101C20007F936F938AE190E1A4C0C3E9D4E305E117
:101C300010E189911F928F931F930F930E94499AED
:101C40000F900F900F900F90B4E3CB39DB0789F71B
:101C500020E030E048EC52E4C701B6010E949C8FBE
:101C60009F938F937F936F9385E090E19F938F93E2
:101C70000E94499A0F900F900F900F900F900F9025
:101C800080919B34811103C084E194E002C080EA1A
:101C900093E09F938F9381E090E19F938F930E94B5
:101CA000499A0F900F900F900F906DC000E010E0D8
:101CB000FE01E00FF11F80811F928F93A9EEBFE01C
:101CC000BF93AF930E94499A0F5F1F4F0F900F90E1
:101CD0000F900F900830110559F720E030E048ECE4
:101CE00052E4C301B2010E949C8F9F938F937F9314
:101CF0006F933F922F920E94499A0F900F900F90EE
:101D00000F900F900F908885811151C084E194E06D
:101D10009F938F939F928F920E94499A0E94B60D33
:101D2000FFEFEF1AFF0A29960F900F900F900F9078
:101D3000D6018C9190E0E816F906E4F5CE010E94F8
:101D40001066BC01990F880B990B0E9450902B01D3
:101D50003C01A114B10409F4A9CF20E030E048EC23
:101D600052E40E949C8F9F938F937F936F938EEE8C
:101D70009FE09F938F930E94499A0F900F900F902E
:101D80000F900F900F90DF91CF911F910F91FF90C7
:101D9000EF90DF90CF90BF90AF909F908F907F900B
:101DA0006F905F904F903F902F900C94B60D80EA0B
:101DB00093E0AECFDF91CF911F910F91FF90EF9005
:101DC000DF90CF90BF90AF909F908F907F906F905B
:101DD0005F904F903F902F900895CF93DF9300D066
:101DE000CDB7DEB7E3E9F4E38181898387818A8314
:101DF000CE0101960E9433590F900F90DF91CF9141
:101E00000895CF93DF93EC01209193343091943473
:101E100040919534509196346091973470919834F4
:101E20008091993490919A34AFEF0E949695E1F4A5
:101E300027E04AE250E06BE270E089E290E00E9425
:101E4000A16380E090E00E944E0DC55CD54F888371
:101E500049E050E06EE070E083E994E30E944D9D1C
:101E6000DF91CF910C94ED0EDF91CF9108951F92E9
:101E70000F920FB60F9211240BB60F92FF920F9391
:101E80001F932F933F934F935F936F937F938F9302
:101E90009F93AF93BF93CF93DF93EF93FF93809183
:101EA0009E34826080939E348091620286FD2B9ADC
:101EB0008091620287FD2B9A80918E0290918F0211
:101EC0001816190614F4749A739A8091410A909125
:101ED000420AA091430AB091440A85FF02C0749857
:101EE00073988091020290910302019790930302EC
:101EF00080930202892B09F04CC18091510A909184
:101F0000520A01969093520A8093510A8091D02FE1
:101F10009091D12FA091D22FB091D32F0196A11DD6
:101F2000B11D8093D02F9093D12FA093D22FB09337
:101F3000D32F80E190E0909303028093020280917E
:101F4000620280FD02C01D9B05C010923F0A1092E4
:101F50003E0A06C081E090E090933F0A80933E0ADB
:101F60008091410A9091420AA091430AB091440A9B
:101F700097FF08C080913E0A90913F0A892B49F053
:101F8000749A73980DEA1BE1C5EEDFE2FF24F39427
:101F900021C0739A7498F6CF8091510A9091520A99
:101FA00001960E943393892BE1F0F80160857185D9
:101FB00061157105A1F5F8016085718561157105DF
:101FC00009F03FC0065F1F4F2596FFE2C93FDF07BC
:101FD00009F44CC0F801608571856115710529F31C
:101FE000DBCF4281417020E030E050E060E070E003
:101FF00080E090E0A0E00E949695B9F277988091F9
:10200000410A9091420AA091430AB091440A92FF7A
:10201000CCCF749810928F0210928E02C6CF80910E
:10202000510A9091520A01960E943393892B19F616
:102030001C821B82AE0162E180E292E00E94445B5E
:10204000BACF8091510A9091520A0E943393892B02
:1020500009F0B8CFF8821A8309831C821B82AE0173
:1020600062E18EE392E00E94445BACCF6091680233
:102070007091690261157105A1F18091510A9091E9
:10208000520A0E943393892B61F5809179349091A3
:102090007A34A0917B34B0917C344091C227509126
:1020A000C3276091C4277091C527841B950BA60B8D
:1020B000B70B8093D51B9093D61BA093D71BB093DF
:1020C000D81B8091793490917A34A0917B34B0916F
:1020D0007C348093C2279093C327A093C427B093E6
:1020E000C527609166027091670261157105A1F1C3
:1020F0008091510A9091520A0E943393892B61F585
:1021000080917D3490917E34A0917F34B091803461
:102110004091C6275091C7276091C8277091C92761
:10212000841B950BA60BB70B8093D91B9093DA1BDE
:10213000A093DB1BB093DC1B80917D3490917E34A7
:10214000A0917F34B09180348093C6279093C727A5
:10215000A093C827B093C9278091620286FD2B986F
:102160008091620290916302A0916402B091650235
:1021700091FF0FC00E9408708A3119F0C1E0C80FAA
:1021800001C0CBE00E94BE6E8C2F0E9420700E9486
:10219000066F40E050E060E080E992E00E94445B1E
:1021A000FF91EF91DF91CF91BF91AF919F918F916F
:1021B0007F916F915F914F913F912F911F910F915F
:1021C000FF900F900BBE0F900FBE0F901F901895B1
:1021D0008091FD1B9091E42F891B08950E94E810C7
:1021E000882371F0E091E42FEF73F0E0E25BF34EAF
:1021F000808190E02091E42F2F5F2093E42F0895B9
:102200008FEF9FEF0895CF93DF93EC011092760A42
:102210001092750A888199810097C1F0843E93409D
:1022200021F01982188283E0BDC0613109F0B9C084
:102230000E94EE1099279093710A8093700A8D3056
:10224000910509F444C08F3F910549F40E94E810BC
:102250008111EECF84EE93E099838883A2C082310E
:10226000910509F45AC08F37910509F052C0809149
:102270006E0A90916F0A181619060CF560915A3D76
:1022800070915B3D88E090E00E94FD9960915A3D1D
:1022900070915B3D80E290E00E94FD9960915A3D13
:1022A00070915B3D88E090E00E94FD9980916E0AFC
:1022B00090916F0A019790936F0A80936E0A8091B4
:1022C0006E0A90916F0A8F37910509F0BFCF109277
:1022D000E42F1092FD1B80916E0A90916F0AFC0111
:1022E000E750F04D10829093760A8093750A109211
:1022F0006F0A10926E0A80919C3490919D340097E1
:1023000009F4A4CF40E050E0609184120E94445B45
:102310009DCF8830910571F5AACF60915A3D70919B
:102320005B3D8DE090E00E94FD9910926D0A109245
:102330006C0A20916C0A30916D0A80916E0A90911E
:102340006F0A281739070CF0BACFF901E750F04DA2
:10235000808160915A3D70915B3D90E00E94FD99B3
:1023600080916C0A90916D0A019690936D0A80930A
:102370006C0ADFCF60915A3D70915B3D0E94FD99E0
:1023800020916E0A30916F0A8091700AF901E7502E
:10239000F04D80832F5F3F4F30936F0A20936E0A7A
:1023A0008ECF81E0DF91CF91089580913E0A909188
:1023B0003F0A892BD1F08091620290916302A09133
:1023C0006402B091650293FD10C00E94BE6E83B797
:1023D000817F866083BFF89483B7816083BF7894E0
:1023E000889583B78E7F83BF78940895CF93DF93CA
:1023F000FC01208131812115310519F02E30324147
:10240000A1F4EC010E947B6D0E94D51140E050E0E8
:1024100065E880918812909189120E94445B8EE059
:1024200092E19983888381E004C0FC0111821082CB
:1024300083E0DF91CF910895CF93DF9300D0CDB7A4
:10244000DEB7892B81F05F934F938AED9FE09F93D6
:102450008F9369837A830E94499A0F900F900F900F
:102460000F907A8169817F936F9387ED9FE09F93AF
:102470008F930E94499A0F900F900F900F900F909A
:102480000F90DF91CF910895EF92FF920F931F93DA
:10249000CF93DF930E947B6D80EB0E949A6681113F
:1024A0001CC00E94F7668091CA2B9091CB2B816053
:1024B0009093CB2B8093CA2B89EA93E09F938F93C1
:1024C00087ED9FE09F938F930E94499A0F900F9002
:1024D0000F900F90C1E0D0E002C0C0E0D0E01EB18C
:1024E0001470729A0E947B6D8EE40E949A6681112C
:1024F00017C00E94F7668091CA2B9091CB2B826007
:102500009093CB2B8093CA2B7E018FEFE81AF80AA9
:102510004BE959E061EB73E0CE010E941C12E70128
:10252000111101C072980E947B6D8EEE0E949A6616
:10253000811116C00E94F7668091CA2B9091CB2B17
:1025400084609093CB2B8093CA2B8E010F5F1F4F1B
:102550004BE959E069EB73E0CE010E941C12E801DF
:102560000E947B6D86EA0E949A66811116C00E94C5
:10257000F7668091CA2B9091CB2B88609093CB2BE0
:102580008093CA2B8E010F5F1F4F4BE959E060EC1F
:1025900073E0CE010E941C12E8010E947B6D8CE367
:1025A0000E949A6681111EC00E94F7668091CA2B14
:1025B0009091CB2B80619093CB2B8093CA2B8E0173
:1025C0000F5F1F4F4BE959E068EC73E0CE010E94AA
:1025D0001C128FEC9FE09F938F930E94499A0F905B
:1025E0000F90E8010E947B6D82ED0E949A66811136
:1025F00016C00E94F7668091CA2B9091CB2B806207
:102600009093CB2B8093CA2B8E010F5F1F4F4BE90A
:1026100059E060ED73E0CE010E941C12E8010E94B7
:102620007B6D80E80E949A66811116C00E94F76651
:102630008091CA2B9091CB2B91609093CB2B809360
:10264000CA2B8E010F5F1F4F4BE959E069ED73E014
:10265000CE010E941C12E8010E947B6D80ED0E9459
:102660009A66811116C00E94F7668091CA2B9091DC
:10267000CB2B80689093CB2B8093CA2B8E010F5F5E
:102680001F4F4BE959E06FED73E0CE010E941C1221
:10269000E8010E947B6D8CEE0E949A66811116C043
:1026A0000E94F7668091CA2B9091CB2B92609093F9
:1026B000CB2B8093CA2B8E010F5F1F4F4BE959E044
:1026C00067EE73E0CE010E941C12E80107E010E003
:1026D0000E947B6D8CE70E949A66811113C00E9454
:1026E000F7668091CA2B9091CB2B80649093CB2B73
:1026F0008093CA2B4BE959E06EEE73E0CE010E9445
:102700001C1203C00150110919F70E94F766DF91EE
:10271000CF911F910F91FF90EF900C94B60DCF9336
:10272000DF9300D0CDB7DEB74A8369830E94CE66BF
:102730006981862F0E94FF664A81842F0E94FF666E
:102740000F900F90DF91CF910C94F766AF92BF92EC
:10275000CF92DF92EF92FF920F931F93CF93DF936D
:1027600000D01F92CDB7DEB7182F022F4A835B83AC
:1027700069830E94CE666981862F0E94FF66812F41
:1027800081600E94F5664A81A42E5B81B52E10E01F
:10279000E12CF12C680181E0C81AD108E016F1069D
:1027A00089F0EC14FD0419F40E941A6702C00E941B
:1027B0001067F5018083FFEFEF1AFF0A8FEFA81A69
:1027C000B80AECCF0F900F900F90DF91CF911F912F
:1027D0000F91FF90EF90DF90CF90BF90AF900C944F
:1027E000F766BF92CF92DF92EF92FF920F931F9303
:1027F000CF93DF93CDB7DEB760970FB6F894DEBF07
:102800000FBECDBFF82EE42E6623D9F18E010F5FE7
:102810001F4F80E1F80111928A95E9F728E0A8019D
:1028200068E980EB0E94A613FF2041F087EF93E058
:102830009F938F930E94359A0F900F902EEFC22E88
:1028400023E0D22E37E0B32EB00EF80181918F0134
:102850001F928F93DF92CF920E94359A0F900F9024
:102860000F900F90B012F1CF88851F928F9383E560
:1028700094E09F938F930E94359A0F900F900F9042
:102880000F90EE20D9F18E010F5F1F4F80E1F8010C
:1028900011928A95E9F720E1A80160E880EB0E9497
:1028A000A613FF2041F083E094E09F938F930E9452
:1028B000359A0F900F908EEFE82E83E0F82E9FE070
:1028C000D92ED00EF80181918F011F928F93FF9224
:1028D000EF920E94359A0F900F900F900F90D012A8
:1028E000F1CF88891F928F9383E594E09F938F9314
:1028F0000E94359A0F900F900F900F9060960FB630
:10290000F894DEBF0FBECDBFDF91CF911F910F9125
:10291000FF90EF90DF90CF90BF9008950F931F939B
:10292000CF93DF9300D0CDB7DEB71A82198222E0B1
:10293000AE014F5F5F4F6AEA8EEE0E94A6130EE86B
:102940001CE1898190E0982F88272A81822BF80149
:102950009183808322E0AE014F5F5F4F6CEA8EEE81
:102960000E94A613898190E0982F88272A81822BC4
:10297000F8019383828322E0AE014F5F5F4F6EEADE
:102980008EEE0E94A613898190E0982F88272A81D5
:10299000822BF8019583848322E0AE014F5F5F4F65
:1029A00060EB8EEE0E94A613898190E0982F882715
:1029B0002A81822BF801938B828B22E0AE014F5F3C
:1029C0005F4F62EB8EEE0E94A613898190E0982FF4
:1029D00088272A81822BF801958B848B22E0AE0117
:1029E0004F5F5F4F64EB8EEE0E94A613898190E0EB
:1029F000982F88272A81822BF801978B868B22E0DB
:102A0000AE014F5F5F4F66EB8EEE0E94A613898189
:102A100090E0982F88272A81822BF801978386835C
:102A200022E0AE014F5F5F4F68EB8EEE0E94A6136F
:102A3000898190E0982F88272A81822BF80191873D
:102A4000808722E0AE014F5F5F4F6AEB8EEE0E94FF
:102A5000A613898190E0982F88272A81822BF8017C
:102A60009587848722E0AE014F5F5F4F6CEB8EEE5F
:102A70000E94A613898190E0982F88272A81822BB3
:102A8000F8019787868722E0AE014F5F5F4F6EEBBC
:102A90008EEE0E94A613898190E0982F88272A81C4
:102AA000822BF801918B808B0F900F90DF91CF914B
:102AB0001F910F9108952F923F924F925F926F92C4
:102AC0007F928F929F92AF92BF92CF92DF92EF92BE
:102AD000FF920F931F93CF93DF93CDB7DEB76C9721
:102AE0000FB6F894DEBF0FBECDBF182F042F2D8B6D
:102AF00019821A821B828091B21C811107C06C8FCF
:102B00000E948E1481E08093B21C6C8D662309F4C0
:102B100072C04EE264EF8EEE0E948F1369E07AE19C
:102B200080E090E00E94776622E0AE014F5F5F4F49
:102B300066EF8EEE0E94A6132981822F90E0A0E01E
:102B4000B0E04427582F692F7A2F8A81482B809133
:102B5000A41C9091A51C9A01AB01281B390B4109BB
:102B60005109A091A21CB091A31C0E94CA936B01B1
:102B70007C013FE0F594E794D794C7943A95D1F758
:102B800060919C1C70919D1CCB01770FAA0BBB0B15
:102B9000BC01CD014BE0660F771F881F991F4A9536
:102BA000D1F720919E1C30919F1C4901330FAA0838
:102BB000BB08A7019601280D391D4A1D5B1D0E9407
:102BC0007D93C20ED31ED092991CC092981C28E00F
:102BD000C20ED11C54E0D594C7945A95E1F70D2C40
:102BE000000CEE08FF08C092A61CD092A71CE09231
:102BF000A81CF092A91C812F8295880F880F807CD9
:102C00008C5C8887212E312CA3E0B0E0012E02C01D
:102C1000AA0FBB1F0A94E2F725E335E00E94C39395
:102C20009B01AC012E5F3F4F4F4F5F4F29873A8783
:102C30004B875C8780E593ECA0E0B0E09C01AD01A0
:102C400004C055954795379527951A95D2F7298B46
:102C50003A8B4B8B5C8B10E0412C512C320188E07D
:102C600090E0AC01421953095B8F4A8F101709F4A9
:102C70003EC1488564EF8EEE0E948F1369857A8588
:102C80008B859C850E94776623E0AE014F5F5F4F86
:102C900066EF8EEE0E94A613E091981CF091991CAD
:102CA000E05AFF409F01DF010E94AC936C837D835B
:102CB0008E839F838091901C9091911C9E878D871D
:102CC00020918E1C30918F1C388B2F872091921C65
:102CD0003091931C0E94AC936B017C01ADE0F594A4
:102CE000E794D794C794AA95D1F7A091941CB0917A
:102CF000951C2C813D814E815F818CE055954795D7
:102D0000379527958A95D1F70E94D593BB2797FDD4
:102D1000B095AB2F8C0D9D1DAE1DBF1D0296A11D44
:102D2000B11D32E0B595A795979587953A95D1F75E
:102D30009C01AD0130584F4F5F4FA091A01CB09146
:102D4000A11C0E94CA934B015C014FE0B694A7946A
:102D5000979487944A95D1F739818A8190E0A0E0D1
:102D6000B0E0BA2FA92F982F8827A32B2B81822B75
:102D70009C01AD010A8C04C0559547953795279560
:102D80000A94D2F72E8B3F8B488F598F4F855889E5
:102D90006A01550FEE08FF0862E0CC0CDD1CEE1C4A
:102DA000FF1C6A95D1F7A091961CB091971C2C81BD
:102DB0003D814E815F810E94D5939B01AC0177E1FB
:102DC00055954795379527957A95D1F72C833D836F
:102DD0004E835F832D853E85DF010E94AC93DC012D
:102DE000CB01EBE0B595A79597958795EA95D1F737
:102DF0002C813D814E815F81820F931FA41FB51FDF
:102E0000C80ED91EEA1EFB1E022C04C0CC0CDD1C11
:102E1000EE1CFF1C0A94D2F732E0C30ED11CE11C59
:102E2000F11CF2E0F594E794D794C794FA95D1F7A2
:102E30002E893F89488D598D2C193D094E095F090E
:102E400069897A898B899C890E94179397FD0BC0A9
:102E5000660F771F881F991FA50194010E945B933D
:102E600069017A010AC0A50194010E945B9369017E
:102E70007A01CC0CDD1CEE1CFF1C9927F7FC9A95FF
:102E80008F2D7E2D6D2D9B01AC010E9417939B0110
:102E9000AC01AEEDBBE00E94CA934C01BB2497FC91
:102EA000B094AB2CA3E4B3EEA70196010E94D89393
:102EB000BB2797FDB095AB2F880E991EAA1EBB1E8F
:102EC0004FEC840E4EE0941EA11CB11C44E0B5945E
:102ED000A794979487944A95D1F7C80CD91CEA1CFB
:102EE000FB1C4C0C5D1C6E1C7F1C1F5FBFCE112396
:102EF00081F0212F30E040E050E0C301B2010E9498
:102F00005B932093AA1C3093AB1C4093AC1C509352
:102F1000AD1C5D89552389F16091AA1C7091AB1C91
:102F20008091AC1C9091AD1C6115710581059105D6
:102F300021F10E94509020E836EE45EC57E40E94C3
:102F40009C8F21E03EED42E45EE30E94B5929B013E
:102F5000AC0160E070E080E89FE30E94B88E2BE453
:102F60003AE34DEB57E30E949C8F6093AE1C709345
:102F7000AF1C8093B01C9093B11C6C960FB6F89464
:102F8000DEBF0FBECDBFDF91CF911F910F91FF909C
:102F9000EF90DF90CF90BF90AF909F908F907F90F9
:102FA0006F905F904F903F902F9008950F931F93D5
:102FB000CF93DF9300D000D000D0CDB7DEB78E0125
:102FC0000F5F1F4F86E0F80111928A95E9F7809113
:102FD000A41B811113C040E061E386EA0E948F13B5
:102FE0004AE06CE286EA0E948F1381E08093A41B82
:102FF0006CE77EE380E090E00E94776648E06DE257
:1030000086EA0E948F136CE77EE380E090E00E94E6
:10301000776626E0A80162E386EA0E94A61347E0ED
:103020006DE286EA0E948F138A8190E0982F8827AC
:103030002981822B90939F1B80939E1B2C8130E0D3
:10304000322F22274B81242B3093A11B2093A01BCE
:103050004E8150E0542F44276D81462B5093A31B83
:103060004093A21B5F934F933F932F939F938F9314
:1030700087E094E09F938F930E94359A0FB6F8945F
:10308000DEBF0FBECDBF26960FB6F894DEBF0FBED3
:10309000CDBFDF91CF911F910F910895CF92DF9215
:1030A000EF92FF920F931F93CF93DF93CDB7DEB7CD
:1030B0002A970FB6F894DEBF0FBECDBF8E010F5F0B
:1030C0001F4F86E0F80111928A95E9F741E062E02E
:1030D0008CE30E948F1348E560E08CE30E948F131D
:1030E00062E174E380E090E00E94776626E0A80148
:1030F00063E08CE30E94A61343E062E08CE30E944D
:103100008F13098110E0102F00278A81082BEEE72A
:10311000FBE111830083EB80F12CFE2CEE248C81EB
:10312000E82AF382E282CD80D12CDC2CCC248E8163
:10313000C82AD582C482B801012E000C880B990BD5
:103140000E9450909B01AC01B7010F2C000C880B22
:10315000990B2F83388749875A870E9450902F8177
:10316000388549855A850E94388F20EE3EE245E633
:1031700052E40E94489220E030E044E353E40E948D
:10318000B98E9F938F937F936F93DF92CF92FF922D
:10319000EF921F930F9385E194E09F938F930E948A
:1031A000359A0FB6F894DEBF0FBECDBF2A960FB684
:1031B000F894DEBF0FBECDBFDF91CF911F910F916D
:1031C000FF90EF90DF90CF900895CF93DF93EC01C5
:1031D00088819981009759F1873F914121F01982A7
:1031E000188283E06FC08BE59AE00E94F05D892B26
:1031F00041F18091410A9091420AA091430AB09115
:10320000440A93FD20C08091410A9091420AA09106
:10321000430AB091440A94FD47C08091410A9091BD
:10322000420AA091430AB091440A95FD44C060E867
:1032300070E08BE59AE00E94C95D87EF91E1998388
:10324000888381E03FC08091CA2B82FFDCCF21E0E0
:1032500048E061E083E00E945B158091B11C8F9390
:103260008091B01C8F938091AF1C8F938091AE1C86
:103270008F938091AD1C8F938091AC1C8F93809124
:10328000AB1C8F938091AA1C8F9383E990E19F934D
:103290008F930E94499A8DB79EB70A960FB6F894FD
:1032A0009EBF0FBE8DBFAFCF8091CA2B83FFB5CF1E
:1032B0000E94D617B2CF8091CA2B84FFB8CF0E944C
:1032C0004E18B5CFDF91CF910895CF93C82F8CEED4
:1032D0000E94F5668C2F0E94FF6665E375E080E032
:1032E00090E00E9477668DEE0E94F5660E9410675E
:1032F000C82F0E941A672C2F30E0322F2227A901F5
:10330000482BCA01CF9108950F931F93CF93DF935A
:10331000C82F8CEE0E94F5668C2F0E94FF6662E13A
:1033200074E380E090E00E9477668CEE0E94F56680
:1033300080E00E94FF6665E375E080E090E00E9417
:1033400077668DEE0E94F5660E941067C82F0E9476
:103350001067D82F0E941A674D2F50E060E070E090
:10336000762F652F542F44276C2B8A019B01082B45
:10337000C901B801DF91CF911F910F9108952F924C
:103380003F924F925F926F927F928F929F92AF92F5
:10339000BF92CF92DF92EF92FF920F931F93CF9342
:1033A000DF93CDB7DEB7CB54D1090FB6F894DEBFAB
:1033B0000FBECDBF8091000290910102892BD1F107
:1033C00010920102109200028CEE0E94F5668EE1CE
:1033D0000E94FF666BE17EE480E090E00E947766E9
:1033E00082EA0E9465199093500A80934F0A84EAFA
:1033F0000E94651990934E0A80934D0A86EA0E94B6
:10340000651990934C0A80934B0A88EA0E946519CB
:1034100090934A0A8093490A8AEA0E946519909318
:10342000480A8093470A8CEA0E9465199093460ADD
:103430008093450A88E40E9484196DAB7EAB8FAB04
:1034400098AF88E50E9484194B015C018091470A7E
:103450009091480A8C0120E030E040E050E0BA0151
:1034600022968FAF229723961FAF239724962FAFD4
:10347000249725963FAF259726964FAF26972796F8
:103480005FAF279728966FAF289729967FAF299728
:103490009C0140E050E060E070E080E090E008E0F7
:1034A0000E9438950E94F1943901B42FA52FF62F70
:1034B000E72F8C019401A50160E070E080E090E0CE
:1034C0005301CB2EDA2EEF2EFE2E0E946F952CA3E9
:1034D0003BA34B83252E362E472E582E792E632D57
:1034E000742D852D972D315041095F4F6F4F7F4FC0
:1034F0008F4F9F4F88248394912C21153F4F4F4F1E
:103500005140610571058105910509F010F4812C88
:10351000912C9A8289820091450A1091460A58019D
:10352000C12CD12CE12CF12C00E010E02CA13BA10E
:103530004B81522D632D742D852D972D0E94DD9387
:10354000F22E032F142FB52FF62FE72FD82EE92EAA
:10355000A0E00E94969584F42150310940485F4FC5
:103560006F4F7F4F8F4F9F4FF22E032F142FB52F8A
:10357000F62FE72FD82EE92E2F2D302F412F5B2F3E
:103580006F2F7E2F8D2D9E2D07E10E9451952B8F41
:103590003C8F4D8F5E8F6F8F78A389A39AA32053A2
:1035A000384F4F4F5F4F6F4F7F4F8F4F9F4F2B8B3A
:1035B0003C8B4D8B5E8B6F8B788F898F9A8F2056CB
:1035C000304F4F4F5F4F6F4F7F4F8F4F9F4F243D77
:1035D000304341055105610571058105910529F0CB
:1035E00020F0F4013196FA83E98380904D0A90909F
:1035F0004E0A940140E050E060E070E080E090E02E
:1036000000E10E9438952C833D834E835F83662EB4
:1036100078874C014091490A50914A0AACA0BBA05E
:10362000CB80D22CE32CF42C052D172D9A0140E0F1
:1036300050E060E070E080E090E00E94DD93F22EC8
:10364000032F142FB52FF62FE72FD82EE92EA0E049
:103650000E9496955CF4AFE70E947895F22E032FB6
:10366000142FB52FF62FE72FD82EE92E2F2D302F20
:10367000412F5B2F6F2F7E2F8D2D9E2D07E00E94F7
:10368000519559016A017B018C012C813D814E814C
:103690005F81662D7885C4010E946F952C833D83E0
:1036A0004E835F8368877E878F87988B2E5F3F4F1F
:1036B000434051096E4F7F4F8F4F9F4F223031054E
:1036C000494F5F4F644071058105910539F030F035
:1036D00009811A810F5F1F4F1A83098360914F0A76
:1036E0007091500A80E090E020E030E840E050E047
:1036F0000E94369429873A874B875C87662E7D87A0
:103700004C0140914B0A50914C0AACA0BBA0CB801D
:10371000D22CE32CF42C052D172D9A0140E050E01B
:1037200060E070E080E090E00E94DD93F22E032FD5
:10373000142FB52FF62FE72FD82EE92EA0E00E94E8
:10374000969584F421503F4F4F4F5F4F6F4F7F4FFF
:103750008F4F9F4FF22E032F142FB52FF62FE72FE9
:10376000D82EE92E2F2D302F412F5B2F6F2F7E2F3C
:103770008D2D9E2D08E00E94519559016A017B0113
:103780008C0129853A854B855C85662D7D85C40134
:103790000E946F9529873A874B875C876D87798B65
:1037A0008A8B692E2F5F3F4F414051096109710992
:1037B00081099109213030484C4F5F4761407105C4
:1037C0008105910539F030F029813A812F5F3F4F13
:1037D0003A8329832B893C894D895E896F89788D4D
:1037E000898D9A8D2F3C3740410551056105710542
:1037F0008105910511F00CF0A4C1ACA0BBA0CB8059
:10380000D22CE32CF42C052D172D95014C2D522D87
:10381000632D742D852D972D0E94DD93A12CB12C45
:10382000C12CE0E8DE2EE12CF12C00E010E00E943B
:10383000639429AF3AAF4BAF5CAF6DAF7EAF8FAF44
:1038400021969FAF2197AB8CBC8CCD8CDE8CEF8CFE
:10385000F8A009A11AA19501A601B701C8010E940B
:10386000DD9359016A017B01E82F192F02E00E94C4
:1038700038950E2F0E946F957901142F552EF62F33
:10388000E72F6C01922EAF2CB42E052F462EB72FAA
:10389000782E8D2CA0E00E9496955CF4A1E00E9409
:1038A0007895922EA32EB42E052F462EB72F782E64
:1038B000892E292D3A2D4B2D502F642D7B2F872DAE
:1038C000982D01E00E9451952AA7732E4A012C964B
:1038D0006FAF2C972B967FAF2B978BA79CA72B8333
:1038E0003BA34CA39DA26EA37FA388A799A7B52D48
:1038F0009701412F552D6F2F7E2FC601A0E00E940A
:1039000096954CF4A3E00E9478957901142FB52F79
:10391000F62FE72F6C019701412F5B2F6F2F7E2F22
:10392000C60102E00E9451952DA73EA74FA758ABB4
:1039300069AB7AAB8BAB9CAB2901B42FA52F229638
:103940006FAF2297F72F1C012B893C894D895E8927
:103950006F89788D898D9A8D24323A4F4F4F5F4F02
:103960006F4F7F4F8F4F9F4F0CF08BC02B8D3C8D37
:103970004D8D5E8D6F8D78A189A19AA12455324F0E
:103980004F4F5F4F6F4F7F4F8F4F9F4F59016A01CE
:103990007B018C010E94DD9319012A01B62FA72F0C
:1039A000FC0103E00E94389551016201EB2EFA2ED2
:1039B0008F010E94849559016A017B018C012AA51F
:1039C000372DA4012C966FAD2C972B967FAD2B979E
:1039D0008BA59CA50E946F952B833BA34CA35DA355
:1039E0006EA37FA388A799A79101A2016B2F7A2FBD
:1039F000CF0102E00E94389551016201EB2EFA2EB0
:103A00008F010E94849502E00E9438950E2F0E943B
:103A10008495122FD32EE42EB52FF62FE72FF82EF4
:103A2000092FA0E00E9496955CF4A1E00E94789591
:103A3000122FD32EE42EB52FF62FE72FF82E092FB5
:103A4000212F3D2D4E2D5B2F6F2F7E2F8F2D902FF1
:103A500001E00E94519559016A017B018C012DA55D
:103A60003EA54FA558A969A97AA98BA99CA90E942E
:103A70006F952901B42FA52F22966FAF2297F72FAC
:103A80001C012C813D814E815F8168857E858F85FB
:103A90009889AB80BBA0CCA0DDA0EEA0FFA008A5BC
:103AA00019A50E9484952C833D834E835F8368878C
:103AB0007E878F87988B29853A854B855C856D85B8
:103AC00079898A89962D5201CB2EDA2E2296EFAC77
:103AD0002297FF2E81010E94849529873A874B8780
:103AE0005C876D87798B8A8B692E2B893C894D8900
:103AF0005E896F89788D898D9A8DA9ACBAACCBAC73
:103B0000DCACEDACFEAC0FAD21961FAD21970E9451
:103B100084952056304F4F4F5F4F6F4F7F4F8F4FE1
:103B20009F4F243D304341055105610571058105D5
:103B3000910539F030F009811A810F5F1F4F1A8308
:103B400009834DA95EA96FA978AD9A01AB0160E028
:103B500070E0CB0122962FAF229723963FAF239799
:103B600024964FAF249725965FAF259726966FAF83
:103B7000269727967FAF279728968FAF2897299665
:103B80009FAF2997A984BA84CB84DC84ED84F9881B
:103B90000A89162D60E070E080E090E00E94DD93DD
:103BA000122FD32EE42EB52FF62FE72FF82E092F44
:103BB000A0E00E94969584F421503109404E5F4F59
:103BC0006F4F7F4F8F4F9F4F122FD32EE42EB52F65
:103BD000F62FE72FF82E092F212F3D2D4E2D5B2F8D
:103BE0006F2F7E2F8F2D902F05E10E945195AC8075
:103BF000BD80CE80DF80E884FE840F8518890E9416
:103C00008495122FD32EE42EB52FF62FE72FF82E02
:103C1000092FA0E00E94969584F4215030484F4F20
:103C20005F4F6F4F7F4F8F4F9F4F122FD32EE42E3A
:103C3000B52FF62FE72FF82E092F212F3D2D4E2DD2
:103C40005B2F6F2F7E2F8F2D902F0FE00E945195AD
:103C500039014A015B016C0179018A011B012C01C8
:103C6000285E3340410951096109710981099109AF
:103C7000283D304D41405105610571058105910593
:103C800031F028F0E981FA813196FA83E9830E94C4
:103C9000F76629813A81232B51F09301A401B501E4
:103CA000C6010E94F19479018A011B012C01970140
:103CB000A801B101C2010E94489020E030E048EC28
:103CC00052E40E949C8FC55BDF4F0FB6F894DEBFB5
:103CD0000FBECDBFDF91CF911F910F91FF90EF905D
:103CE000DF90CF90BF90AF909F908F907F906F901C
:103CF0005F904F903F902F9008954F925F926F92F8
:103D00007F928F929F92AF92BF92CF92DF92EF926B
:103D1000FF922B013C0169017A0123EC35EF4CE85D
:103D200051E4C701B6010E9448924B015C0128EBA7
:103D30003EE143E753E4C701B6010E94B98E9B01FF
:103D4000AC01C501B4010E949C8F0E9416904B01EA
:103D50005C0120E030E048EC52E4C301B2010E9473
:103D60009C8F21E835E943EC50E40E944892A5017C
:103D700094010E9448924B015C0123E333E948E837
:103D800053E4C701B6010E94B98E9B01AC01C50185
:103D9000B4010E949C8F23E333EB48E553E40E9477
:103DA0004892FF90EF90DF90CF90BF90AF909F90A0
:103DB0008F907F906F905F904F9008954F925F9299
:103DC0006F927F928F929F92AF92BF92CF92DF922B
:103DD000EF92FF9269017A010E94BC9120E030E0ED
:103DE00040E050E40E94B88E22E93CE54EED5EE3EF
:103DF0000E949C8F4B015C0123EC35EF4CE851E4B1
:103E0000C701B6010E9448922B013C0128EB3EE11C
:103E100043E753E4C701B6010E94B98E9B01AC0190
:103E2000C301B2010E949C8F9B01AC01C501B4018A
:103E30000E94B98E6B017C0128EB3EE143E753E41D
:103E40000E9448924B015C01A701960163EC75EF5B
:103E50008CE891E40E94B88E9B01AC01C501B401CD
:103E60000E949C8FFF90EF90DF90CF90BF90AF901B
:103E70009F908F907F906F905F904F9008954F929A
:103E80005F926F927F928F929F92AF92BF92CF92EA
:103E9000DF92EF92FF922B013C0169017A0123EC42
:103EA00035EF4CE851E4C701B6010E9448924B013E
:103EB0005C0128EB3EE143E753E4C701B6010E94F1
:103EC000B98E9B01AC01C501B4010E949C8F0E9478
:103ED00016904B015C0120E030E048EC52E4C30155
:103EE000B2010E949C8FA50194010E94489220E09B
:103EF00030E040E251E40E94B88E24EE38E34EE018
:103F00005FE30E9448929B01AC01C701B6010E9489
:103F1000B98EFF90EF90DF90CF90BF90AF909F90C1
:103F20008F907F906F905F904F90089580E80E94EF
:103F3000F56681110DC08EEF0E94FF66811108C0E9
:103F40006BE17EE480E090E00E9477660C94F76677
:103F50000E94F7668091DC2F9091DD2FA091DE2FDB
:103F6000B091DF2F0196A11DB11D8093DC2F90939E
:103F7000DD2FA093DE2FB093DF2F0895FC01DC012D
:103F8000AC014E5F5F4F90E031E38D91982788E060
:103F9000292F220F97FF03C0922F932701C0922F42
:103FA0008150B1F7A417B50781F721E030E0828195
:103FB000981711F020E030E0C9010895DF92EF92E8
:103FC000FF920F931F93CF93DF930E94961F80E879
:103FD0000E94F56681116DC08AEF0E94FF66811113
:103FE00068C08FE00E94FF66811163C065E375E0E1
:103FF00080E090E00E94776681E80E94F56681117A
:1040000058C00E941067D82F0E9410670E94106746
:10401000182F0E9410670E941067082F0E941067D7
:104020000E941A67F82E80E80E94F566811141C04F
:104030008CEF0E94FF6681113CC089EC0E94FF66F4
:10404000811137C065E375E080E090E00E947766FB
:1040500081E80E94F5660E941067E82E0E941067B2
:10406000D82E0E9410670E941067C82F0E941A67FE
:104070001F92DF921F92EF921F92FF921F920F9357
:104080001F921F931F92DF931F928F931F92CF93C4
:104090008AE294E09F938F930E94359A0E94F7667C
:1040A0008DB79EB742960FB6F8949EBF0FBE8DBFD8
:1040B00017C00E94F7668091DC2F9091DD2FA091B0
:1040C000DE2FB091DF2F0196A11DB11D8093DC2F53
:1040D0009093DD2FA093DE2FB093DF2F0E94961FC9
:1040E00020E030E040E050E060E070E080E090E010
:1040F000DF91CF911F910F91FF90EF90DF90089586
:10410000EF92FF920F931F93CF93DF9300D01F92F4
:10411000CDB7DEB78C0180E80E94F566811154C0EE
:104120000115110551F085EE0E94FF6681114CC00A
:1041300061E077E980E090E009C083EE0E94FF66CD
:10414000811142C069E97AEB81E090E00E947766D4
:1041500081E80E94F566811137C00E941067E82E41
:1041600089830E941067F82E8A830E941A678B83C6
:104170000E94F766CE0101960E94BE1F892B21F195
:104180006F2D70E07E296C7F80E090E0012B69F05C
:104190000E944E9020E030E04AEF5AE30E9448929D
:1041A00020E030E040EC50E40CC00E944E9022E54C
:1041B00038EB4FE25BE30E94489226E636E64BE39B
:1041C00052E40E94B88E1BC00E94F7668091DC2FDB
:1041D0009091DD2FA091DE2FB091DF2F0196A11DD0
:1041E000B11D8093DC2F9093DD2FA093DE2FB09331
:1041F000DF2F0E94961F60EF7FEF89E794E40F9016
:104200000F900F90DF91CF911F910F91FF90EF9042
:1042100008950F931F93CF93DF93729A8091620258
:1042200083FF08C08EE40E949A66811165C0C0E5D4
:10423000D0E009C0C0E5D0E087EE93E00E94290AF3
:104240002197D1F7EFCF87EE93E00E94290A2197BB
:10425000D1F78FE40E949A660E941067D82FDF730F
:104260000E941067082F0E941067C82F0E941A67CB
:10427000182F0E94F7668091620283FF72986D2F5B
:1042800070E0762F6627600F711D80E090E00E943D
:104290004E9020E134E048EC5BE30E94489260934A
:1042A000BE277093BF278093C0279093C1276C2FA0
:1042B00070E0762F6627610F711D7695679576956C
:1042C000679580E090E00E944E9024EA3CEF44E243
:1042D0005CE30E94489220E030E040E252E40E9419
:1042E000B88E60939F347093A0348093A1349093E0
:1042F000A23480E090E002C081E090E0DF91CF91B5
:104300001F910F9108957298729A8EE40E949A6696
:1043100080EA0E94FF6680E00E94FF6680E00E94C3
:10432000FF668FE40E949A660E9410678EE40E94E6
:104330009A6680E80E94FF6680E00E94FF6680E047
:104340000E94FF660E94F76680E090E0089582EC8C
:104350009FE09F938F930E94499A80917D020F90D6
:104360000F90882361F01F928F938FEB9FE09F93B4
:104370008F930E94499A0F900F900F900F9008957D
:104380008AE99FE09F938F930E94499A82E79FE07A
:104390009F938F930E94499A8BE49FE09F938F9302
:1043A0000E94499A80E19FE09F938F930E94499ACF
:1043B00084ED9EE09F938F930E94499A82EA9EE04B
:1043C0009F938F930E94499A86E69EE09F938F93D6
:1043D0000E94499A80E49EE09F938F930E94499A9D
:1043E0008AE09EE09F938F930E94499A8091CA2B06
:1043F0009091CB2B827091702DB73EB72E5E3F4FC0
:104400000FB6F8943EBF0FBE2DBF892B41F08AED49
:104410009DE09F938F930E94499A0F900F908EEA90
:104420009DE09F938F930E94499A82E79DE09F931E
:104430008F930E94499A89E49DE09F938F930E94F5
:10444000499A8DE19DE09F938F930E94499A8EEE49
:104450009CE09F938F930E94499A8CEB9CE09F93E2
:104460008F930E94499A8BE89CE09F938F930E94C0
:10447000499A81E59CE09F938F930E94499A8BE132
:104480009CE09F938F930E94499A8BEE9BE09F93B1
:104490008F930E94499A8FEB9BE09F938F930E948A
:1044A000499A80E99BE09F938F930E94499A87E500
:1044B0009BE09F938F930E94499A8EE19BE09F938C
:1044C0008F930E94499A87EE9AE09F938F930E9460
:1044D000499A89EB9AE09F938F930E94499A8DB7EE
:1044E0009EB780960FB6F8949EBF0FBE8DBF85E82D
:1044F0009AE09F938F930E94499A84E59AE09F9354
:104500008F930E94499A85E29AE09F938F930E942D
:10451000499A86EF99E09F938F930E94499A8FEC76
:1045200099E09F938F930E94499A89E999E09F931C
:104530008F930E94499A83E699E09F938F930E94FC
:10454000499A8DE299E09F938F930E94499A84E063
:1045500099E09F938F930E94499A8CEC98E09F93E7
:104560008F930E94499A81EA98E09F938F930E94CB
:10457000499A2DB73EB72A5E3F4F0FB6F8943EBF1B
:104580000FBE2DBF089589E594E00C94719A4F9267
:104590005F926F927F928F929F92AF92BF92CF92D3
:1045A000DF92EF92FF92CF93DF93CDB7DEB72897DC
:1045B0000FB6F894DEBF0FBECDBF8091D02F909183
:1045C000D12FA091D22FB091D32F89839A83AB831F
:1045D000BC834090D02F5090D12F6090D22F7090FC
:1045E000D32F8091D02F9091D12FA091D22FB09125
:1045F000D32F8D839E83AF83B8876091D02F709126
:10460000D12F8091D22F9091D32F2CE3822E912CF9
:10461000A12CB12CA50194010E945B937F936F9311
:1046200030E1C32E3EE0D32EE12CF12C6D817E8152
:104630008F819885A70196010E945B93A501940143
:104640000E945B933F932F9340E8842E41E5942E84
:10465000AA24A394B12CC301B201A50194010E9424
:104660005B93A70196010E945B933F932F9369810F
:104670007A818B819C81A50194010E945B933F9379
:104680002F938BE798E09F938F930E94499A0FB6E0
:10469000F894DEBF0FBECDBF28960FB6F894DEBFEC
:1046A0000FBECDBFDF91CF91FF90EF90DF90CF9005
:1046B000BF90AF909F908F907F906F905F904F9042
:1046C0000895E0E6FDE3808191818234924479F09F
:1046D000E056FD43FF93EF938DE598E09F938F9312
:1046E0000E94499A0F900F900F900F9008953A965C
:1046F000E53F81E4F80738F30895CF93DF93EC01A9
:104700008C9A0E94A50C9F938F937F936F9381E562
:1047100098E09F938F930E94499A0F900F900F906B
:104720000F900F900F90209719F00E94B60D08C0BF
:104730008FE498E09F938F930E94499A0F900F9077
:1047400081E00E94570C20918202309183024091B7
:104750008402509185020E9448929F938F937F9389
:104760006F9383E498E09F938F930E94499A0F90F0
:104770000F900F900F900F900F90209719F00E94BC
:10478000B60D08C081E498E09F938F930E94499AE8
:104790000F900F9082E00E94570C20917E02309182
:1047A0007F0240918002509181020E9448929F9323
:1047B0008F937F936F9385E398E09F938F930E94ED
:1047C000499A0F900F900F900F900F900F90209795
:1047D00019F00E94B60D08C083E398E09F938F9371
:1047E0000E94499A0F900F9083E00E94570C9F936C
:1047F0008F937F936F9384E298E09F938F930E94AF
:10480000499A8C980F900F900F900F900F900F90E7
:10481000209719F00E94B60D08C082E298E09F939D
:104820008F930E94499A0F900F908091CA2B87FF17
:1048300083C021E042E161E080ED0E9461689F93C6
:104840008F937F936F9385E198E09F938F930E945E
:10485000499A0F900F900F900F900F900F90209704
:1048600019F00E94B60D08C083E198E09F938F93E2
:104870000E94499A0F900F9021E042E162E080EDA2
:104880000E9461689F938F937F936F9386E098E077
:104890009F938F930E94499A0F900F900F900F90C3
:1048A0000F900F90209719F00E94B60D08C084E079
:1048B00098E09F938F930E94499A0F900F9021E068
:1048C00042E163E080ED0E9461689F938F937F9344
:1048D0006F9387EF97E09F938F930E94499A0F9071
:1048E0000F900F900F900F900F90CD2B19F00E940A
:1048F000B60D08C085EF97E09F938F930E94499A69
:104900000F900F9021E042E164E080ED0E94616829
:104910009F938F937F936F9388EE97E09F938F93EE
:104920000E94499A0F900F900F900F900F900F9048
:10493000DF91CF910C94B60DCD2BD1F3DF91CF91B8
:1049400008950F931F93CF93DF93882389F049E055
:1049500050E06FEF70E083E994E30E94839949E0AF
:1049600050E06EE070E083E994E30E944D9D13C037
:10497000C3E9D4E303EE17E089911F928F931F934D
:104980000F930E94499A0F900F900F900F9084E31D
:10499000CB39D80789F7DF91CF911F910F910C94F4
:1049A000B60D882311F0299A08952998089588232F
:1049B00011F02A9A08952A980895882311F02B9AC5
:1049C00008952B980895CF92DF92EF92FF92CF93A4
:1049D000DF936B017C0160FF11C086E994E09F9337
:1049E0008F9387ED9FE09F938F930E94499A0F903A
:1049F0000F900F900F9081E090E002C080E090E077
:104A0000C1FE09C0EC0121964BE959E06BE974E065
:104A10000E941C12CE01C2FE09C0EC0121964BE996
:104A200059E063EA74E00E941C12CE01C3FE09C083
:104A3000EC0121964BE959E06BEA74E00E941C12EC
:104A4000CE01C4FE09C0EC0121964BE959E066E1B4
:104A500076E00E941C12CE01C5FE09C0EC01219631
:104A60004BE959E06FEA74E00E941C12CE01C6FEC9
:104A700009C0EC0121964BE959E063EB74E00E9418
:104A80001C12CE01C7FE09C0EC0121964BE959E08A
:104A900069EB74E00E941C12CE01D0FE09C0EC014B
:104AA00021964BE959E061EC74E00E941C12CE01A2
:104AB000D1FE09C0EC0121964BE959E069EC74E0A4
:104AC0000E941C12CE01D2FE09C0EC0121964BE9D6
:104AD00059E06DEC74E00E941C12CE012091CA2BAB
:104AE0003091CB2B24703270232B59F0D3FE09C0A8
:104AF000EC0121964BE959E063ED74E00E941C1231
:104B0000CE012091CA2B23FF0BC0D4FE09C0EC01BB
:104B100021964BE959E068ED74E00E941C12CE0129
:104B20002091CA2B24FF0BC0D5FE09C0EC012196B1
:104B30004BE959E06EED74E00E941C12CE01D6FEE6
:104B400009C0EC0121964BE959E066EE74E00E9441
:104B50001C12CE01D7FE09C0EC0121964BE959E0A9
:104B600061EF74E00E941C12CE01E0FE0CC04BE924
:104B700059E062E075E0DF91CF91FF90EF90DF9018
:104B8000CF900C941C12CD28CE28CF2841F48EED66
:104B900097E09F938F930E94499A0F900F90DF9117
:104BA000CF91FF90EF90DF90CF900895CF92DF925A
:104BB000EF92FF92CF93DF93EC01C12CD12C7601C1
:104BC000209709F4A3C069ED77E0CE010E946299B5
:104BD000892B11F46894C0F861ED77E0CE010E9452
:104BE0006299892B11F46894C1F869EC77E0CE01E1
:104BF0000E946299892B11F46894C2F865EC77E001
:104C0000CE010E946299892B11F46894C3F862EC7A
:104C100077E0CE010E946299892B11F46894C4F860
:104C20006EEB77E0CE010E946299892B11F46894B3
:104C3000C5F868EB77E0CE010E946299892B11F4E8
:104C40006894C6F860EB77E0CE010E946299892BE8
:104C500011F46894C7F868EA77E0CE010E9462997F
:104C6000892B11F46894D0F864EA77E0CE010E94B1
:104C70006299892B11F46894D1F86EE977E0CE013E
:104C80000E946299892B11F46894D2F869E977E05F
:104C9000CE010E946299892B11F46894D3F863E9DC
:104CA00077E0CE010E946299892B11F46894D4F8C0
:104CB0006BE877E0CE010E946299892B11F4689429
:104CC000D5F860E877E0CE010E946299892B11F453
:104CD0006894D6F86FE677E0CE010E946299892B3E
:104CE00011F46894D7F86AE677E0CE010E946299E1
:104CF000892B11F46894E0F860917B0270917C023A
:104D000080E090E00E947699EC015ACFC701B6018D
:104D1000DF91CF91FF90EF90DF90CF900895AF9209
:104D2000BF92CF92DF92EF92FF920F931F93CF9398
:104D3000DF93122FD32FC42F052FF62EC72ED82E78
:104D4000E92E217030E040E050E060E070E080E06B
:104D500090E0A0E00E94969589F087E095E09F930F
:104D60008F9387ED9FE09F938F930E94499A0F90B6
:104D70000F900F900F90E1E0F0E002C0E0E0F0E073
:104D80008091CA2B80FF19C0212F247030E040E0B1
:104D900050E060E070E080E090E0A0E00E94969536
:104DA00061F05F018FEFA81AB80A4BE959E06BE098
:104DB00075E0CF010E941C12F501212F227030E016
:104DC00040E050E060E070E080E090E0A0E00E9411
:104DD000969561F05F018FEFA81AB80A4BE959E088
:104DE0006FE075E0CF010E941C12F501212F2870A1
:104DF00030E040E050E060E070E080E090E0A0E073
:104E00000E94969561F05F018FEFA81AB80A4BE9EE
:104E100059E067E275E0CF010E941C12F501212FD5
:104E2000207130E040E050E060E070E080E090E031
:104E3000A0E00E94969561F05F018FEFA81AB80A72
:104E40004BE959E062E175E0CF010E941C12F501C7
:104E5000212F207230E040E050E060E070E080E020
:104E600090E0A0E00E94969561F05F018FEFA81A94
:104E7000B80A4BE959E065E175E0CF010E941C12C8
:104E8000F501212F207430E040E050E060E070E058
:104E900080E090E0A0E00E94969561F05F018FEFC6
:104EA000A81AB80A4BE959E06BE175E0CF010E94FE
:104EB0001C12F501212F207830E040E050E060E046
:104EC00070E080E090E0A0E00E94969561F05F01C4
:104ED0008FEFA81AB80A4BE959E061E275E0CF01FB
:104EE0000E941C12F50120E03D2F317040E050E09F
:104EF00060E070E080E090E0A0E00E94969561F0B4
:104F00005F018FEFA81AB80A4BE959E064E275E037
:104F1000CF010E941C12F50120E03D2F327040E0CD
:104F200050E060E070E080E090E0A0E00E949695A4
:104F300061F05F018FEFA81AB80A4BE959E069E206
:104F400075E0CF010E941C12F50120E03D2F347066
:104F500040E050E060E070E080E090E0A0E00E947F
:104F6000969561F05F018FEFA81AB80A4BE959E0F6
:104F700060E375E0CF010E941C12F50120E03D2F97
:104F8000387040E050E060E070E080E090E0A0E049
:104F90000E94969561F05F018FEFA81AB80A4BE95D
:104FA00059E063E375E0CF010E941C12F50120E097
:104FB0003D2F307140E050E060E070E080E090E034
:104FC000A0E00E94969561F05F018FEFA81AB80AE1
:104FD0004BE959E068E375E0CF010E941C12F5012E
:104FE00020E03D2F307240E050E060E070E080E073
:104FF00090E0A0E00E94969561F05F018FEFA81A03
:10500000B80A4BE959E06FE375E0CF010E941C122A
:10501000F50120E030E040E050E06F2D647070E07A
:1050200080E090E0A0E00E94969561F05F018FEF34
:10503000A81AB80A4BE959E066E475E0CF010E946E
:105040001C12F5018091CA2B81FF19C020E03D2F71
:10505000307440E050E060E070E080E090E0A0E07C
:105060000E94969561F05F018FEFA81AB80A4BE98C
:1050700059E06AE475E0CF010E941C12F5018091AD
:10508000CA2B9091CB2B90FF19C020E030E040E07C
:10509000502F507160E070E080E090E0A0E00E944E
:1050A000969561F05F018FEFA81AB80A4BE959E0B5
:1050B0006DE475E0CF010E941C12F5018091CA2BAE
:1050C0009091CB2B90FF19C020E030E040E0502FB2
:1050D000507260E070E080E090E0A0E00E94969561
:1050E00061F05F018FEFA81AB80A4BE959E060E55B
:1050F00075E0CF010E941C12F5018091CA2B90919E
:10510000CB2B90FF19C020E030E040E0502F5074CE
:1051100060E070E080E090E0A0E00E94969561F091
:105120005F018FEFA81AB80A4BE959E066E575E010
:10513000CF010E941C12F50120E03D2F307840E0A5
:1051400050E060E070E080E090E0A0E00E94969582
:1051500061F05F018FEFA81AB80A4BE959E061E6E8
:1051600075E0CF010E941C12F50120E030E04C2FC9
:10517000417050E060E070E080E090E0A0E00E94CC
:10518000969561F05F018FEFA81AB80A4BE959E0D4
:1051900066E675E0CF010E941C12F50120E030E0C8
:1051A0004C2F427050E060E070E080E090E0A0E0C2
:1051B0000E94969561F05F018FEFA81AB80A4BE93B
:1051C00059E069E675E0CF010E941C12F50120E06C
:1051D00030E04C2F447050E060E070E080E090E000
:1051E000A0E00E94969561F05F018FEFA81AB80ABF
:1051F0004BE959E06CE675E0CF010E941C12F50105
:105200008091CA2B87FF19C020E030E04C2F4870F6
:1052100050E060E070E080E090E0A0E00E949695B1
:1052200061F05F018FEFA81AB80A4BE959E06FE609
:1052300075E0CF010E941C12F5018091CA2B87FFF7
:1052400019C020E030E04C2F407150E060E070E089
:1052500080E090E0A0E00E94969561F05F018FEF02
:10526000A81AB80A4BE959E063E775E0CF010E943C
:105270001C12F5018091CA2B87FF19C020E030E095
:105280004C2F407250E060E070E080E090E0A0E0E1
:105290000E94969561F05F018FEFA81AB80A4BE95A
:1052A00059E067E775E0CF010E941C12F50180917B
:1052B000CA2B87FF19C020E030E04C2F407450E02B
:1052C00060E070E080E090E0A0E00E94969561F0E0
:1052D0005F018FEFA81AB80A4BE959E06BE775E058
:1052E000CF010E941C12F5018091CA2B82FF19C0C8
:1052F00020E030E04C2F407850E060E070E080E04B
:1053000090E0A0E00E94969561F05F018FEFA81AEF
:10531000B80A4BE959E069EA76E0CF010E941C1215
:10532000F5018091CA2B82FF19C020E030E040E0F7
:10533000502F517060E070E080E090E0A0E00E94AB
:10534000969561F05F018FEFA81AB80A4BE959E012
:105350006FE775E0CF010E941C12F5018091CA2B06
:105360009091CB2B90FF19C020E030E040E0502F0F
:10537000527060E070E080E090E0A0E00E949695BE
:1053800061F05F018FEFA81AB80A4BE959E062E8B3
:1053900075E0CF010E941C12F5018091CA2B9091FB
:1053A000CB2B90FF19C020E030E040E0502F54702C
:1053B00060E070E080E090E0A0E00E94969561F0EF
:1053C0005F018FEFA81AB80A4BE959E06AE875E067
:1053D000CF010E941C12F5018091CA2B9091CB2B1A
:1053E00091FF1EC020E030E040E0502F587060E098
:1053F00070E080E090E0A0E00E94969589F04BE993
:1054000059E063E975E0CF01DF91CF911F910F91D2
:10541000FF90EF90DF90CF90BF90AF900C941C1254
:10542000212F3D2F4C2F502F6F2D7C2D8D2D9E2DFC
:10543000A0E00E94969541F485E697E09F938F93B4
:105440000E94499A0F900F90DF91CF911F910F9179
:10545000FF90EF90DF90CF90BF90AF900895AF9204
:10546000BF92DF92EF92FF920F931F93CF93DF9340
:10547000EC015B01FB01108260E677E00E9462991B
:10548000892B59F58091CA2B3DE4F32E00E882FF69
:1054900003C024E8E22E02C094E0E92E10E0D12CF3
:1054A00081FD00EC26E04AE250E06BE270E089E228
:1054B00090E00E94A16381E090E00E944E0D88235D
:1054C00011F08DE5F82E8091CA2B9091CB2B90FD99
:1054D00016E091FF07C0186005C0F12C00E0E12C38
:1054E00010E0D12C6EE577E0CE010E946299892B05
:1054F00061F481E0F501808360917B0270917C0210
:1055000080E090E00E947699EC016CE577E0CE01B6
:105510000E946299892B61F48FEFF501808360917D
:105520007B0270917C0280E090E00E947699EC0111
:10553000209709F424C168E577E0CE010E946299C2
:10554000892B19F4FF2DF160FF2E64E577E0CE0181
:105550000E946299892B19F48F2D8460F82E61E5E1
:1055600077E0CE010E946299892B19F4EF2DE26059
:10557000FE2E6FE477E0CE010E946299892B19F428
:10558000FF2DF860FF2E6CE477E0CE010E94629957
:10559000892B19F48F2D8061F82E66E477E0CE0117
:1055A0000E946299892B19F4EF2DE062FE2E60E4CF
:1055B00077E0CE010E946299892B19F4FF2DF064E7
:1055C000FF2E6DE377E0CE010E946299892B19F4DA
:1055D0008F2D8068F82E68E377E0CE010E946299F3
:1055E000892B09F4016061E377E0CE010E946299A2
:1055F000892B09F402606EE277E0CE010E94629985
:10560000892B09F4046069E277E0CE010E94629977
:10561000892B09F4086062E277E0CE010E9462996A
:10562000892B09F400616BE177E0CE010E94629959
:10563000892B09F4006267E177E0CE010E9462994C
:10564000892B19F4ED2DE460DE2E64E177E0CE01C4
:105650000E946299892B09F400646FE077E0CE0123
:105660000E946299892B09F400686CE077E0CE0112
:105670000E946299892B19F4FE2DF160EF2E69E0EA
:1056800077E0CE010E946299892B19F48E2D8260F9
:10569000E82E66E077E0CE010E946299892B19F42A
:1056A000EE2DE460EE2E62E077E0CE010E9462997A
:1056B000892B19F4FE2DF860EF2E6EEF76E0CE0107
:1056C0000E946299892B19F48E2D8061E82E6AEF71
:1056D00076E0CE010E946299892B19F4EE2DE062EA
:1056E000EE2E66EF76E0CE010E946299892B19F4C6
:1056F000FE2DF064EF2E64EF76E0CE010E946299F9
:10570000892B19F48E2D8068E82E61EF76E0CE01AA
:105710000E946299892B09F4116069EE76E0CE014E
:105720000E946299892B09F4126060EE76E0CE0146
:105730000E946299892B09F4146067ED76E0CE012E
:105740000E946299892B09F4186064ED76E0CE011D
:105750000E946299892B09F410616EEC76E0CE010B
:105760000E946299892B09F4106263EC76E0CE0105
:105770000E946299892B09F0D2CE1064D0CE2F2DD1
:10578000302F4E2D512F6D2D70E080E090E0DF9195
:10579000CF911F910F91FF90EF90DF90BF90AF904E
:1057A00008955F926F927F928F929F92AF92BF9275
:1057B000CF92DF92EF92FF920F931F93CF93DF93DD
:1057C000782ECDEADBE100E010E08DEBE82E86E0FC
:1057D000F82E872D8170582E872D8270682E98EABA
:1057E000C92E96E0D92E20EBA22E26E0B22E3EEA5C
:1057F000832E36E0932E772051F01F930F93FF9264
:10580000EF920E94499A0F900F900F900F905520A1
:10581000A1F089858F9388858F93BF92AF920E9464
:10582000499A0F900F900F900F906620C1F09F92B1
:105830008F920E94499A0F900F90662081F0DF921C
:10584000CF920E94499A288139814A815B816C817B
:105850007D818E819F810E948F260F900F900E94E4
:10586000B60D0F5F1F4F2A960430110521F6DF9108
:10587000CF911F910F91FF90EF90DF90CF90BF904D
:10588000AF909F908F907F906F905F90089583EA84
:1058900096E09F938F930E94499A8091BA279091A6
:1058A000BB27A091BC27B091BD270F900F908130EE
:1058B00027EA92072EE1A207B10519F485E996E0DF
:1058C0001DC0823026EA92072EE1A207B10519F425
:1058D00088E896E013C0823027EA92072EE1A207FB
:1058E000B10519F48AE796E009C0823028EA9207E8
:1058F0002EE1A207B10549F48CE696E09F938F93C1
:105900000E94499A0F900F900895BF93AF939F9371
:105910008F9386E696E09F938F930E94499A0F900B
:105920000F900F900F900F900F90089586E596E0DE
:105930009F938F930E94499A0E94C3220E94472CF2
:105940000E94B60D84E99BE19F938F938EE496E0CD
:105950009F938F930E94499A60915C0270915D02BF
:1059600080915E0290915F0228EE33E040E050E0CB
:105970000E945B935F934F933F932F938EE396E048
:105980009F938F930E94499A85E396E09F938F930C
:105990000E94499A0E9444128091CA2B2DB73EB7AB
:1059A000225F3F4F0FB6F8943EBF0FBE2DBF80FF62
:1059B00005C041E061E081E00E94F11381E396E0DF
:1059C0009F938F930E94499A80E00E94A1240E9495
:1059D000C722809161021F928F9388E296E09F9385
:1059E0008F930E94499A80913D0A1F928F938FE175
:1059F00096E09F938F930E94499A80918D028F9396
:105A000080918C028F9380918B028F9380918A0278
:105A10008F9381E196E09F938F930E94499A1F9202
:105A200080E48F9389EF95E09F938F930E94499A2A
:105A30008091A4341F928F938091A3341F928F93EF
:105A400086EE95E09F938F930E94499A8091600221
:105A50001F928F938DED95E09F938F930E94499AAB
:105A60008091620290916302A0916402B0916502FC
:105A70002DB73EB7225E3F4F0FB6F8943EBF0FBE24
:105A80002DBF96FD03C08FE995E002C08CE995E03B
:105A90009F938F9383ED95E09F938F930E94499AF4
:105AA00083E00E94D12B0F900F900F900F901D99C3
:105AB00003C08FE995E002C08CE995E09F938F9336
:105AC00087EC95E09F938F930E94499A8DEB95E028
:105AD0009F938F930E94499A809162020F900F903A
:105AE0000F900F900F900F9081FF09C087EB95E00A
:105AF0009F938F930E94499A0F900F9013C080FD3F
:105B000003C08FE995E002C08CE995E09F938F93E5
:105B100083EB95E09F938F930E94499A0F900F908B
:105B20000F900F908091620290916302A0916402A5
:105B3000B091650297FD03C08FE995E002C08CE942
:105B400095E09F938F938AEA95E09F938F930E94AD
:105B5000499A83EA95E09F938F930E94499A6091B6
:105B6000410A7091420A8091430A9091440A0E942E
:105B7000E3240E94B60D0F900F900F900F900F909E
:105B80000F90779B03C08FE995E002C08CE995E008
:105B90009F938F938AE995E09F938F930E94499AF0
:105BA0000E942F0A0E940A0D9F938F937F936F93F9
:105BB0008CE895E09F938F930E94499A0E94B90CBC
:105BC0009F938F937F936F938EE795E09F938F932F
:105BD0000E94499A81E090E00E947D23809179346F
:105BE00090917A34A0917B34B0917C34BF93AF9381
:105BF0009F938F9380E795E09F938F930E94499A9C
:105C000080918E348F9380918D348F9380918C34DA
:105C10008F9380918B348F938CE595E09F938F9336
:105C20000E94499A80917D3490917E34A0917F3476
:105C3000B0918034BF93AF939F938F938EE495E0A0
:105C40009F938F930E94499A8DB79EB782960FB605
:105C5000F8949EBF0FBE8DBF809192348F93809138
:105C600091348F93809190348F9380918F348F9360
:105C70008AE395E09F938F930E94499A61E070E0D8
:105C800080E090E00E94BF0D61E070E081E090E074
:105C90000E94BF0D0F900F900F900F900F900F90DC
:105CA000299903C08FE995E002C08CE995E09F93A4
:105CB0008F9382E395E09F938F930E94499A0F9070
:105CC0000F900F900F902A9903C08FE995E002C0C2
:105CD0008CE995E09F938F938AE295E09F938F9351
:105CE0000E94499A0F900F900F900F900895F8948A
:105CF00091E2E0E0F0E0909357008491E2E0F0E080
:105D0000909357002491E4E0F0E090935700E491E1
:105D100090E0A0E0B0E0BC0155274427822F90E03E
:105D2000A0E0B0E0BA2FA92F982F8827840F951FE5
:105D3000A61FB71F8E0F911DA11DB11D8093BA27FD
:105D40009093BB27A093BC27B093BD277894089568
:105D5000CF93DF93CDB7DEB761970FB6F894DEBF70
:105D60000FBECDBF48E250E062E270E08DEA9BE1F9
:105D70000E942F9D2091AD1B3091AE1B4091AF1B17
:105D80005091B01B6091B11B7091B21B8091B31BFD
:105D90009091B41BAFEF0E94969509F05DC08DE421
:105DA0008093AD1B80E88093AE1B84E08093AF1B93
:105DB0001092B01B1092B11B1092B21B1092B31B29
:105DC0001092B41B8CE390E09093B61B8093B51BAC
:105DD0001092B71B1092B81B1092B91B1092BA1BED
:105DE0001092BB1B1092BC1B1092BD1B1092BE1BCD
:105DF0001092C01B1092BF1B1092C11B1092C21BAD
:105E00001092C31B1092C41B1092C51B1092C61B8C
:105E10001092C71B1092C81B1092CA1B1092C91B6C
:105E20001092CB1B1092CC1B1092CD1B1092CE1B4C
:105E30001092CF1B1092D01B1092D11B1092D21B2C
:105E40001092D41B1092D31B48E250E062E270E043
:105E50008DEA9BE10E944D9D44E050E06EE170E0D0
:105E6000CE010B960E942F9D8B859C85AD85BE85AE
:105E70008F3F2FEF9207A207B207A9F48AE090E4C0
:105E8000A0E0B0E08093620290936302A09364026A
:105E9000B093650244E050E06EE170E082E692E08B
:105EA0000E944D9D08C08093620290936302A0936C
:105EB0006402B09365028091620290916302A091A6
:105EC0006402B0916502A2FF02C02A9A03C080E07A
:105ED0000E94D72444E050E06AE570E0CE010B96C2
:105EE0000E942F9D8B859C85AD85BE858F3F2FEFB2
:105EF0009207A207B20789F41092410A1092420A4F
:105F00001092430A1092440A44E050E06AE570E0BF
:105F100081E49AE00E944D9D08C08093410A9093CD
:105F2000420AA093430AB093440A49E050E06EE06D
:105F300070E083E994E30E942F9D0E94ED0E44E0FF
:105F400050E06EE470E0CE010B960E942F9D8B8591
:105F50009C85AD85BE8544E050E06EE470E08F3FE7
:105F60009F4FAF4FBF4F29F482E892E00E944D9DB2
:105F700004C082E892E00E942F9D44E050E06AE471
:105F800070E0CE010B960E942F9D8B859C85AD8580
:105F9000BE8544E050E06AE470E08F3F9F4FAF4F12
:105FA000BF4F29F48EE792E00E944D9D04C08EE71A
:105FB00092E00E942F9D44E050E062E570E0CE0147
:105FC0000B960E942F9D8B859C85AD85BE8544E0F8
:105FD00050E062E570E08F3F9F4FAF4FBF4F29F415
:105FE00086E892E00E944D9D04C086E892E00E94FF
:105FF0002F9D41E050E06DE170E0CE0141960E949E
:106000002F9D898941E050E06DE170E08F3F29F4D8
:106010008DE39AE00E944D9D04C08DE39AE00E94BA
:106020002F9D41E050E06CE170E0CE0141960E946E
:106030002F9D898941E050E06CE170E08F3F29F4A9
:1060400081E692E00E944D9D04C081E692E00E94AC
:106050002F9D41E050E06BE170E0CE0141960E943F
:106060002F9D898941E050E06BE170E08F3F29F47A
:1060700080E692E00E944D9D04C080E692E00E947E
:106080002F9D4AE050E064E070E0CE0101960E944E
:106090002F9D89814AE050E064E070E08F3F29F451
:1060A00084E99BE10E944D9D04C084E99BE10E942C
:1060B0002F9D44E050E066E570E0CE010B960E9413
:1060C0002F9D8B859C85AD85BE8544E050E066E5BF
:1060D00070E08F3F9F4FAF4FBF4F29F48AE892E0A7
:1060E0000E944D9D04C08AE892E00E942F9D44E0EA
:1060F00050E067E170E0CE010B960E942F9D8B85EA
:106100009C85AD85BE8544E050E067E170E08F3F3F
:106110009F4FAF4FBF4F29F48CE592E00E944D9DF9
:1061200004C08CE592E00E942F9D42E050E062E0C6
:1061300070E0CE010F960E942F9D8F85988942E0D6
:1061400050E062E070E08F3F910529F488E39AE027
:106150000E944D9D04C088E39AE00E942F9D42E07A
:1061600050E060E070E0CE010F960E942F9D8F8579
:10617000988942E050E060E070E08F3F910529F49B
:1061800086E39AE00E944D9D04C086E39AE00E9457
:106190002F9D61960FB6F894DEBF0FBECDBFDF9185
:1061A000CF910895CF92DF92EF92FF9260917B02A0
:1061B00070917C0280E090E00E94769963EA75E03D
:1061C0000E948A99892B09F03BC18DE48093AD1B15
:1061D00080E88093AE1B84E08093AF1B1092B01BCD
:1061E0001092B11B1092B21B1092B31B1092B41BF1
:1061F0008CE390E09093B61B8093B51B1092B71B75
:106200001092B81B1092B91B1092BA1B1092BB1BB4
:106210001092BC1B1092BD1B1092BE1B1092C01B93
:106220001092BF1B1092C11B1092C21B1092C31B75
:106230001092C41B1092C51B1092C61B1092C71B54
:106240001092C81B1092CA1B1092C91B1092CB1B34
:106250001092CC1B1092CD1B1092CE1B1092CF1B14
:106260001092D01B1092D11B1092D21B1092D41BF3
:106270001092D31B48E250E062E270E08DEA9BE1AD
:106280000E944D9D8AE090E4A0E0B0E0809362021D
:1062900090936302A0936402B093650244E050E0DF
:1062A0006EE170E082E692E00E944D9D1092410AFC
:1062B0001092420A1092430A1092440A44E050E0BD
:1062C0006AE570E081E49AE00E944D9D82E2C82E6A
:1062D000DD24DA948CECE82E8BE3F82EC092820257
:1062E000D0928302E0928402F092850244E050E072
:1062F0006EE470E082E892E00E944D9DC0927E02C2
:10630000D0927F02E0928002F092810244E050E05D
:106310006AE470E08EE792E00E944D9D87ED94E381
:10632000AFEEBCE38093860290938702A09388022D
:10633000B093890244E050E062E570E086E892E0C4
:106340000E944D9D8AE999E9A9E1B0E480938A020F
:1063500090938B02A0938C02B0938D0244E050E0A6
:1063600066E570E08AE892E00E944D9D10923D0A39
:1063700080E00E94637141E050E06DE170E08DE3E8
:106380009AE00E944D9D8AE1809361020E940B7009
:1063900041E050E06CE170E081E692E00E944D9DAA
:1063A0008FE08093600241E050E06BE170E080E6B6
:1063B00092E00E944D9D8AE0E4E9FBE1DF011D923D
:1063C0008A95E9F74AE050E064E070E0CF010E946E
:1063D0004D9D80EA96E8A1E0B0E080935C02909346
:1063E0005D02A0935E02B0935F0244E050E067E17B
:1063F00070E08CE592E00E944D9D1092390A109257
:10640000380A42E050E062E070E088E39AE00E94DF
:106410004D9D1092370A1092360A42E050E060E03B
:1064200070E086E39AE00E944D9D81E00E94A124E5
:1064300080E090E0FF90EF90DF90CF900C94010F00
:10644000FF90EF90DF90CF9008950E94616D6C9A5D
:106450006B9A6A9A6F9A729A749A739A779A8098DA
:1064600080B3897F80BB8398849887E080937E0087
:10647000549A0E94772E0E94A82E0E949D0A80E0C6
:1064800090E00E94010F60915C0270915D0280912A
:106490005E0290915F020E9484660E94B90C609334
:1064A000CC2F7093CD2F8093CE2F9093CF2F8091B0
:1064B000620286FD239A219A229A239A0E94B20AA6
:1064C0001D9B05C010923F0A10923E0A089581E07C
:1064D00090E090933F0A80933E0A0895CF93DF9314
:1064E00090E04091410A5091420A6091430A7091B4
:1064F000440A41FD08C02091620220FD04C021FF32
:106500008CC01D9B8AC02DE8289FE001299FD00DDB
:106510001124CE018654934E9F938F938AEA95E07F
:106520009F938F930E94359AFE01ED54F34EDF0145
:10653000AA57BF4F2C910F900F900F900F9043814F
:106540005481658176818091D02F9091D12FA09137
:10655000D22FB091D32F841B950BA60BB70B222300
:10656000D1F1BF93AF939F938F93DF01A257BF4F9A
:1065700011968C9111978F938C918F9312971196FE
:106580008C9111978F938C918F9313978C911F926D
:106590008F9311978C911F928F9313968C911F92CA
:1065A0008F9311978C911F928F93E957FF4F8081A2
:1065B0001F928F931F922F9380EB95E09F938F9361
:1065C0000E94359A8DB79EB746960FB6F8949EBF37
:1065D0000FBE8DBF10C0BF93AF939F938F9387EF74
:1065E00095E09F938F930E94359A0F900F900F9094
:1065F0000F900F900F900E94B60D80917D0288231E
:1066000061F01F928F9383EE91E09F938F930E948E
:10661000499A0F900F900F900F90DF91CF910895AE
:106620008091B31C882341F08091B41C90E00E94BB
:106630006E320E94A30BF4CF0895CF93DF93EC0149
:1066400088819981823D2EE09207E9F018F4892B28
:10665000B9F048C08A3D2EE0920709F449C08E3D4A
:106660009E4009F03FC083E59AE00E94F05D892BCF
:10667000E9F183E59AE00E94D35D80E00E94D12495
:1066800082ED9EE02CC0623189F5299A6091360A2C
:106690007091370A7695762F66277795679583E50B
:1066A0009AE00E94C95D8091410A9091420AA091AE
:1066B000430AB091440AA0FF10C08091370A8F931B
:1066C0008091360A8F938CE790E19F938F930E947D
:1066D000499A0F900F900F900F908AED9EE099834A
:1066E000888304C01982188283E017C081E015C036
:1066F00083E59AE00E94F05D892BC1F383E59AE07F
:106700000E94D35D0E94103360E270E083E59AE05E
:106710000E94C95D8EED9EE0E2CFDF91CF9108959A
:106720002F923F924F925F926F927F928F929F92A1
:10673000AF92BF92CF92DF92EF92FF920F931F938F
:10674000CF93DF93CDB7DEB72B970FB6F894DEBFAC
:106750000FBECDBF9B878A873A01FC018081918162
:10676000892B11F00C94CA4760917B0270917C02D6
:10677000CA010E94769960E870E0C3010E94A9995D
:10678000009759F460915A3D70915B3D8AE090E02A
:106790000E94FD9981E00C94CF478130910561F40E
:1067A000F3011081912E990C9908892C092D292C1F
:1067B000392C492C592CB9C082309105B9F4F30118
:1067C0008081082E000C990B982F88272181820F39
:1067D000911D27FD9A95182F992E892E880C8808CF
:1067E000082D282C382C482C582C9FC0833091051C
:1067F000B1F5F3012081922F990F990B392F492F71
:10680000592F692F792F892F00E10E94389519019E
:106810002A014B01B82FA92F2181922F990F990B93
:10682000392F492F592F692F792F892F08E00E947E
:10683000389559016A017B018C019101A201B401D3
:106840008B2F9A2F0E946F95A2801A2D110F110B7A
:10685000B12EC12ED12EE12EF12E012F55C004975D
:106860000CF45BC0F3012081922F990F990B392F03
:10687000492F592F692F792F892F08E10E943895C8
:1068800019012A014B01B82FA92F2181922F990FAD
:10689000990B392F492F592F692F792F892F00E113
:1068A0000E94389559016A017B018C019101A20176
:1068B000B4018B2F9A2F0E946F95A3801A2D110F70
:1068C000110BB12EC12ED12EE12EF12E012F0E94DF
:1068D0006F9519012A014B01B82FA92F2281922F00
:1068E000990F990B392F492F592F692F792F892FFC
:1068F00008E00E94389559016A017B018C019101E1
:10690000A201B4018B2F9A2F0E946F95122F932E04
:10691000842E052F1B012C0108C01AE0912C812C1C
:1069200000E0212C312C412C512C0E94B60D212F3E
:10693000392D482D502FB101C2012537F3E63F070D
:10694000FDE64F075105610571058105910511F4BB
:106950000C94AF422537E3E63E07EDE64E075105BE
:10696000610571058105910511F008F0B2C1233769
:10697000F2E73F0741055105610571058105910564
:1069800011F40C9448452337E2E73E0741055105D1
:10699000610571058105910511F008F0B9C0253632
:1069A000F4E63F0741055105610571058105910533
:1069B00009F4DBC72536E4E63E07410551056105CC
:1069C00071058105910511F008F041C0A6E70E940C
:1069D000969511F40C94373F0E94969509F070F447
:1069E000A8E60E94969511F40C94063DA5E70E9436
:1069F000969511F40C94213F0C94C847212F392D02
:106A0000482D502FB101C2012436F1E63F07410560
:106A10005105610571058105910511F40C947045CE
:106A20002537E2E63E0741055105610571058105FF
:106A3000910509F431C52A333642410551056105F6
:106A400071058105910509F430C30C94C847212FC5
:106A5000392D482D502FB101C2012737EFE63E07EF
:106A600041055105610571058105910511F40C94ED
:106A700015432737FFE63F074105510561057105BD
:106A80008105910509F0C8F42436E9E63E07410581
:106A90005105610571058105910511F40C94FA3ECB
:106AA00025363E4641055105610571058105910573
:106AB00011F40C9449430C94C847212F392D482DCB
:106AC000502FB101C2012536E2E73E0741055105CD
:106AD000610571058105910511F40C941544293661
:106AE000F2E73F07410551056105710581059105F3
:106AF00011F40C94F74423333147410551056105E6
:106B000071058105910511F00C94C8470C947045EE
:106B1000212F392D482D502FB101C2012236F5E623
:106B20003F07F4E64F0751056105710581059105A1
:106B300009F41BC72236E5E63E07E4E64E07510599
:106B4000610571058105910511F008F05BC02133E5
:106B5000F4E63F07F1E64F07510561057105810530
:106B6000910509F4B6C22133E4E63E07E1E64E079B
:106B70005105610571058105910509F0C0F42337C0
:106B8000F3E73F0741055105610571058105910551
:106B900011F40C945C4528373447410551056105D3
:106BA00071058105910509F480C20C94C847212F15
:106BB000392D482D502FB101C2012837F4E63F0787
:106BC000F1E64F075105610571058105910509F44D
:106BD0007CC22C36E5E73E07E2E64E07510561052B
:106BE00071058105910509F457C4233634464146A1
:106BF0005105610571058105910511F00C94C84797
:106C00000C947045212F392D482D502FB101C20110
:106C10002D36E5E73E07E8E64E07510561057105AB
:106C20008105910511F40C9486452D36F5E73F0753
:106C3000F8E64F075105610571058105910509F0D9
:106C4000E0F42237E2E73E07E5E64E07510561052D
:106C500071058105910511F40C94604223363D467F
:106C600048465105610571058105910511F00C94A7
:106C7000C8470E944E180C94CA47212F392D482D21
:106C8000502FB101C2012436E3E63E07ECE64E0781
:106C90005105610571058105910511F40C94C341FD
:106CA0002736FFE63F07FCE64F07510561057105F2
:106CB0008105910511F40C94C641233632434946AF
:106CC0005105610571058105910511F00C94C847C6
:106CD00020C2212F392D482D502FB101C20120375C
:106CE000FCE63F07F5E64F07F8E65F07610571052B
:106CF0008105910509F48AC62037ECE63E07E5E6F2
:106D00004E07E8E65E07610571058105910511F002
:106D100008F0E0C02437F8E73F07F4E74F075105D4
:106D2000610571058105910511F40C94A33F243789
:106D3000E8E73E07E4E74E07510561057105810567
:106D4000910511F008F05DC02033F1E33F07F1E752
:106D50004F075105610571058105910511F40C94EA
:106D600060422033E1E33E07E1E74E07510561054C
:106D700071058105910509F0C0F42133F2E63F0762
:106D8000F0E74F075105610571058105910509F48B
:106D900098C222333246404751056105710581058D
:106DA000910509F4E3C20C94C847212F392D482DD1
:106DB000502FB101C2012037F5E63F07F2E74F0738
:106DC0005105610571058105910511F40C94154477
:106DD0002C36E4E73E074E07510561057105810534
:106DE000910511F40C94EE4621333143414751058E
:106DF000610571058105910511F00C94C8470C944B
:106E0000AF42212F392D482D502FB101C2012B3611
:106E1000ECE63E07E5E74E07E2E65E076105710531
:106E20008105910509F438C32B36FCE63F07F5E7E9
:106E30004F07F2E65F07610571058105910509F0CD
:106E4000E0F42437E4E63E07E7E74E075105610525
:106E500071058105910511F40C943C4724373F4698
:106E60004F465246610571058105910511F00C945C
:106E7000C8470C9400000C94CA47212F392D482D87
:106E8000502FB101C2012E36E1E63E07E8E64E077B
:106E9000E3E65E07610571058105910511F40C9427
:106EA000773F2633F9E63F07F5E74F07F5E65F073B
:106EB000610571058105910509F4ACC529363C468B
:106EC00041465346610571058105910511F00C9409
:106ED000C84789C3212F392D482D502FB101C20138
:106EE0002437F3E73F07F5E64F07F2E75F07610551
:106EF00071058105910511F40C94C5432437E3E72E
:106F00003E07E5E64E07E2E75E076105710581058C
:106F1000910511F008F062C02337F5E63F07F2E76C
:106F20004F07F0E75F07610571058105910511F4D1
:106F30000C9436462337E5E63E07E2E74E07E0E7E6
:106F40005E07610571058105910509F0D0F42136D0
:106F5000FDE63F07F5E74F07F8E65F0761057105B6
:106F60008105910511F40C9433432237374740478C
:106F70005047610571058105910509F45CC20C94C7
:106F8000C847212F392D482D502FB101C201243679
:106F9000FDE63F07F3E64F07F2E75F07610571057E
:106FA0008105910509F441C62136ECE63E07E5E688
:106FB0004E07E2E75E07610571058105910509F459
:106FC00046C523373247474750476105710581055C
:106FD000910511F00C94C8470C94C843212F392D0A
:106FE000482D502FB101C2012437E2E73E07E1E608
:106FF0004E07E5E75E07610571058105910509F416
:107000006FC62437F2E73F07F1E64F07F5E75F0762
:10701000610571058105910509F0C8F42437E3E79E
:107020003E07E5E64E07E4E75E0761057105810569
:10703000910509F4B3C727373047484754476105DE
:1070400071058105910509F428C70C94C847212FC3
:10705000392D482D502FB101C2012F36ECE63E07E5
:10706000EFE54E07E6E75E076105710581059105CD
:1070700009F486C52C36F1E63F07F4E74F07F8E739
:107080005F07610571058105910511F40C94B846FF
:1070900022373746404755476105710581059105FF
:1070A00011F00C94C8470C949F4183E08093813485
:1070B000109283341092823441E854E362E18EE30B
:1070C00092E00E94445B0C94CA470E94D6170C942D
:1070D000CA4721E042E161E080ED0E94616821E061
:1070E00042E161E080ED0E94616821E042E161E0FF
:1070F00080ED0E94616821E042E161E080ED0E9444
:10710000616821E042E161E080ED0E9461680C94D9
:10711000CA4760917B0270917C0280E090E00E94FF
:10712000769963E076E00E948A99892B09F0C5C0C0
:1071300060917B0270917C0280E090E00E947699E1
:107140008C01009709F497C06CEE73E00E948A9955
:10715000892BE1F488EE93E0A0E0B0E080935C023C
:1071600090935D02A0935E02B0935F0268EE73E0BD
:1071700080E090E00E94846644E050E067E170E0C7
:107180008CE592E00E944D9D0C94CA4769E076E040
:10719000C8010E948A99892BE1F480E197E2A0E07E
:1071A000B0E080935C0290935D02A0935E02B09386
:1071B0005F0260E177E280E090E00E94846644E054
:1071C00050E067E170E08CE592E00E944D9D0C94E8
:1071D000CA476CE076E0C8010E948A99892BE1F4E5
:1071E00080EA96E8A1E0B0E080935C0290935D02B3
:1071F000A0935E02B0935F0260EA76E881E090E0DF
:107200000E94846644E050E067E170E08CE592E023
:107210000E944D9D0C94CA4760E176E0C8010E942F
:107220008A99892BE1F480E89AE1A6E0B0E08093A6
:107230005C0290935D02A0935E02B0935F0260E8EF
:107240007AE186E090E00E94846644E050E067E1E5
:1072500070E08CE592E00E944D9D0C94CA4782E656
:1072600093E09F938F930E94499A0E94B60D0F90CE
:107270000F900C94CA4760915C0270915D028091FE
:107280005E0290915F0228EE33E040E050E00E9401
:107290005B935F934F933F932F938EE593E09F9380
:1072A0008F930E94499A0E94B60D0F900F900F90F5
:1072B0000F900F900F900C94CA470E9444120C94A8
:1072C000CA4760917B0270917C0280E090E00E944E
:1072D00076998C016CE975E00E948A99892BA1F45A
:1072E0008091620290916302A0916402B091650264
:1072F000A2608093620290936302A0936402B093B1
:107300006502299A0C94CA476FE975E0C8010E948A
:107310008A99892BB1F48091620290916302A091C5
:107320006402B0916502AD7F809362029093630224
:10733000A0936402B093650280E00E94D1240C9473
:10734000CA47299903C08FE995E002C08CE995E00E
:107350009F938F9386E593E09F938F930E94499A22
:107360000F900F900F900F900C94CA4760917B0282
:1073700070917C0280E090E00E9476998C016CE92B
:1073800075E00E948A99892BE1F4809162029091C4
:107390006302A0916402B0916502A46080936202CE
:1073A00090936302A0936402B09365022A9A44E02A
:1073B00050E06EE170E082E692E00E944D9D0C94F8
:1073C000CA476FE975E0C8010E948A99892BF1F4D8
:1073D0008091620290916302A0916402B091650273
:1073E000AB7F8093620290936302A0936402B09398
:1073F000650280E00E94D72444E050E06EE170E036
:1074000082E692E00E944D9D0C94CA472A9903C0DF
:107410008FE995E002C08CE995E09F938F938EE40D
:1074200093E09F938F930E94499A0F900F900F9033
:107430000F900C94CA4760917B0270917C0280E0AF
:1074400090E00E9476998C016CE975E00E948A991F
:10745000892B19F477980C94CA476FE975E0C80135
:107460000E948A99892B19F4779A0C94CA47779BC2
:1074700003C08FE995E002C08CE995E09F938F935C
:1074800084E195E09F938F930E94499A0F900F900B
:107490000F900F900C94CA4760917B0270917C0210
:1074A00080E090E00E9476998C0164E176E00E9491
:1074B0008A99892BD1F48091B31C1F928F9380916C
:1074C000B51C1F928F938091B41C1F928F931F92B3
:1074D00084E18F9384E293E09F938F930E94499A73
:1074E0000FB6F894DEBF0FBECDBF69E176E0C801EC
:1074F0000E948A99892B19F40E94103370C061E2AE
:1075000076E0C8010E948A99892B09F047C06091F2
:107510007B0270917C0280E090E00E947699009757
:1075200009F45DC00E9463988531910570F59093D0
:10753000390A8093380A42E050E062E070E088E364
:107540009AE00E944D9D60917B0270917C0280E0E8
:1075500090E00E947699009709F441C00E946398D8
:107560009093370A8093360A42E050E060E070E082
:1075700086E39AE00E944D9D60917B0270917C02AF
:1075800080E090E00E9476992AC082E193E09F9388
:107590008F930E94499A0F900F9021C08091390AD1
:1075A0008F938091380A8F9389E093E09F938F9314
:1075B0000E94499A0E94B60D8091370A8F9380915C
:1075C000360A8F938AEF92E09F938F930E94499A95
:1075D0000E94B60D0FB6F894DEBF0FBECDBF0E945D
:1075E000B60D0C94CA4760917B0270917C0280E0DA
:1075F00090E00E9476998C0166E675E00E948A9977
:10760000892B09F077C060917B0270917C0280E049
:1076100090E00E9476998C01009711F40C94CA476F
:107620006FE176E00E948A99892BB1F482E29FEFA4
:10763000ACECBBE38093820290938302A09384021C
:10764000B093850244E050E06EE470E082E892E09E
:107650000E944D9D0C94CA4765E276E0C8010E94E5
:107660008A99892BB1F482E29FEFACECBAE3809364
:10767000820290938302A0938402B093850244E037
:1076800050E06EE470E082E892E00E944D9D0C9420
:10769000CA47C8010E945F982B013C0120E030E0FE
:1076A000A9010E94978F8823D9F081E00E94570C8E
:1076B0009B01AC01C301B2010E949C8F60938202C6
:1076C00070938302809384029093850244E050E09B
:1076D0006EE470E082E892E00E944D9D0C94CA47EF
:1076E0008DEE92E09F938F930E94499A0F900F9096
:1076F0000C94CA4769E675E0C8010E948A99892BF3
:1077000009F077C060917B0270917C0280E090E08C
:107710000E9476998C01009711F40C94CA476FE18E
:1077200076E00E948A99892BB1F482E29FEFACEC5B
:10773000BBE380937E0290937F02A0938002B0937C
:10774000810244E050E06AE470E08EE792E00E943B
:107750004D9D0C94CA4765E276E0C8010E948A9963
:10776000892BB1F482E29FEFACECBAE380937E0206
:1077700090937F02A0938002B093810244E050E096
:107780006AE470E08EE792E00E944D9D0C94CA4737
:10779000C8010E945F982B013C0120E030E0A90164
:1077A0000E94978F8823D9F082E00E94570C9B019A
:1077B000AC01C301B2010E949C8F60937E02709362
:1077C0007F02809380029093810244E050E06AE45B
:1077D00070E08EE792E00E944D9D0C94CA4780EEC7
:1077E00092E09F938F930E94499A0F900F900C9470
:1077F000CA4761E675E0C8010E948A99892B09F0A1
:1078000073C060917B0270917C0280E090E00E94E6
:1078100076998C01009711F40C94CA476FE176E0D9
:107820000E948A99892BB1F487ED94E3AFEEBCE313
:107830008093860290938702A0938802B093890276
:1078400044E050E062E570E086E892E00E944D9DE1
:107850000C94CA4765E276E0C8010E948A99892B98
:1078600051F481ED92E09F938F930E94499A0F907B
:107870000F900C94CA47C8010E945F982B013C01ED
:1078800020E030E0A9010E94978F882319F180E061
:107890000E94570C4B015C0121EE3AE744E95EE39C
:1078A000C301B2010E94B88EA50194010E949C8F71
:1078B0006093860270938702809388029093890276
:1078C00044E050E062E570E086E892E00E944D9D61
:1078D0000C94CA4784EC92E09F938F930E94499A3C
:1078E0000F900F900C94CA470E94A50C9F938F9302
:1078F0007F936F938DEB92E09F938F930E94499AB1
:1079000082E00E94570C20917E0230917F024091CC
:107910008002509181020E944892162F072FF82E64
:10792000E92E81E00E94570CEF92FF920F931F9374
:10793000209182023091830240918402509185020D
:107940000E9448929F938F937F936F9381EB92E075
:107950009F938F930E94499A0E94B60D0FB6F89498
:10796000DEBF0FBECDBF0C94CA4760917B02709101
:107970007C0280E090E00E947699009711F10E94CD
:10798000D6250091410A1091420A2091430A309174
:10799000440A601771078207930739F16093410A1F
:1079A0007093420A8093430A9093440A44E050E063
:1079B0006AE570E081E49AE00E944D9D8DE095E0DB
:1079C00002C086E095E09F938F930E94499A609150
:1079D000410A7091420A8091430A9091440A0E94A0
:1079E000E3240E94B60D0F900F908BEF94E09F93CD
:1079F0008F930E94499A6FEF7FEFCB010E94E3249F
:107A00000E94B60D0F900F900C94CA470E94C0219F
:107A10000C94CA47F3018481843329F440E061E087
:107A200080E00E94F11380917D02882311F40C9470
:107A3000CA471F928F9388EF94E09F938F930E9481
:107A4000499A0F900F900F900F900C94CA47F30132
:107A50008481893709F080C060917B0270917C023B
:107A600080E090E00E9476998C016CE975E00E94BC
:107A70008A99892B51F48091620290916302A091BE
:107A80006402B0916502906410C06FE975E0C801AE
:107A90000E948A99892BD1F48091620290916302AD
:107AA000A0916402B09165029F7B809362029093E3
:107AB0006302A0936402B093650244E050E06EE17B
:107AC00070E082E692E00E944D9D46C06AE276E058
:107AD000C8010E948A99892B21F58091AC1B8F9354
:107AE0008091AB1B8F938091AA1B8F938091A91BD0
:107AF0008F938091A81B8F938091A71B8F93809168
:107B0000A61B8F938091A51B8F9386E892E09F938D
:107B10008F930E94499A0FB6F894DEBF0FBECDBF77
:107B20001BC08091620290916302A0916402B091A7
:107B3000650296FD03C08FE995E002C08CE995E0EF
:107B40009F938F9382E892E09F938F930E94499A2C
:107B50000F900F900F900F9080917D02882311F469
:107B60000C94CA471F928F9385EF94E09F938F9355
:107B70000E94499A0F900F900F900F900C94CA4753
:107B8000F30184818737E9F560917B0270917C0273
:107B900080E090E00E9476990097D9F00E945F986B
:107BA0002B013C0120E030E0A9010E94978F88233F
:107BB00081F040928A0250928B0260928C02709205
:107BC0008D0244E050E066E570E08AE892E00E94B1
:107BD0004D9D80918D028F9380918C028F93809127
:107BE0008B028F9380918A028F9384E792E09F9318
:107BF0008F930E94499A0F900F900F900F900F90C3
:107C00000F9080917D02882311F40C94CA471F9233
:107C10008F9382EF94E09F938F930E94499A0F90E5
:107C20000F900F900F900C94CA4760917B02709157
:107C30007C0280E090E00E9476998C016CE975E00E
:107C40000E948A99409062025090630260906402A0
:107C500070906502892B19F4689457F809C06FE990
:107C600075E0C8010E948A99892B99F4E89457F825
:107C700040926202509263026092640270926502C6
:107C800044E050E06EE170E082E692E00E944D9D9B
:107C900013C057FC03C08FE995E002C08CE995E062
:107CA0009F938F9380E792E09F938F930E94499ACE
:107CB0000F900F900F900F9080917D02882311F408
:107CC0000C94CA471F928F938FEE94E09F938F93EB
:107CD0000E94499A0F900F900F900F900C94CA47F2
:107CE00060917B0270917C0280E090E00E94769926
:107CF0008C0160E376E00E948A99892B11F489E176
:107D000008C064E376E0C8010E948A99892B49F48F
:107D100080E18093C4001092C50082E08093C0008F
:107D200055C068E376E0C8010E948A99892B11F456
:107D300088E0EFCF6DE376E0C8010E948A99892B35
:107D400039F062E476E0C8010E948A99892B11F427
:107D500083E0DFCF8091C400893141F48BE692E06B
:107D60009F938F930E94499A0F900F908091C40027
:107D7000803141F486E692E09F938F930E94499A66
:107D80000F900F908091C400883041F480E692E01B
:107D90009F938F930E94499A0F900F908091C400F7
:107DA000833041F48AE592E09F938F930E94499A31
:107DB0000F900F908091C400883041F484E592E0E8
:107DC0009F938F930E94499A0F900F9080917D020C
:107DD000882311F40C94CA471F928F938CEE94E081
:107DE0009F938F930E94499A0F900F900F900F903E
:107DF0000C94CA4760917B0270917C0280E090E015
:107E00000E9476996FE176E00E948A99892B11F49D
:107E100081E001C080E00E94A12480917D0288233E
:107E200011F40C94CA471F928F9389EE94E09F93AC
:107E30008F930E94499A0F900F900F900F900C947F
:107E4000CA470E94C72280917D02882311F40C94B6
:107E5000CA471F928F9386EE94E09F938F930E9460
:107E6000499A0F900F900F900F900C94CA470E9460
:107E7000C32280917D02882311F40C94CA471F927B
:107E80008F9383EE94E09F938F930E94499A0F9073
:107E90000F900F900F900C94CA4760917B027091E5
:107EA0007C0280E090E00E9476990E946398803185
:107EB00070F480933D0A0E94637141E050E06DE1EF
:107EC00070E08DE39AE00E944D9D0C94CA4780912A
:107ED0003D0A1F928F938AE492E09F938F930E94B2
:107EE000499A0F900F900F900F900C94CA47609191
:107EF0007B0270917C0280E090E00E9476990E9463
:107F0000639895EF980F903170F4809361020E940E
:107F10000B7041E050E06CE170E081E692E00E947D
:107F20004D9D0C94CA47809161021F928F9381E40A
:107F300092E09F938F930E94499A0F900F900F9019
:107F40000F900C94CA4760917B0270917C0280E094
:107F500090E00E947699009789F04AE050E0BC01D9
:107F600084E99BE10E949A994AE050E064E070E065
:107F700084E99BE10E944D9D0C94CA4784E99BE1F2
:107F80009F938F9387E496E09F938F930E94359AF7
:107F90000F900F900F900F900C94CA4760917B0246
:107FA00070917C0280E090E00E9476998C016CEEEA
:107FB00073E00E948A99892BD9F4219A80916202F8
:107FC00090916302A0916402B091650280618093F8
:107FD000620290936302A0936402B093650244E04E
:107FE00050E06EE170E082E692E00E944D9DD2C7C3
:107FF0006AE675E0C8010E948A99892BD9F4229A11
:108000008091620290916302A0916402B091650236
:1080100080628093620290936302A0936402B093A3
:10802000650244E050E06EE170E082E692E00E947A
:108030004D9DB0C76EEC73E0C8010E948A99892BF0
:10804000D9F4239A8091620290916302A091640214
:10805000B091650280648093620290936302A09362
:108060006402B093650244E050E06EE170E082E6A5
:1080700092E00E944D9D8EC76DE075E0C8010E94A0
:108080008A99892BD9F4239A809162029091630294
:10809000A0916402B091650280688093620290931F
:1080A0006302A0936402B093650244E050E06EE185
:1080B00070E082E692E00E944D9D6CC764EE79E02C
:1080C000C8010E948A99892B71F581E08093E52F80
:1080D0008DEA9BE19093E72F8093E62F1092E92F92
:1080E0001092E82F8091620290916302A091640245
:1080F000B091650291608093620290936302A093B5
:108100006402B093650244E050E06EE170E082E604
:1081100092E00E944D9D45EE5FE262E18EE392E0C7
:108120000E94445B37C765EF73E0C8010E948A99DB
:10813000892B11F5EDEDFBE1119211922BE1ED3F51
:10814000F207D1F78091620290916302A0916402DC
:10815000B091650292608093620290936302A09353
:108160006402B093650244E050E06EE170E082E6A4
:1081700092E00E944D9D0EC76FE975E0C8010E9414
:108180008A994091620250916302609164027091F9
:108190006502892BC1F44F705C7F4093620250935B
:1081A000630260936402709365022B9A44E050E08E
:1081B0006EE170E082E692E00E944D9D80918A34EB
:1081C0000E942070E7C644FD03C08FE995E002C01D
:1081D0008CE995E09F938F9386E392E09F938F9332
:1081E0000E94499A809162020F900F900F900F9019
:1081F00085FD03C08FE995E002C08CE995E09F936F
:108200008F938BE292E09F938F930E94499A809183
:1082100062020F900F900F900F9086FD03C08FE9C0
:1082200095E002C08CE995E09F938F9380E292E005
:108230009F938F930E94499A809162020F900F90B2
:108240000F900F9087FD03C08FE995E002C08CE985
:1082500095E09F938F9385E192E09F938F930E9487
:10826000499A8091620290916302A0916402B09158
:1082700065020F900F900F900F9090FD03C08FE953
:1082800095E002C08CE995E09F938F938AE092E09D
:108290009F938F930E94499A80916202909163020A
:1082A000A0916402B09165020F900F900F900F9013
:1082B00091FD03C08FE995E002C08CE995E09F93A2
:1082C0008F938FEF91E09F938F930E94499A8091B3
:1082D000620290916302A0916402B09165020F90D6
:1082E0000F900F900F9091FF55C68FE496E00E947B
:1082F000719A9DEDE92E9BE1F92E00E010E027E553
:10830000822E26E0922EF70180819181F2E0EF0E1D
:10831000F11C9F938F93C8010B969F938F939F920D
:108320008F920E94359A0F5F1F4F0F900F900F9002
:108330000F900F900F900031110529F72BC68FED8C
:1083400094E09F938F930E94499A80917D020F90B1
:108350000F90882361F01F928F938CED94E09F9390
:108360008F930E94499A0F900F900F900F90F8945E
:1083700098E088E10FB6F894A895809360000FBE4E
:1083800090936000FFCF0E94126804C660917B0248
:1083900070917C0280E090E00E9476998C016CE9FB
:1083A00075E00E948A99892BE9F40E94066F8091FA
:1083B000620290916302A0916402B09165028D7F88
:1083C00081608093620290936302A0936402B093F1
:1083D000650244E050E06EE170E082E692E00E94C7
:1083E0004D9DD8C56FE975E0C8010E948A99892B17
:1083F000E1F40E94BE6E8091620290916302A091AE
:108400006402B09165028C7F809362029093630254
:10841000A0936402B093650244E050E06EE170E026
:1084200082E692E00E944D9DB5C562E676E0C80105
:108430000E948A99892BE9F40E94BE6E80916202A3
:1084400090916302A0916402B09165028E7F826078
:108450008093620290936302A0936402B0936502DA
:1084600044E050E06EE170E082E692E00E944D9DB3
:1084700091C58091620281FF0FC082E696E09F93D2
:108480008F938BEF91E09F938F930E94499A0F9067
:108490000F900F900F907EC580FD03C08FE995E08F
:1084A00002C08CE995E09F938F9387EF91E09F93B3
:1084B0008F930E94499A0F900F900F900F906AC56A
:1084C0008091E32F8F938091E22F8F938091E12F02
:1084D0008F938091E02F8F938091DF2F8F938091E6
:1084E000DE2F8F938091DD2F8F938091DC2F8F93E0
:1084F0008091DB2F8F938091DA2F8F938091D92FEA
:108500008F938091D82F8F938091D72F8F938091C5
:10851000D62F8F938091D52F8F938091D42F8F93C7
:1085200080EB94E09F938F930E94499A0E94B60D2E
:1085300080917D020FB6F894DEBF0FBECDBF8823B9
:1085400009F428C51F928F938DEA94E09F938F932F
:108550000E94499A0F900F900F900F901BC5F894AE
:1085600089E021E030E0F90180935700C895E02CC4
:1085700020E030E0F90180935700C895F02C789402
:10858000F89423E030E0F90180935700C895002D5E
:1085900022E030E0F90180935700C895102D7894BF
:1085A0008091BD278F938091BC278F938091BB27AB
:1085B0008F938091BA278F9383EA94E09F938F9350
:1085C0000E94499A1F92EF921F92FF921F920F935F
:1085D0001F921F938CE794E09F938F930E94499A78
:1085E0000E946123809166001F928F9380E794E040
:1085F0009F938F930E94499A0E94B60D80917D02AD
:108600000FB6F894DEBF0FBECDBF882309F4C2C4F5
:108610001F928F938DE694E09F938F930E94499AC7
:108620000F900F900F900F90B5C460E070E080E065
:1086300090E00E94BF0D60E070E081E090E00E9459
:10864000BF0D80917D02882309F4A4C41F928F93EB
:108650008AE694E09F938F930E94499A0F900F901F
:108660000F900F9097C40E9483210E94B60D8091B5
:108670007D02882309F48EC41F928F9387E694E0CD
:108680009F938F930E94499A0F900F900F900F9095
:1086900081C460917B0270917C0280E090E00E9436
:1086A000769969E176E00E948A99892B31F5F894F0
:1086B00082E89AE00E94335C8C01892B69F0C80142
:1086C0000F960E943B5FB80184E092E00E94EC5B51
:1086D000C8010E94DF5CF0CF82E89AE00E94C45C8F
:1086E000892B29F082E89AE00E946C5CF5CF82E841
:1086F0009AE00E942F5C789436C082E89AE00E944B
:10870000335C8C0187E6E82E86E0F82E0115110512
:1087100051F1F80186811F928F9380851F928F936C
:1087200085811F928F9381851F928F9387811F92DE
:108730008F9384811F928F9383811F928F93828165
:108740001F928F9382851F928F93FF92EF920E94C8
:10875000359AC8010E94DF5C8C010FB6F894DEBF29
:108760000FBECDBFD3CF80917D02882309F412C400
:108770001F928F9384E694E09F938F930E94499A6F
:108780000F900F900F900F9005C40E94D23002C43A
:1087900060917B0270917C0280E090E00E9476996B
:1087A0008C0166EA76E00E948A99892BD1F4809147
:1087B000620290916302A0916402B0916502977F7A
:1087C0008093620290936302A0936402B093650267
:1087D00044E050E06EE170E082E692E00E944D9D40
:1087E000D9C365E276E0C8010E948A99892BD1F449
:1087F0008091620290916302A0916402B09165023F
:1088000098608093620290936302A0936402B09395
:10881000650244E050E06EE170E082E692E00E9482
:108820004D9DB8C30E942F0AB5C360917B02709121
:108830007C0280E090E00E947699FC012081233246
:10884000C1F44AE050E060E070E001960E94FC95BF
:108850007B836A8360917B0270917C0280E090E070
:108860000E9476992A813B81243031050CF096C014
:1088700002C01B821A82009709F490C01982BE01BF
:108880006F5F7F4F0E942F2A19013A014B01B82FC9
:10889000A92F8AE02A813B81829FF001839FF00DFE
:1088A0001124E355F44E4080518032813C83838112
:1088B0008D8394819E8325812F833681388787819C
:1088C00089879101A301B4018B2F9A2F5201CC808B
:1088D000DD80EE80FF80088519850E948D9509F462
:1088E00060C08981811103C0208231822AC018169C
:1088F00084F4422853289C81692A2D81722A3E8162
:10890000832A8F81982A9885B92B2985A22B4082AA
:1089100017C0209430946094709480949094B09593
:10892000A095242053203C8163228D8178229E8152
:1089300089222F8192223885B3238985A82320821A
:1089400051826282738284829582B683A78348E2D1
:1089500050E062E270E08DEA9BE10E944D9D8CE563
:1089600094E09F938F930E94499A8AE02A813B81E9
:10897000829FF001839FF00D1124E355F44E208176
:1089800031814281538164817581868197810E9402
:108990008F260E94B60D0F900F9003C082E00E94B8
:1089A000D12B80E594E09F938F930E94499A2FEFFB
:1089B0003FEF4FEF5FEF6FEF7FEF8FEF9FEF0E9483
:1089C0008F260E94B60D80917D020F900F90882314
:1089D00009F4E0C21F928F938DE494E09F938F93EC
:1089E0000E94499A0F900F900F900F90D3C2609100
:1089F0007B0270917C0280E090E00E947699FC01FD
:108A000020812332A1F44AE050E060E070E001965A
:108A10000E94FC958B0160917B0270917C0280E04A
:108A200090E00E94769904301105ECF402C000E059
:108A300010E00097C1F04AE050E060E070E00E9472
:108A400027972AE0209FF001219FF00D1124E35584
:108A5000F44E7187608748E250E062E270E08DEA90
:108A60009BE10E944D9D81E00E94D12B80917D026F
:108A7000882309F48FC21F928F938AE494E09F9316
:108A80008F930E94499A0F900F900F900F9082C27F
:108A90000E94735F80917D02882309F47BC21F923C
:108AA0008F9387E494E09F938F930E94499A0F904D
:108AB0000F900F900F906EC20E94962C80917D02B5
:108AC000882309F467C21F928F9384E494E09F93F4
:108AD0008F930E94499A0F900F900F900F905AC257
:108AE00080E090E00E947D2380917D02882309F43C
:108AF00051C21F928F9381E494E09F938F930E94C1
:108B0000499A0F900F900F900F9044C28091CA2BFA
:108B100081FF2DC00E940921892B49F58091C12731
:108B20008F938091C0278F938091BF278F938091DF
:108B3000BE278F9386E394E09F938F930E94499A78
:108B40008091A2348F938091A1348F938091A0342F
:108B50008F9380919F348F9389E294E09F938F93BA
:108B60000E94499A0FB6F894DEBF0FBECDBF0E9497
:108B7000B60D8091CA2B9091CB2B90FF63C081E002
:108B800090E00E9480207B011C0180E090E00E9428
:108B900080204B018C010E94DE1F3F922F92FF929A
:108BA000EF9288E194E09F938F930E94499A1F93DC
:108BB0000F939F928F9288E094E09F938F930E94EF
:108BC000499A240138019401A80147018101B701A4
:108BD000C1010E947D1E9F938F937F936F938DEFB2
:108BE00093E09F938F930E94499A242D352D462D13
:108BF000572D6E2D792D822D912F0E94DE1E9F9371
:108C00008F937F936F938FEE93E09F938F930E9448
:108C1000499A242D352D462D572D6E2D792D822DD7
:108C2000912F0E943F1F9F938F937F936F938CEDA3
:108C300093E09F938F930E94499A0FB6F894DEBFFA
:108C40000FBECDBF0E94B60D80917D02882309F42E
:108C5000A1C11F928F9389ED93E09F938F930E9400
:108C6000499A0F900F900F900F9094C18091CA2B4A
:108C700082FF2BC021E048E061E083E00E945B15A9
:108C80008091B11C8F938091B01C8F938091AF1C09
:108C90008F938091AE1C8F938091AD1C8F938091A8
:108CA000AC1C8F938091AB1C8F938091AA1C8F93E7
:108CB00082EC93E09F938F930E94499A0E94B60D95
:108CC0000FB6F894DEBF0FBECDBF8091CA2B909136
:108CD000CB2B91FF3BC00E94BF1920E030E048EC55
:108CE00052E4162F072FF82EE92E0E94489220E812
:108CF00036EE45EC57E40E949C8F21E03EED42E4C5
:108D00005EE30E94B5929B01AC0160E070E080E8F8
:108D10009FE30E94B88E2BE43AE34DEB57E30E94A9
:108D20009C8F9F938F937F936F93EF92FF920F93FC
:108D30001F9389EA93E09F938F930E94499A0E9420
:108D4000B60D0FB6F894DEBF0FBECDBF80917D0289
:108D5000882309F41FC11F928F9386EA93E09F93A3
:108D60008F930E94499A0F900F900F900F9012C10D
:108D700060917B0270917C0280E090E00E94769985
:108D80006BEA76E00E948A99892BB1F460917B02AC
:108D900070917C0280E090E00E947699009709F43F
:108DA000F9C00E946398803108F0F4C0909152019C
:108DB000892B80935201EEC0809152018F701F92D7
:108DC0008F938AEE91E09F938F930E94499A0E941D
:108DD000B60D0F900F900F900F90DCC060917B024A
:108DE00070917C0280E090E00E947699009711F1EA
:108DF0004AE050E060E070E00E94FC95603198F439
:108E0000609360021F926F9389E993E09F938F9321
:108E10000E94499A41E050E06BE170E080E692E008
:108E20000E944D9D11C0809160021F928F9380E936
:108E300093E006C0809160021F928F9387E893E0D1
:108E40009F938F930E94499A0F900F900F900F90CD
:108E50000E94B60D80917D02882309F49BC01F9269
:108E60008F9384E893E09F938F930E94499A0F9089
:108E70000F900F900F908EC060917B0270917C02DA
:108E800080E090E00E9476998C016CE975E00E9488
:108E90008A99892BE1F40E94706D80916202909111
:108EA0006302A0916402B0916502906180936202B6
:108EB00090936302A0936402B093650244E050E093
:108EC0006EE170E082E692E00E944D9D63C06FE922
:108ED00075E0C8010E948A99892B99F5F8940E943F
:108EE0007D6D0FB6F894A89580916000886180939D
:108EF0006000109260000FBE84B7877F84BF8091AE
:108F00006000886180936000109260007894809186
:108F1000620290916302A0916402B09165029F7E0B
:108F20008093620290936302A0936402B0936502FF
:108F300044E050E06EE170E082E692E00E944D9DD8
:108F400029C060EB76E0C8010E948A9940916202D4
:108F5000509163026091640270916502892B21F443
:108F600054FF18C0F894FFCF54FD03C08FE995E07B
:108F700002C08CE995E09F938F9386EE91E09F93DA
:108F80008F930E94499A0F900F900F900F9002C0FC
:108F90000E94A721EA85FB851182108283E02B962F
:108FA0000FB6F894DEBF0FBECDBFDF91CF911F91FA
:108FB0000F91FF90EF90DF90CF90BF90AF909F9078
:108FC0008F907F906F905F904F903F902F9008957B
:108FD000CF93DF93EC0188819981009741F0803D28
:108FE000914109F48CC01982188283E093C00E94D9
:108FF00025328091620280FD05C081FF01C01D9B6A
:109000000E94BE6E809170008C7F80937000809172
:10901000B60080628093B6001092B20082E0809326
:10902000B1008091B6008770E1F780917000816097
:10903000809370006DE47AE080E090E00E944A6DD9
:109040000E94C32280E00E94A12488EA90E19F93BD
:109050008F930E94499A0E9444128091CA2B0F90CC
:109060000F9086FD0E94BE678091CA2B9091CB2BFA
:1090700090FD0E94961F8091CA2B87FF06C021E0B9
:109080004CE061E080ED0E94616880913D0A0E94A1
:109090006371809161020E940B700E94087080933E
:1090A000720A809161020E940B7080913D0A1F92AA
:1090B0008F938091720A1F928F9385EB96E09F9316
:1090C0008F930E94359A1092740A1092730A0F902F
:1090D0000F900F900F900F900F9082E592E0909379
:1090E0009D3480939C3483E290E09093851280932A
:1090F000841280ED91E19983888381E00BC0633213
:10910000E1F749EF5FE260E070E083E79AE00E94F8
:109110009033E3CFDF91CF9108950F931F93CF93B7
:10912000DF93EC018A0188819981009711F1853ED6
:10913000914121F01982188283E020C06231E9F464
:10914000A80162E170E083E79AE00E94903384E036
:10915000809381341092833410928234109385343A
:109160000093843441E854E362E18EE392E00E948C
:10917000445B85EE91E19983888381E0DF91CF9113
:109180001F910F910895AF92BF92CF92DF92EF920D
:10919000FF920F931F93CF93DF93EC018091410ACD
:1091A0009091420AA091430AB091440A81FD08C0FF
:1091B0009091620290FD04C091FF57C01D9B55C065
:1091C0005A018B01FB01C384D484E584F684A4E6B0
:1091D000B0E0A70196010E94CA93672F782F892FCC
:1091E000992724E630E040E050E00E945B937F93B3
:1091F0006F93CD2CDE2CEF2CFF24DF92CF92F80161
:1092000086811F928F9385811F928F9388818F70A3
:109210001F928F9389811F928F93F50181811F92F5
:109220008F9380811F928F932296DF93CF9387EC49
:1092300096E09F938F930E94359A80917D02EDB7BF
:10924000FEB774960FB6F894FEBF0FBEEDBF88232D
:1092500061F01F928F9380EE91E09F938F930E9415
:10926000499A0F900F900F900F90DF91CF911F911F
:109270000F91FF90EF90DF90CF90BF90AF90089547
:109280008436910514F19F938F938BE097E09F9321
:109290008F930E94359A8091D42F9091D52FA091D1
:1092A000D62FB091D72F0196A11DB11D8093D42F39
:1092B0009093D52FA093D62FB093D72F0F900F90C8
:1092C0000F900F9081E090E0089580E090E0089585
:1092D0002F923F924F925F926F927F928F929F92C6
:1092E000AF92BF92CF92DF92EF92FF920F931F93B4
:1092F000CF93DF93CDB7DEB7CC59D1090FB6F89431
:10930000DEBF0FBECDBFCB56DF4F99838883C559D3
:10931000D0408A01633871F487E79AE0C456DF4F82
:109320006883CC59D0400E948359C456DF4F68816E
:10933000CC59D040CB56DF4FA881B981C559D04018
:109340002D913C912D37B1E13B0709F4EDC340F479
:109350002115310581F0213B3F4009F42FC423C47E
:109360002F3841E1340709F4FFC32639314111F4A4
:109370000C94AC5618C444EF52E061E870E087E703
:109380009AE00E94685981EB9FE0C5C35A01E3E06F
:10939000F0E0EC0FFD1FE40FF51F1082CA010E94E0
:1093A0004049892B81F720E030E040E050E0CC5686
:1093B000DF4F6881C459D040627070E080E090E077
:1093C000A0E00E94969509F094C6212F287030E005
:1093D00040E050E060E070E080E090E0A0E00E94BB
:1093E000969599F127E04AE250E06BE270E089E25D
:1093F00090E00E94A16383E994E30E941066BC019F
:10940000990F880B990B0E94509020E030E048ECB7
:1094100052E40E949C8F9F938F937F936F938FE36F
:1094200097E09F938F931F9287E78F93CE018A0DCA
:109430009B1D03969F938F930E94A19AA80EB91E1D
:109440000FB6F894DEBF0FBECDBF212F207130E0E4
:1094500040E050E060E070E080E090E0A0E00E943A
:109460009695E9F126E04AE250E06BE270E089E28D
:1094700090E00E94A16381E090E00E944E0D8093F5
:109480003C0A86E09CE10E941066BC01990F880BA3
:10949000990B0E94509020E030E048EC52E40E948A
:1094A0009C8F9F938F937F936F9389E497E09F9313
:1094B0008F931F9287E78F93C501029621E030E0DA
:1094C0002C0F3D1F820F931F9F938F930E94A19A91
:1094D000A80EB91E0FB6F894DEBF0FBECDBFC2579F
:1094E000DF4F2881CE58D04030E040E050E060E0CF
:1094F00070E080E090E0A0E00E94969501F10E946B
:109500000A0D9F938F937F936F9384E597E09F93CA
:109510008F931F9287E78F93C5010296A1E0B0E079
:10952000AC0FBD1F8A0F9B1F9F938F930E94A19A20
:10953000A80EB91E0FB6F894DEBF0FBECDBF212F07
:10954000207430E040E050E060E070E080E090E0C7
:10955000A0E00E94969531F18091CF2F8F9380915A
:10956000CE2F8F938091CD2F8F938091CC2F8F937F
:1095700082E697E09F938F931F9287E78F93C501B1
:10958000029621E030E02C0F3D1F820F931F9F9326
:109590008F930E94A19AA80EB91E0FB6F894DEBF51
:1095A0000FBECDBF212F207830E040E050E060E0DA
:1095B00070E080E090E0A0E00E94969541F1F89480
:1095C0008091793490917A34A0917B34B0917C343D
:1095D0007894BF93AF939F938F9380E797E09F9387
:1095E0008F931F9287E78F93C5010296A1E0B0E0A9
:1095F000AC0FBD1F8A0F9B1F9F938F930E94A19A50
:10960000A80EB91E0FB6F894DEBF0FBECDBF20E086
:10961000302F317040E050E060E070E080E090E09A
:10962000A0E00E94969509F076C520E0302F3270B8
:1096300040E050E060E070E080E090E0A0E00E9458
:10964000969509F0E6C520E0302F347040E050E0F8
:1096500060E070E080E090E0A0E00E94969509F064
:1096600009C620E0302F387040E050E060E070E044
:1096700080E090E0A0E00E94969509F02AC620E0E4
:10968000302F307140E050E060E070E080E090E02A
:10969000A0E00E94969509F09AC620E0302F307223
:1096A00040E050E060E070E080E090E0A0E00E94E8
:1096B000969509F0BCC620E030E040E050E0CC5682
:1096C000DF4F6881C459D040647070E080E090E062
:1096D000A0E00E94969509F0D8C620E0C856DF4F5A
:1096E0003881C859D04040E050E060E070E080E050
:1096F00090E0A0E00E94969509F034C720E0C7569C
:10970000DF4F3881C959D04040E050E060E070E060
:1097100080E090E0A0E00E94969509F051C7CE56F7
:10972000DF4F5881C259D0405170952E20E030E073
:10973000452F50E060E070E080E090E0A0E00E9403
:10974000969509F06BC720E030E0CE56DF4F488198
:10975000C259D040427050E060E070E080E090E09C
:10976000A0E00E94969509F08CC720E030E0C65733
:10977000DF4F4881CA58D04050E060E070E080E0A0
:1097800090E0A0E00E94969509F0AEC720E030E09E
:10979000CE56DF4F4881C259D040487050E060E05B
:1097A00070E080E090E0A0E00E94969509F0C6C7C6
:1097B00020E030E0CE56DF4F4881C259D0404071A2
:1097C00050E060E070E080E090E0A0E00E949695BC
:1097D00009F0E5C720E030E0CE56DF4F4881C2599E
:1097E000D040407250E060E070E080E090E0A0E0A7
:1097F0000E94969511F00C94005420E030E0CE5673
:10980000DF4F4881C259D040407450E060E070E0C2
:1098100080E090E0A0E00E94969511F00C94335403
:10982000CE56DF4FF881C259D040F0787F2E20E02D
:1098300030E04F2F50E060E070E080E090E0A0E08A
:109840000E94969511F00C946654CD56DF4F2881F6
:10985000C359D0402170622E20E030E040E0562D08
:1098600060E070E080E090E0A0E00E94969511F446
:109870000C94BF568091CA2B82FD02C00C94AE544A
:1098800021E046E061E083E00E945B1520E030E0EB
:10989000472D50E060E070E080E090E0A0E00E94A2
:1098A000969511F40C94AE548091CA2B82FF02C09D
:1098B0000C94735420E030E040E0CD56DF4F5881E7
:1098C000C359D040527060E070E080E090E0A0E0CA
:1098D0000E94969511F00C94E35420E030E040E0B3
:1098E000CD56DF4F5881C359D040547060E070E0CE
:1098F00080E090E0A0E00E94969511F00C9416553F
:1099000020E030E040E0CD56DF4F5881C359D040D1
:10991000507160E070E080E090E0A0E00E949695D9
:1099200011F00C94495520E030E040E0CD56DF4F77
:109930005881C359D040507260E070E080E090E000
:10994000A0E00E94969511F00C94885520E030E03C
:1099500040E0CD56DF4F5881C359D040507460E08D
:1099600070E080E090E0A0E00E94969511F00C94E9
:10997000C75520E030E040E0CD56DF4F5881C35955
:10998000D040587060E070E080E090E0A0E00E947D
:10999000969511F00C94065620E030E040E0C65653
:1099A000DF4F5881CA59D04060E070E080E090E01D
:1099B000A0E00E94969511F00C94375620E030E01C
:1099C000492D50E060E070E080E090E0A0E00E946F
:1099D000969511F00C946E56212F302FCE56DF4FF6
:1099E0004881C259D040CD56DF4F5881C359D0402D
:1099F000CC56DF4F6881C459D0407D2DC956DF4F0A
:109A00008881C759D0409C2DA0E00E94969511F006
:109A10000C947956809160028061898380916B0AF1
:109A20008A83FE01EA0DFB1D13828091410A909109
:109A3000420AA091430AB091440A85010D5F1F4F6D
:109A400080FF0CC01F930F9380E099E09F938F934A
:109A50000E94359A0F900F900F900F90B801CE0191
:109A600001960E9498628091620282FF0AC029E7F3
:109A700030E3A801BE016F5F7F4F8BE692E00E944A
:109A800024678091410A9091420AA091430AB091C3
:109A9000440A82FD73980E94066F87E79AE00E944D
:109AA00085598091620290916302A0916402B09105
:109AB000650290FF40C03FEFA31AB30A0E940870EE
:109AC000F82E89E10E9420708091620290916302D9
:109AD000A0916402B091650290FF29C073988091B3
:109AE0006B0A8F5F80936B0A8A83B5016F5F7F4F2C
:109AF000CE0101960E94986287E79AE00E948559FC
:109B000040E050E065E880918812909189120E94AF
:109B1000445B8DE791E1CB56DF4FA881B981C559F0
:109B2000D0408D939C933CC0A12CB12CCDCF8F2DD8
:109B30000E942070739A80913E0A90913F0A892B6F
:109B400011F00E94BE6E80916B0A8F5F80936B0A4A
:109B50008091410A9091420AA091430AB091440A2F
:109B600082FF11CC739A0FCC83E69AE00E94F05DDD
:109B7000892BB1F00E94066F8091620287FD2B98BD
:109B800060E470E083E69AE00E94C95D86E991E1B5
:109B9000CB56DF4FE881F981C559D040918380834E
:109BA00081E00C94CF56CB56DF4FA881B981C559BF
:109BB000D0401D921C9283E00C94CF56623181F705
:109BC0008090620290906302A0906402B09065025F
:109BD00091FCD9CBF8018081813021F50180F2819F
:109BE000E02D108101812281CE56DF4F2883C2599A
:109BF000D0403381CD56DF4F3883C359D0404481A4
:109C0000CC56DF4F4883C459D040D5805681C956C1
:109C1000DF4F5883C759D040C780E084F184212C9E
:109C2000312C52C08230B9F423803480E12CF12CE5
:109C300011E000E0CE56DF4F1882C259D040B0E8A4
:109C4000CD56DF4FB883C359D040CC56DF4F188272
:109C5000C459D04032C08330D1F0843009F093CB66
:109C6000E12CF12C212C312C15E000E0CE56DF4FF9
:109C70001882C259D040CD56DF4F1882C359D04008
:109C8000E2E0CC56DF4FE883C459D04016C0E12C47
:109C9000F12C212C312C15E000E0CE56DF4F18823C
:109CA000C259D040CD56DF4F1882C359D040F1E0A1
:109CB000CC56DF4FF883C459D040D12CC956DF4F62
:109CC0001882C759D040C12C4090CC2F5090CD2F36
:109CD0006090CE2F7090CF2F20918A0230918B020E
:109CE00040918C0250918D02C657DF4F28833983F3
:109CF0004A835B83CA58D0402DEC3CEC4CE45EE3D5
:109D0000C657DF4F688179818A819B81CA58D040CC
:109D10000E94B98E9B01AC01C301B2010E947591F2
:109D200087FD0BC0E894A0F88092620290926302D3
:109D3000A0926402B092650246C0C657DF4F2881E8
:109D400039814A815B81CA58D040C301B2010E9467
:109D5000978F87FF38C08091D82F9091D92FA091ED
:109D6000DA2FB091DB2F0196A11DB11D8093D82F62
:109D70009093D92FA093DA2FB093DB2FA0FC03CBC5
:109D80006894A0F88092620290926302A0926402AA
:109D9000B092650215E400E2CE56DF4F1882C25938
:109DA000D040CD56DF4F1882C359D04034E0CC5656
:109DB000DF4F3883C459D040D12CC956DF4F1882A9
:109DC000C759D040C12CCE56DF4F4881C259D04030
:109DD0004470C657DF4F4883CA58D04020E030E077
:109DE00050E060E070E080E090E0A0E00E94969596
:109DF00009F08C9A512F5072C257DF4F5883CE58BA
:109E0000D040252F30E040E050E060E070E080E09E
:109E100090E0A0E00E94969511F00E940A0D802F1C
:109E20008074C856DF4F8883C859D04020E0382F4F
:109E300040E050E060E070E080E090E0A0E00E9450
:109E4000969511F00E940921902F9078C756DF4F08
:109E50009883C959D04020E0392F40E050E060E0BD
:109E600070E080E090E0A0E00E94969551F00E94A2
:109E7000A50C6093863470938734809388349093D4
:109E80008934212F217030E040E050E060E070E044
:109E900080E090E0A0E00E949695F1F084E99BE1DB
:109EA0009F938F938FE197E09F938F931F9287E704
:109EB0008F93CE0103969F938F930E94A19A4C019A
:109EC0000E9440490FB6F894DEBF0FBECDBF892B6C
:109ED00009F059CA540102C0A12CB12C212F2270C3
:109EE00030E040E050E060E070E080E090E0A0E032
:109EF0000E949695D1F1C501029667E277E0E1E014
:109F0000F0E0EC0FFD1F8E0F9F1F0E949399F3E06E
:109F1000AF0EB11C23E9622E24E3722E3EEF832E96
:109F200033E0932E47E7542ED3018D913D011F92CC
:109F30008F939F928F921F925F92C5010296E1E0EC
:109F4000F0E0EC0FFD1F8E0F9F1F9F938F930E94D9
:109F5000A19AA80EB91E0FB6F894DEBF0FBECDBFF2
:109F60003BE9631634E37306F9F6212F247030E0E1
:109F700040E050E060E070E080E090E0A0E00E940F
:109F8000969509F450C0C50102966BE277E041E076
:109F900050E04C0F5D1F840F951F0E94939954E071
:109FA000A50EB11C2E018AE7480E511C80E1D2019A
:109FB0001D928A95E9F728E0A20168E980EB0E94EA
:109FC000A6133201B8E06B0E711C9EEF892E93E050
:109FD000992E27E7F20181912F011F928F939F9273
:109FE0008F921F922F93C501029641E050E04C0FD3
:109FF0005D1F840F951F9F938F93C556DF4F288356
:10A00000CB59D0400E94A19AA80EB91E0FB6F89461
:10A01000DEBF0FBECDBFC556DF4F2881CB59D04024
:10A0200046145704B9F6CD56DF4F9881C359D04036
:10A030009078C656DF4F9883CA59D04020E030E070
:10A0400040E0592F60E070E080E090E0A0E00E94E6
:10A050009695E1F480913E0A90913F0A9F938F93E9
:10A0600080E397E09F938F931F9287E78F93CE01B2
:10A070008A0D9B1D03969F938F930E94A19AA80E11
:10A08000B91E0FB6F894DEBF0FBECDBF20E030E0A2
:10A0900040E050E0CC56DF4F6881C459D040617039
:10A0A00070E080E090E0A0E00E94969509F47BC902
:10A0B000E3E0F0E0EC0FFD1FEA0DFB1D80E2808382
:10A0C000A50183E090E08A199B09FC01E40FF51FCC
:10A0D000E750F04D20814F5F5F4F222309F456C9AE
:10A0E0002081E1E0F0E0EC0FFD1FE40FF51F22837B
:10A0F000ECCFCE018A0D9B1D67E377E003960E94AB
:10A100009399B7E0AB0EB11CC5010E944049892B61
:10A1100009F039C95AC9E114F10409F486CAF8945E
:10A120004090793450907A3460907B3470907C34D5
:10A1300078948091FE1B9091FF1BA091001CB09120
:10A14000011CA3019201281B390B4A0B5B0BCA01AE
:10A15000B9010E944E90C257DF4F688379838A838A
:10A160009B83CE58D040B70180E090E00E944E9093
:10A170009B01AC01C257DF4F688179818A819B8145
:10A18000CE58D0400E949C8F4C019F928F937F931A
:10A190006F938BE797E09F938F931F9287E78F933F
:10A1A0009E012A0D3B1D2D5F3F4F3F932F93C456B9
:10A1B000DF4F6883CC59D040C556DF4F7883CB59E9
:10A1C000D0400E94A19AA80EB91EC456DF4F6881E4
:10A1D000CC59D040C556DF4F7881CB59D040862F1F
:10A1E000972FA82DB92D80938B3490938C34A09306
:10A1F0008D34B0938E344092FE1B5092FF1B6092C0
:10A20000001C7092011C0FB6F894DEBF0FBECDBFCC
:10A210000CCAE114F10409F416CAF8948091D51B14
:10A220009091D61BA091D71BB091D81B78949F9387
:10A230008F93809169028F93809168028F9388E851
:10A2400097E09F938F931F9287E78F93C5010296A4
:10A25000A1E0B0E0AC0FBD1F8A0F9B1F9F938F93AF
:10A260000E94A19AA80EB91E0FB6F894DEBF0FBEC9
:10A27000CDBFE9C9F89480917D3490917E34A0914E
:10A280007F34B09180347894BF93AF939F938F9332
:10A2900088E997E09F938F931F9287E78F93C5017B
:10A2A000029621E030E02C0F3D1F820F931F9F93F9
:10A2B0008F930E94A19AA80EB91EC5010E94404921
:10A2C0000FB6F894DEBF0FBECDBF892B09F05BC877
:10A2D000C8C9E114F10409F4D2C9F89440907D345E
:10A2E00050907E3460907F34709080347894809168
:10A2F000021C9091031CA091041CB091051CA301A9
:10A300009201281B390B4A0B5B0BCA01B9010E9451
:10A310004E90C257DF4F688379838A839B83CE58E0
:10A32000D040B70180E090E00E944E909B01AC01CC
:10A33000C257DF4F688179818A819B81CE58D04096
:10A340000E949C8F4C019F928F937F936F9383EA1F
:10A3500097E09F938F931F9287E78F939E012A0D1B
:10A360003B1D2D5F3F4F3F932F93C456DF4F6883B4
:10A37000CC59D040C556DF4F7883CB59D0400E948E
:10A38000A19AA80EB91EC456DF4F6881CC59D0409F
:10A39000C556DF4F7881CB59D040862F972FA82DF7
:10A3A000B92D80938F3490939034A0939134B093CF
:10A3B00092344092021C5092031C6092041C7092D2
:10A3C000051C0FB6F894DEBF0FBECDBF58C9EF28ED
:10A3D00009F463C9F8948091D91B9091DA1BA0917C
:10A3E000DB1BB091DC1B78949F938F938091670265
:10A3F0008F93809166028F9380EB97E09F938F936A
:10A400001F9287E78F93C5010296A1E0B0E0AC0FE1
:10A41000BD1F8A0F9B1F9F938F930E94A19AA80E26
:10A42000B91E0FB6F894DEBF0FBECDBF36C98091FE
:10A43000D02F9091D12FA091D22FB091D32FBF9335
:10A44000AF939F938F9380EC97E09F938F931F928E
:10A4500087E78F93C501029621E030E02C0F3D1F66
:10A46000820F931F9F938F930E94A19AA80EB91EEB
:10A47000C5010E9440490FB6F894DEBF0FBECDBFA4
:10A48000892B11F00C94C34916C98091DB2F8F934F
:10A490008091DA2F8F938091D92F8F938091D82F2D
:10A4A0008F938091D72F8F938091D62F8F93809108
:10A4B000D52F8F938091D42F8F938BEC97E09F9320
:10A4C0008F931F9287E7982E9F92C5010296A1E075
:10A4D000B0E0AC0FBD1F8A0F9B1F9F938F930E940C
:10A4E000A19AA80EB91EC5010E9440490FB6F89462
:10A4F000DEBF0FBECDBF892B11F00C94C3498091F4
:10A50000CA2B9091CB2B90FFE8C88091DF2F8F93BF
:10A510008091DE2F8F938091DD2F8F938091DC2FA0
:10A520008F938FEE97E09F938F931F929F92C50119
:10A53000029621E030E02C0F3D1F820F931F9F9366
:10A540008F930E94A19AA80EB91EC5010E9440498E
:10A550000FB6F894DEBF0FBECDBF892B11F00C945F
:10A56000C349BBC88091C1278F938091C0278F9327
:10A570008091BF278F938091BE278F9381E098E0D1
:10A580009F938F931F9287E78F93C5010296A1E057
:10A59000B0E0AC0FBD1F8A0F9B1F9F938F930E944B
:10A5A000A19AA80EB91EC5010E9440490FB6F894A1
:10A5B000DEBF0FBECDBF892B11F00C94C3499EC8DE
:10A5C000809189348F93809188348F9380918734E0
:10A5D0008F93809186348F938CE098E09F938F9334
:10A5E0001F9287E78F93C501029621E030E02C0F80
:10A5F0003D1F820F931F9F938F930E94A19AA80ED5
:10A60000B91EC5010E9440490FB6F894DEBF0FBEC7
:10A61000CDBF892B11F00C94C34981C881E00E9401
:10A62000570C209182023091830240918402509114
:10A6300085020E9448929F938F937F936F9389E145
:10A6400098E09F938F931F9287E78F93C50102969F
:10A65000A1E0B0E0AC0FBD1F8A0F9B1F9F938F93AB
:10A660000E94A19AA80EB91EC5010E9440490FB6CA
:10A67000F894DEBF0FBECDBF892B11F00C94C349F7
:10A6800062C882E00E94570C20917E0230917F02C6
:10A6900040918002509181020E9448929F938F9333
:10A6A0007F936F9386E298E09F938F931F9287E743
:10A6B0008F93C501029621E030E02C0F3D1F820FE1
:10A6C000931F9F938F930E94A19AA80EB91EC50154
:10A6D0000E9440490FB6F894DEBF0FBECDBF892B54
:10A6E00011F00C94C34941C883E00E94570C9F931A
:10A6F0008F937F936F9383E398E09F938F931F9241
:10A7000087E78F93C5010296A1E0B0E0AC0FBD1FB3
:10A710008A0F9B1F9F938F930E94A19AA80EB91E28
:10A720008C98C5010E9440490FB6F894DEBF0FBE59
:10A73000CDBF892B11F00C94C34928C88091CA2B36
:10A7400087FF36C821E042E161E080ED0E94616848
:10A750009F938F937F936F9380E498E09F938F9361
:10A760001F9287E78F93C501029621E030E02C0FFE
:10A770003D1F820F931F9F938F930E94A19AA80E53
:10A78000B91EC5010E9440490FB6F894DEBF0FBE46
:10A79000CDBF892B11F00C94C3490C94D84B8091F8
:10A7A000CA2B87FF17C821E042E162E080ED0E94DA
:10A7B00061689F938F937F936F938EE498E09F934C
:10A7C0008F931F9287E78F93C5010296A1E0B0E0B7
:10A7D000AC0FBD1F8A0F9B1F9F938F930E94A19A5E
:10A7E000A80EB91EC5010E9440490FB6F894DEBFFD
:10A7F0000FBECDBF892B11F00C94C3490C94EA4BCA
:10A800008091CA2B87FD02C00C94FD4B21E042E1F0
:10A8100063E080ED0E9461689F938F937F936F93B5
:10A820008CE598E09F938F931F9287E78F93C501E4
:10A83000029621E030E02C0F3D1F820F931F9F9363
:10A840008F930E94A19AA80EB91EC5010E9440498B
:10A850000FB6F894DEBF0FBECDBF892B11F00C945C
:10A86000C3490C94FD4B8091CA2B87FD02C00C9408
:10A87000104C21E042E164E080ED0E9461689F930A
:10A880008F937F936F938AE698E09F938F931F92A5
:10A8900087E78F93C5010296A1E0B0E0AC0FBD1F22
:10A8A0008A0F9B1F9F938F930E94A19AA80EB91E97
:10A8B000C5010E9440490FB6F894DEBF0FBECDBF60
:10A8C000892B11F00C94C3490C94104C8091CA2B25
:10A8D00082FD02C00C94254C46E061E083E00E94BA
:10A8E0005B150C94254C8091AD1C8F938091AC1C12
:10A8F0008F938091AB1C8F938091AA1C8F9388E7D4
:10A9000098E09F938F931F9287E78F93C5010296DC
:10A9100041E050E04C0F5D1F840F951F9F938F9374
:10A920000E94A19AA80EB91EC5010E9440490FB607
:10A93000F894DEBF0FBECDBF892B11F00C94C34934
:10A9400020E030E040E0562D60E070E080E090E0F4
:10A95000A0E00E94969511F40C945A4C8091CA2B59
:10A9600082FD02C00C945A4C8091B11C8F9380914F
:10A97000B01C8F938091AF1C8F938091AE1C8F93EE
:10A9800080E898E09F938F931F9287E78F93C5018C
:10A990000296E1E0F0E0EC0FFD1F8E0F9F1F9F93EA
:10A9A0008F930E94A19AA80EB91EC5010E9440492A
:10A9B0000FB6F894DEBF0FBECDBF892B11F00C94FB
:10A9C000C3490C945A4C8091CA2B9091CB2B90FD8B
:10A9D00002C00C946D4C80E090E00E9480209F9318
:10A9E0008F937F936F938BE898E09F938F931F9241
:10A9F00087E78F93C501029641E050E04C0F5D1F41
:10AA0000840F951F9F938F930E94A19AA80EB91E41
:10AA1000C5010E9440490FB6F894DEBF0FBECDBFFE
:10AA2000892B11F00C94C3490C946D4C8091CA2B66
:10AA30009091CB2B90FD02C00C94804C81E090E073
:10AA40000E9480209F938F937F936F938BE998E070
:10AA50009F938F931F9287E78F93C5010296E1E042
:10AA6000F0E0EC0FFD1F8E0F9F1F9F938F930E94AE
:10AA7000A19AA80EB91EC5010E9440490FB6F894CC
:10AA8000DEBF0FBECDBF892B11F00C94C3490C94CF
:10AA9000804C8091CA2B9091CB2B90FD02C00C94DE
:10AAA000934C81E090E00E9480202B013C0180E0EB
:10AAB00090E00E9480209B01AC01C301B2010E9482
:10AAC0007D1E9F938F937F936F938CEA98E09F9363
:10AAD0008F931F9287E78F93C501029641E050E064
:10AAE0004C0F5D1F840F951F9F938F930E94A19A17
:10AAF000A80EB91EC5010E9440490FB6F894DEBFEA
:10AB00000FBECDBF892B11F00C94C3490C94934C0C
:10AB10008091CA2B9091CB2B90FD02C00C94A64C37
:10AB200081E090E00E9480202B013C0180E090E0D9
:10AB30000E9480209B01AC01C301B2010E94DE1E75
:10AB40009F938F937F936F9387EB98E09F938F935F
:10AB50001F9287E78F93C5010296E1E0F0E0EC0FCA
:10AB6000FD1F8E0F9F1F9F938F930E94A19AA80E87
:10AB7000B91EC5010E9440490FB6F894DEBF0FBE52
:10AB8000CDBF892B11F00C94C3490C94A64C809135
:10AB9000CA2B9091CB2B90FD02C00C94B94C81E054
:10ABA00090E00E9480202B013C0180E090E00E9418
:10ABB00080209B01AC01C301B2010E943F1F9F9303
:10ABC0008F937F936F9385EC98E09F938F931F9261
:10ABD00087E78F93C501029641E050E04C0F5D1F5F
:10ABE000840F951F9F938F930E94A19AA80EB91E60
:10ABF000C5010E9440490FB6F894DEBF0FBECDBF1D
:10AC0000892B11F00C94C3490C94B94C8091CA2B38
:10AC10009091CB2B91FD02C00C94CC4C0E94BF199B
:10AC20009F938F937F936F9388ED98E09F938F937B
:10AC30001F9287E78F93C5010296E1E0F0E0EC0FE9
:10AC4000FD1F8E0F9F1F9F938F930E94A19AA80EA6
:10AC5000B91EC5010E9440490FB6F894DEBF0FBE71
:10AC6000CDBF892B11F00C94C3490C94CC4CD1016D
:10AC700016968C9116971F928F9315968C91159717
:10AC80001F928F9313968C9113971F928F93129606
:10AC90008C911F928F9389EE98E09F938F931F92D0
:10ACA00087E78F93C5010296E1E0F0E0EC0FFD1F0E
:10ACB0008E0F9F1F9F938F930E94A19AA80EB91E7B
:10ACC000C5010E9440490FB6F894DEBF0FBECDBF4C
:10ACD000892B11F00C94C3490C94DE4C779A809127
:10ACE000410A9091420AA091430AB091440A92FD10
:10ACF000749A8091410A9091420AA091430AB091BE
:10AD0000440A82FD0CC08091620280FD08C081FD72
:10AD100002C00C940A4D1D9902C00C940A4D40E0EB
:10AD200050E060E070E0CE0101960E94B80A809188
:10AD3000B31C90E02091380A3091390A82179307AA
:10AD400010F40C940A4D40E050E062E18CE092E097
:10AD50000E94445B0C940A4D83E69AE00E94F05DE9
:10AD6000892B11F40C94D04D0E94BE6E809162022A
:10AD700087FD02C00C94C3492B9A0C94C34920E070
:10AD800030E0472D50E060E070E080E090E0A0E02F
:10AD90000E94969511F00C94544C0C945A4CC45645
:10ADA000DF4F0FB6F894DEBF0FBECDBFDF91CF915E
:10ADB0001F910F91FF90EF90DF90CF90BF90AF90D9
:10ADC0009F908F907F906F905F904F903F902F90CB
:10ADD00008950C94AD594F925F926F927F92AF920B
:10ADE000BF92CF92DF92EF92FF920F931F93CF9378
:10ADF000DF93CDB7DEB760970FB6F894DEBF0FBE16
:10AE0000CDBF6B010E940870E82FF0E0EE0FFF1F2E
:10AE1000E953F44E808191810196918380838091E2
:10AE2000410A9091420AA091430AB091440A81FDDF
:10AE30007498409062025090630260906402709037
:10AE400065020E94EA617C01FC018081982F929545
:10AE50009F70913099F48F7051F48091AB1B909159
:10AE6000AC1B01969093AC1B8093AB1B38C1B60111
:10AE700083EA94E30E942159892B51F08091A91B08
:10AE80009091AA1B01969093AA1B8093A91B27C19E
:10AE9000D301C2013EE0B695A795979587953A955F
:10AEA000D1F7F82FF170AF2E82E89AE00E94335C60
:10AEB0008C01892B09F448C0B601C80102960E9492
:10AEC0002159892BE9F1980147E65AE060E074E6E0
:10AED000C8010F960E94B75EF7019181F801848145
:10AEE000981321C082858F5F82878091A71B9091E4
:10AEF000A81B01969093A81B8093A71B84E00E9437
:10AF00000963F801208530E02817390708F077C178
:10AF100084E00E940963F8018087F70180818F70C7
:10AF2000F8018187DCC0F801128684E00E94096381
:10AF3000F8018087F70180818F70F801818760C1F7
:10AF4000C8010E94DF5CB4CF84E092E00E94C75B3E
:10AF50008C01892B09F4C3C0B601C80102960E9476
:10AF60001859F70181818150F801848380E091E0D4
:10AF7000A0E0B0E083879487A587B687128684E037
:10AF80000E940963F8018087F70180818F70F801C2
:10AF90008187B80182E89AE00E94975C980147E6B1
:10AFA0005AE060E074E6C8010F960E94B75EBB24C9
:10AFB000B394F7018181F8018483F70180818F7058
:10AFC000F801878384E00E940963F801858383E0A8
:10AFD0000E940963F801868387818F3009F0B12CC4
:10AFE000F7014180F8018481481A512C612C712CA1
:10AFF00086E0440C551C661C771C8A95D1F7238586
:10B00000348545855685A0ECB0E00E94CA93BB27E5
:10B01000A92F982F872F480E591E6A1E7B1E438624
:10B02000548665867686A601B801C7010E94B80AD3
:10B030008091B31C90E02091380A3091390A821730
:10B04000930738F040E050E062E18CE092E00E942B
:10B05000445B8091380A9091390A029708F44BC0FA
:10B060008091CA2B86FF2AC00E94B067C70105964F
:10B070000E947C67F70181811F928F93F80186817E
:10B080001F928F9385811F928F9381E199E09F9307
:10B090008F931F9280E18F93CE0101966C019F9355
:10B0A0008F930E94A19A82E00E949667C6010E9437
:10B0B0007C670FB6F894DEBF0FBECDBF80916202F1
:10B0C00090916302A0916402B091650297FD4DC01A
:10B0D0008091380A9091390A029708F47AC08091D9
:10B0E000410A9091420AA091430AB091440A81FF1B
:10B0F00089C0749A87C08091620290916302A09186
:10B100006402B091650296FFABCFAA2009F4A8CFE4
:10B11000F7018081982F9F709230E8F09150807FE6
:10B12000892B808387E79AE00E94E9568091A51BCE
:10B130009091A61B01969093A61B8093A51B8091CE
:10B14000410A9091420AA091430AB091440A96FFA5
:10B1500087CF739885CF8091AB1B9091AC1B0196E4
:10B160009093AC1B8093AB1B7BCF84E99BE1209138
:10B17000941B222309F4ACCF9F938F9384E299E030
:10B180009F938F93CE0101963C019F938F930E94D2
:10B19000DE9A6C01B301C70102960E94B4990F9028
:10B1A0000F900F900F900F900F90009709F490CF91
:10B1B000EFEFCE1ADE0A8C0D9D1DAC010196FA014F
:10B1C00020812032D1F362E186E192E00E94445B6B
:10B1D0007FCFBB2009F483CF82E08093E52F1092CC
:10B1E000E72F1092E62F1093E92F0093E82F45EEFA
:10B1F0005FE262E18EE392E00E94445B70CFA12C9B
:10B20000B12CD7CE60960FB6F894DEBF0FBECDBF7F
:10B21000DF91CF911F910F91FF90EF90DF90CF9032
:10B22000BF90AF907F906F905F904F90089508957A
:10B23000FB012081FC012083FB012181FC01218392
:10B240000895FC019081DB018C91981309C021E0E5
:10B2500090E0318111968C91381320E0822F08956F
:10B2600080E090E00895BC0183EA94E30C941859BF
:10B27000DC011996ED91FC911A970280F381E02D83
:10B28000309709F0099408950F931F93CF93DF939C
:10B2900000D0CDB7DEB78C0188E10E941C63BC01F1
:10B2A000CE0101960E941859D8011996ED91FC9192
:10B2B0001A970190F081E02DBE016F5F7F4FC801AA
:10B2C00009950F900F90DF91CF911F910F910895E5
:10B2D000EF92FF920F931F93CF93DF938C01EB01BB
:10B2E0007A014EE053E00E949259F801F286E1861D
:10B2F00062E173E0CE01DF91CF911F910F91FF903A
:10B30000EF900C94EC590C94AB59CF93DF93EC0174
:10B3100063EA74E388E10E941263CE01DF91CF916A
:10B320000C94AD59EF92FF920F931F93CF93DF933D
:10B330008C01EB017A010E94C859F801F086E7827E
:10B3400066E173E0CE01DF91CF911F910F91FF90E5
:10B35000EF900C94EC590C94D0590C947E74DC0151
:10B360001796ED91FC9118970190F081E02D0994CA
:10B37000DC011796ED91FC9118970280F381E02D86
:10B38000309709F00994089586E892E10C942F5CB7
:10B39000FC0173836283BC0186E892E10C94975CA4
:10B3A000BC0186E892E10C94785CCF93DF93EC01CA
:10B3B00086E892E10E94335C009749F0FC0122810B
:10B3C00033812C173D0729F00E94DF5CF5CF80E028
:10B3D00090E0DF91CF9108950F931F93CF93DF9368
:10B3E0008B010E94D559EC01892B31F01D830C8310
:10B3F000C8010E94AC768E83DF91CF911F910F918F
:10B4000008951F93CF93DF93DC011496ED91FC9187
:10B4100015973097E1F0162FEC01909389128093E5
:10B42000881282E08887CD0106960995082E000CC7
:10B43000990B0297029710F0133839F4BE01CE0130
:10B44000DF91CF911F910C94315A81E08887DF9171
:10B45000CF911F910895FC01208520FD0C94015A85
:10B460000895CF92DF92EF92FF920F931F93CF93A5
:10B47000DF93E0908812F0908912C0908A12D090E9
:10B480008B12F601E817F90739F0309709F44BC031
:10B490000190F081E02DF6CF009709F444C08B01B4
:10B4A000EC018885882309F11886C114D10461F064
:10B4B000CC15DD0529F0AE0167E8C6010E942B5AC4
:10B4C000F601C080D180F1CFEC81FD81309769F029
:10B4D000C017D10751F0D0938912C093881240E071
:10B4E00050E063E8CE0106960995E0918A12F0914A
:10B4F0008B12CE17DF0741F48881998190938B12CC
:10B5000080938A120CC0FC01309749F080819181B0
:10B510008C179D07C1F78881998191838083F09270
:10B520008912E0928812DF91CF911F910F91FF90C5
:10B53000EF90DF90CF9008951F93CF93DF931092F9
:10B540009412C0918A12D0918B1211E0209779F059
:10B550008985882341F01887198640E050E062E829
:10B56000CE010E94015A0990D881C02DEFCFDF9102
:10B57000CF911F9108958091371391E0980F909388
:10B580003713089560918812709189120C94315A82
:10B590008AE8809337131092351310923613109265
:10B5A0008B1210928A1210928912109288120895AA
:10B5B0008091941281110E949C5A50913613552308
:10B5C00009F452C0E09135132E2F30E085E0E89F5A
:10B5D000F0011124EB56FD4E608160939312A1811E
:10B5E000B281B0939212A09391128381948190932F
:10B5F000901280938F122F5F3F4F2F71332720932C
:10B600003513515050933613009731F580918A12BB
:10B6100090918B1290938E1280938D1280918D1247
:10B6200090918E12892B01F18091941281110E94C8
:10B630009C5A409191125091921260919312809174
:10B640008D1290918E120E942B5AE0918D12F091E2
:10B650008E1280819181DECF613819F421E0FC01E6
:10B660002087AD010E942B5A8091941220913613AD
:10B6700090E0820F911D08958091941220913613CD
:10B6800090E0820F911D08959C01909136139032A5
:10B69000B9F0E0913513E90FEF71E0938C1285E07A
:10B6A000E89FF0011124EB56FD4E608352834183E5
:10B6B000348323839F5F9093361380E090E0089556
:10B6C00081E090E00895CF93DF93C0918812D091EC
:10B6D00089120E942B5AD0938912C0938812DF914D
:10B6E000CF910895AB0130918A1220918B12E32FF4
:10B6F000F22FE817F907B1F0309721F00190F081AF
:10B70000E02DF7CF009771F0FC01308321839093F7
:10B710008B1280938A1221E020871782168261E8BB
:10B720000C94635B0895009749F0FC01208521503B
:10B73000223020F421E0218720939412089521E003
:10B7400030E0FC018085811102C020E030E0C901B9
:10B750000895CF93DF93EC014A815B8160E070E054
:10B760008C819D810E9483992A813B818881998166
:10B77000289FA001299F500D389F500D112460E093
:10B7800070E08E819F81DF91CF910C948399FC01B1
:10B790008281938120E030E028173907D1F0A4811D
:10B7A000B581A20FB31F4C91411110C081E08C9361
:10B7B00080819181289FA001299F500D389F500DB5
:10B7C000112486819781840F951F08952F5F3F4F25
:10B7D000E3CF80E090E00895FC018681978142816B
:10B7E000538120E030E024173507D1F08617970702
:10B7F00081F4A481B581A20FB31F8C91181614F4A3
:10B8000081508C9384819581FC01E20FF31F80812C
:10B810000895A081B1818A0F9B1F2F5F3F4FE3CF17
:10B820008FEF0895FC012681378162177307A0F01E
:10B83000A081B18142815381A49FC001A59F900D39
:10B84000B49F900D1124280F391F81E090E06217FA
:10B85000730720F080E0089580E090E00895FC01F7
:10B86000118210820895FC01808191810895FB016D
:10B8700020813181FC01318320830895DC01ED9129
:10B88000FC91309741F080819181009711F0FC018B
:10B89000FACFCF01089580E090E00895DC01ED91AA
:10B8A000FC9111973097A9F020813181232B21F44D
:10B8B0001D921C92CF010895A081B1818D919C9120
:10B8C0001197892B11F0FD01F7CF11821082CD0164
:10B8D000089580E090E00895DC01ED91FC911197CE
:10B8E000309721F0208131812D933C93CF01089531
:10B8F000DC01ED91FC913097C9F0A0E0B0E0E617D3
:10B90000F70761F4FB0120813181109709F4DC0114
:10B910002D933C93FB011182108208952081318187
:10B92000DF012115310511F0F901E9CF08950F93D9
:10B930001F93CF93DF938C01EB010E94785C1982F7
:10B940001882C8010E943E5C009711F4F80101C002
:10B95000FC01D183C083DF91CF911F910F91089596
:10B960000F931F93CF93DF93EC018B010E94785CC0
:10B9700088819981F8019183808319830883DF91FD
:10B98000CF911F910F910895DC01ED91FC9180E022
:10B9900090E0309729F001960190F081E02DF9CFE9
:10B9A0000895FB01309719F4BA010C94B05C8081C2
:10B9B0009181DA018D939C93518340830895009780
:10B9C00021F0FC0180819181089580E090E008954C
:10B9D00080913A1390913B13892B29F410923913DB
:10B9E0001092381308950E94066CE0913A13F0917A
:10B9F0003B132281338140815181240F351F281B45
:10BA0000390B0480F581E02D309769F062817381F4
:10BA100040815181460F571F481B590B421753074E
:10BA200080F79A01EECF820F931F90933913809382
:10BA30003813089580E992E00C94935BEF92FF92A3
:10BA40000F931F93CF93DF938C01FC018081918131
:10BA5000009799F08A359105D9F0F801118210828A
:10BA600083E068C0868197818417950709F049C0F3
:10BA70000480F581E02D3097A9F710923B131092C6
:10BA80003A138AE590E0F8019183808381E052C007
:10BA9000673891F16238A9F7C0913A13D0913B13FE
:10BAA000E12CF12C209769F3CE010E94757A892B45
:10BAB000F1F0AE0168E88E819F810E94445B892B82
:10BAC000A1F41F821E828C819D81E114F10421F07A
:10BAD000F7019583848304C090933B1380933A13BA
:10BAE0001D821C820E94E85CD7CF0E941A5D7E01F5
:10BAF0000C80DD81C02DD6CFE0913A13F0913B133D
:10BB0000BACFF0933B13E0933A13A481B581109719
:10BB100009F4B7CF16968D919C91179784179507C6
:10BB200039F414968D919C91159795838483EDCF6C
:10BB3000FD01EBCFDF91CF911F910F91FF90EF901F
:10BB40000895CF93DF93EC010E941A5D2E813F810F
:10BB500090913A1380913B13232B59F0E92FF82F42
:10BB6000309739F0EC17FD0781F00480F581E02D66
:10BB7000F7CF20918812309189123F832E839C83C6
:10BB80008D83D0933B13C0933A13DF91CF910C94E4
:10BB9000E85CCF93DF93EC010E94557ACE01DF91F0
:10BBA000CF910C94A15DCF93DF93EC010E94617A59
:10BBB000CE01DF91CF910C94A15DCF93DF93EC0187
:10BBC0000E946B7ACE01DF91CF910C94A15DFC01B4
:10BBD00020813181620F731F718360830C94E85C54
:10BBE00021E030E0FC0186819781892B11F020E073
:10BBF00030E0C9010895FC01228133818081918167
:10BC0000820F931F0895FC0180819181089581E046
:10BC100090E020913A1330913B13232B11F480E0F4
:10BC200090E0089580913A1390913B13892B29F06D
:10BC30008091381390913913089580E090E0089531
:10BC4000CF93DF93EC01E0913A13F0913B138E1701
:10BC50009F0769F48C819D8190933B1380933A13E5
:10BC60000DC0848195818C179D0721F0FC013097D0
:10BC7000C1F706C08C819D81958384830E94E85C16
:10BC80001D821C821F821E82DF91CF910895EF9248
:10BC9000FF920F931F93CF93DF938C017A01FC01E6
:10BCA00080819181009741F08B34910501F1F80179
:10BCB0001182108283E048C08DE393E10E94335CDF
:10BCC000EC01209751F06C817D81CE0102960E949B
:10BCD000C95D0990D881C02DF4CF81E080933C13D9
:10BCE0008BE490E0F8019183808381E02DC0683877
:10BCF000E1F78DE393E10E94335CEC01209781F33F
:10BD0000CE010296E816F906D9F4BE018DE393E15F
:10BD10000E94785CE0908812F09089128A859B8559
:10BD20009093891280938812EC85FD85309719F0E5
:10BD30008E859F850995F0928912E0928812D0CF66
:10BD40000990D881C02DDACFDF91CF911F910F914B
:10BD5000FF90EF90089510923C138DE393E10E94C1
:10BD60002F5C60E070E08AE992E00C94725B0F93C4
:10BD70001F93CF93DF93EC010091881210918912E9
:10BD80001B870A875D874C873F872E8780913C13EE
:10BD9000882379F08AE992E090938912809388123F
:10BDA000CE0102960E94C95D1093891200938812F9
:10BDB00002C07D836C83BE018DE393E10E94785CB9
:10BDC000BE018DE393E1DF91CF911F910F910C9410
:10BDD000975C0F931F93CF93DF93EC0180913C13FB
:10BDE000882391F000918812109189128AE992E0DB
:10BDF0009093891280938812CE0102960E94D35D9F
:10BE00001093891200938812BE018DE393E10E9482
:10BE1000785CBE018DE393E1DF91CF911F910F918B
:10BE20000C94975C0F931F93CF93DF93EC01809159
:10BE30003C13882391F000918812109189128AE9AD
:10BE400092E09093891280938812CE0102960E940C
:10BE5000DD5D1093891200938812BE018DE393E19A
:10BE60000E94785CBE018DE393E1DF91CF911F9139
:10BE70000F910C94975CCF93DF93EC0180913C136E
:10BE8000882329F0CE0102960E94205E04C01F8202
:10BE90001E8219861886BE018DE393E1DF91CF9152
:10BEA0000C94785CCF93DF9320913C13222329F0EC
:10BEB0000296DF91CF910C94F05DEC018DE393E15C
:10BEC0000E94335C009739F08C179D0739F0FC0114
:10BED00080819181F7CF81E090E002C080E090E026
:10BEE000DF91CF9108952F923F924F925F926F9280
:10BEF0007F928F929F92AF92BF92CF92DF92EF92FA
:10BF0000FF920F931F93CF93DF93CDB7DEB7E897E0
:10BF10000FB6F894DEBF0FBECDBFE2E9F6E3A6EDA3
:10BF2000B6E32C9111963C91119712964C91129771
:10BF300013965C91A2EDB6E35C9011964C9011972C
:10BF400012963C90129713962C9094AC8090CF361A
:10BF50007090D0366090D13680AD898391AD9A8350
:10BF600082AD8B8393AD9C8384A98D8395A99E8399
:10BF700086A98F8397A9988780A9898791A99A878D
:10BF800082A98B8793A99C8784A58D8795A59E8779
:10BF900086A58F8797A5988B80A5898B91A59A8B6D
:10BFA00082A58B8B93A59C8B84A18D8B95A19E8B59
:10BFB00086A18F8B97A1988F80A1898F91A19A8F4D
:10BFC00082A18B8F93A19C8F848D8D8F958D9E8F59
:10BFD000868D8F8F978D98A3808D89A3918D9AA33D
:10BFE000828D8BA3938D9CA384898DA395899EA319
:10BFF00086898FA3978998A7808989A791899AA70D
:10C0000082898BA793899CA784858DA795859EA7F8
:10C0100086858FA7978598AB808589AB91859AABEC
:10C02000B284A384F480E580D680C78080818FAB02
:10C03000918198AF128103812BAB3CAB4DAB5EABD2
:10C040000E94326C5EA95F934DA94F933CA93F9328
:10C050002BA92F932F923F924F925F926F927F92D4
:10C060008F929F922C812F932B812F932A812F9334
:10C0700029812F9328852F932F812F932E812F9302
:10C080002D812F932C852F932B852F932A852F93EA
:10C0900029852F9328892F932F852F932E852F93D2
:10C0A0002D852F932C892F932B892F932A892F93BA
:10C0B00029892F93288D2F932F892F932E892F93A2
:10C0C0002D892F932C8D2F932B8D2F932A8D2F938A
:10C0D000298D2F9328A12F932F8D2F932E8D2F9362
:10C0E0002D8D2F932CA12F932BA12F932AA12F932A
:10C0F00029A12F9328A52F932FA12F932EA12F9302
:10C100002DA12F932CA52F932BA52F932AA52F93E9
:10C1100029A52F9328A92F932FA52F932EA52F93D1
:10C120002DA52F93AF92BF922AA92F9329A92F93C0
:10C13000CF92DF92EF92FF920F931F9328AD2F9330
:10C140002FA92F939F938F937F936F938091A43404
:10C150001F928F93E3EAF4E380811F928F938DE126
:10C1600091E19F938F930E94499AEAEDF6E324A50B
:10C1700035A546A557A550A441A432A423A4848D77
:10C180008983858C768C678C908D9A83818D8B8347
:10C19000928D9C83838D8D8394899E8385898F83E3
:10C1A000968998878789898790899A8781898B87DB
:10C1B00092899C8783898D8794859E8785858F87C3
:10C1C0009685988B8785898B90859A8B81858B8BBB
:10C1D00092859C8B9384D480C580B680A780108183
:10C1E0000181F280E3800FB6F894DEBF0FBECDBFB1
:10C1F0002BAB3CAB4DAB5EAB0E94326C5EA95F9348
:10C200004DA94F933CA93F932BA92F932F923F9277
:10C210004F925F926F927F928F9229812F932D81FF
:10C220002F932C812F932B812F932A812F93298554
:10C230002F9328852F932F812F932E812F932D8538
:10C240002F932C852F932B852F932A852F93298924
:10C250002F9328892F932F852F932E852F939F928D
:10C260002C892F932B892F932A892F93AF92BF92DA
:10C27000CF92DF92EF92FF920F931F939F938F9332
:10C280007F936F938091A4341F928F93E3EAF4E33A
:10C2900080811F928F938EEA90E19F938F930E94EB
:10C2A000499A0FB6F894DEBF0FBECDBFE8960FB621
:10C2B000F894DEBF0FBECDBFDF91CF911F910F91DC
:10C2C000FF90EF90DF90CF90BF90AF909F908F90B6
:10C2D0007F906F905F904F903F902F90089580E3F4
:10C2E0008093F3130895CF93DF936091F31370E07D
:10C2F000C0E3D0E0C61BD70B6F5B7C4EAE010E9443
:10C300007A99CE01DF91CF910895CF92DF92EF928B
:10C31000FF920F931F93CF93DF93C090F613D090AB
:10C32000F7136091F31370E0E601E096C61BD70B9C
:10C33000C138D105E0F47C0100E310E0061B170BC7
:10C340006F5B7C4EA8010E947A9960913F137091B7
:10C3500040138091F4139091F513680F791FA60193
:10C36000C701800F911F0E947A99CE0102C080E020
:10C3700090E0DF91CF911F910F91FF90EF90DF90B0
:10C38000CF9008959091F313890F8093F31308953C
:10C390002091F6133091F7132817390798F0409140
:10C3A000F4135091F513480F591F5093F513409310
:10C3B000F413281B390B3093F7132093F61381E005
:10C3C00090E0089580E090E008959093F7138093B3
:10C3D000F61308958091F4139091F5138F589C4EA5
:10C3E00008958091F31390E08F5B9C4E089581E057
:10C3F00090E020913F13309140132157334111F4C5
:10C4000080E090E008950E94F761892B61F06091CF
:10C410003F13709140134091F6135091F71381E749
:10C4200093E10C947A992091F4133091F51321152E
:10C430003105B9F08091F6139091F713C096E1E7BA
:10C44000F3E1AF01415453414817590734F4DF0178
:10C45000A20FB31F4C914193F4CF1092F513109299
:10C46000F413089580913F139091401308958091A3
:10C47000F6139091F71308959091F31380E3891BBD
:10C4800008958091F31390E3981B2091F613309157
:10C49000F713A901490F511DCA0108950F931F9366
:10C4A000CF938C01C091F3138C2F90E080179107EC
:10C4B0006CF00E944162800F911F8138910530F429
:10C4C000C01BC093F31381E090E002C080E090E0D5
:10C4D000CF911F910F910895CF93DF93EDEAF4E38D
:10C4E0001192119284E3ED3DF807D1F7C5EAD4E348
:10C4F0006CE073E0CE010E941859229684E3CD3A95
:10C50000D807B1F7DF91CF9108951092F5131092EB
:10C51000F4131092F7131092F61380E38093F31341
:10C5200081E793E19093401380933F130C946C62E6
:10C53000EF92FF920F931F93CF93DF9300D0CDB76D
:10C54000DEB78C0169837A830E9485626981E62E59
:10C550007A81F72E81E8E816F10418F080E8E82ED9
:10C56000F12CA701B80180913F13909140130E94D4
:10C570007A99F092F713E092F613C7010F900F909B
:10C58000DF91CF911F910F91FF90EF9008950F933E
:10C590001F93CF93DF938C01EB010E948562109370
:10C5A000401300933F13D093F713C093F613DF911A
:10C5B000CF911F910F910895DC0190E3EDEAF4E330
:10C5C00001900D929A95E1F788E0E5EAF4E3DB014A
:10C5D00001900D928A95E1F70895FC0190E3ADEA90
:10C5E000B4E301900D929A95E1F788E0FB01A5EA8A
:10C5F000B4E301900D928A95E1F70895E82FF0E0F9
:10C60000EE0FFF1FE355FB4C7183608381E090E0E8
:10C610000895E82FF0E0EE0FFF1FE355FB4C8081FB
:10C620009181089590E0880F991F8B589B4C0E9430
:10C63000185981E090E0089590E0880F991F8B5879
:10C640009B4C08958115910511F00197F1F708951C
:10C65000E091E034F091E13490818091DF348923DE
:10C660000895E091DD34F091DE3490818091DF34E3
:10C67000892B8083E091E234F091E33490818091C2
:10C68000DF34892B80830895E091DD34F091DE342E
:10C6900090818091DF34809589238083E091E2341A
:10C6A000F091E33490818091DF34809589238083F9
:10C6B00008951F93CF93DF93E091DD34F091DE3442
:10C6C00090818091DF34809589238083E091E234EA
:10C6D000F091E33490818091DF34892B80838FEB5C
:10C6E00093E00E9422631FB7F894E091E234F09146
:10C6F000E33490818091DF3480958923808383E8BF
:10C7000090E00E942263E091E034F091E134D08126
:10C71000C091DF341FBF78948BE393E00E942263C3
:10C72000E091E034F091E13480819091DF349823FE
:10C7300019F08D2F8C2301C081E0DF91CF911F91E3
:10C7400008955093E3344093E2347093DE34609361
:10C75000DD349093E1348093E03481E001C0880FB0
:10C760002A95EAF78093DF340C945963CF93DF93D3
:10C77000C82FDFB7F894E091E234F091E334908170
:10C780008091DF34892B808383E090E00E942263D4
:10C79000CC2351F0E091E234F091E3349081809128
:10C7A000DF3480958923808387E190E00E942263B3
:10C7B000E091E034F091E13490818091DF3489237D
:10C7C00009F4C0E089E590E00E942263E091E23440
:10C7D000F091E33490818091DF34809589238083C8
:10C7E000DFBF8BE390E00E9422638C2FDF91CF911B
:10C7F0000895CF93DF93C82FD8E08C2F81700E94CB
:10C80000B663C6958111C068D150B9F78C2FDF91FE
:10C81000CF9108958FEF0C94F963DF92EF92FF921E
:10C820000F931F93CF93DF93E82E8B010E945963E0
:10C83000811135C080EF0E94F963D0E0C0E488EF39
:10C84000D82EDC0E81E00E94B663F82E81E00E94B3
:10C85000B663882319F0FF2071F023C0F1100BC0DC
:10C86000CE1530F0F801808180FF05C0EC1619F07C
:10C87000DC2FFF24F3948F2D0E94B663F801908182
:10C880009695FF2011F09068F8019083C150CD116A
:10C89000D9CF0F5F1F4FC111D2CF8D2F03C08FEFA4
:10C8A00001C08EEFDF91CF911F910F91FF90EF901C
:10C8B000DF900895EF92FF921F93CF93DF93182F8D
:10C8C000EB010E945963209771F085E50E94F9639E
:10C8D0007E0188E0E80EF11C89910E94F963CE1573
:10C8E000DF05D1F703C08CEC0E94F963812FDF9143
:10C8F000CF911F91FF90EF900C94F9630F931F93CA
:10C90000CF93DF93DB01EC9111969C911197F0E0AE
:10C91000F92B803179F4EE7F63E0EE0FFF1F6A950B
:10C92000E1F716969C9116976CE070E0691B71090F
:10C93000E60FF71FF7FF07C091E0EA019883F19532
:10C94000E195F10902C0EA011882883279F414965F
:10C950008C91982F9076903649F086FF02C0EE7F3A
:10C9600005C085FF02C0EC7F01C0E87FCF0144E035
:10C97000969587954A95E1F7D9018C93EF70E80178
:10C98000E88380E0DF91CF911F910F9108950F937D
:10C990001F93CF93DF93EC018B01B80188810E9434
:10C9A0000D6488839FEF980F9D3F30F4F8019081CC
:10C9B000983211F0903189F7DF91CF911F910F914B
:10C9C0000895CF93DF93EC010E945963BE0184EB7D
:10C9D0000E945A6481E00E94B663C82F0E94596386
:10C9E00081E0C11101C080E0DF91CF9108951F93D4
:10C9F000CF93DF9300D0CDB7DEB7182F69837A834A
:10CA00000E9459630E94286369817A81882341F0DA
:10CA100084E40E945A64113029F00E94316302C0FC
:10CA200082E001C080E00F900F90DF91CF911F91C5
:10CA300008955F926F927F928F929F92AF92BF9272
:10CA4000CF92DF92EF92FF920F931F93CF93DF93DA
:10CA5000CDB7DEB729970FB6F894DEBF0FBECDBFB6
:10CA60005C014B013A0189010E945963B5018EEBCB
:10CA70000E945A64CE0101967C016C0199E0592E06
:10CA80005E0C0E940A64F60181936F015E12F9CF79
:10CA900069E070E0C7010E94EF7ED82E811108C0C6
:10CAA0009301A401B701F50180810E947E6402C058
:10CAB00083E0D82E8D2D29960FB6F894DEBF0FBED9
:10CAC000CDBFDF91CF911F910F91FF90EF90DF903D
:10CAD000CF90BF90AF909F908F907F906F905F901E
:10CAE00008956F927F928F929F92AF92BF92CF9252
:10CAF000DF92EF92FF920F931F93CF93DF93CDB707
:10CB0000DEB729970FB6F894DEBF0FBECDBF782EE3
:10CB10005B014A01890160E070E08EEB0E945A647B
:10CB2000CE0101967C016C0199E0692E6E0C0E9489
:10CB30000A64F60181936F016E12F9CF69E070E02B
:10CB4000C7010E94EF7ED82E811107C09401A50174
:10CB5000B701872D0E947E6402C083E0D82E8D2D00
:10CB600029960FB6F894DEBF0FBECDBFDF91CF91EF
:10CB70001F910F91FF90EF90DF90CF90BF90AF90FB
:10CB80009F908F907F906F9008950F931F93CF93F6
:10CB9000DF93CDB7DEB728970FB6F894DEBF0FBE90
:10CBA000CDBF182F062F98E0E8E1F3E0DE011196E3
:10CBB00001900D929A95E1F7242F440F330B41E732
:10CBC00052E0249FC001259F900D349F900D1124A9
:10CBD00064E670E00E94479384E6089F600D711D33
:10CBE0001124FE01319688E08E0F419150E0241708
:10CBF000350719F46F5F7F4F02C08E13F6CF1123F4
:10CC000019F0719561957109CB0128960FB6F894CA
:10CC1000DEBF0FBECDBFDF91CF911F910F91089561
:10CC20000F931F93CF93DF93CDB7DEB72B970FB63C
:10CC3000F894DEBF0FBECDBF182F092F682F792FB4
:10CC400088E0810F0E94F764882319F084E391E261
:10CC500043C066E471E48FE090E00E9477669E0135
:10CC6000275F3F4FAE01465F5F4FBE01655F7F4F5D
:10CC7000812F902F0E9419658111E8CF88E0E8E1AB
:10CC8000F3E0DE01119601900D928A95E1F7298576
:10CC900041E752E0249FC001259F900D112464E6D6
:10CCA00070E00E9447938A8594E6899F600D711D0C
:10CCB0001124FE01319688E08E0F9191291303C053
:10CCC0006F5F7F4F02C08E13F8CF8B85882319F0DA
:10CCD000719561957109CB012B960FB6F894DEBF63
:10CCE0000FBECDBFDF91CF911F910F910895DC0151
:10CCF000CB0181159105A105B10529F08150904026
:10CD0000A040B040D9F708959B01AC011092B90042
:10CD100060E072E18AE790E00E945B93DA01C9016A
:10CD20004097A109B109B695A795979587958093E6
:10CD3000B800089594EA9093BC0040EA56E861E098
:10CD400070E09091BC0097FD07C041505109610906
:10CD50007109B9F781E008959091B900987F9830F2
:10CD600011F09031B9F78093BB0084E88093BC0048
:10CD700080EA96E8A1E0B0E02091BC0027FD05C064
:10CD80000197A109B109C1F7E5CF8091B900887F6A
:10CD9000883111F08034F1F680E0089524EA34E817
:10CDA00044E92093BC009091BC0097FFFCCF909188
:10CDB000B900987F983011F0903199F78093BB00BB
:10CDC0003093BC009091BC0097FFFCCF9091B900CC
:10CDD000987F903211F0983539F44093BC009091CF
:10CDE000BC0094FDFCCFDDCF08950C949A6684E9D5
:10CDF0008093BC008091BC0084FDFCCF089580939B
:10CE0000BB0084E88093BC008091BC0087FFFCCF0E
:10CE10009091B900987F81E0983209F480E00895FC
:10CE200084EC8093BC008091BC0087FFFCCF809194
:10CE3000BB00089584E88093BC008091BC0087FF0C
:10CE4000FCCF8091BB000895CF93DF93FC017096D7
:10CE5000EC01A991CE01A0933F01CE17DF07C1F7E6
:10CE600080913C018F7D80933C0180913C01877FC4
:10CE700080933C01DB015096FB01819180933E0140
:10CE8000EA17FB07D1F780913C01806880933C0151
:10CE900080913D0180FFFCCF4051510980913C01C0
:10CEA000806280933C0180913C01877F80933C01AC
:10CEB000141615069CF4FB01819180933E01EA173C
:10CEC000FB07D1F780913C01806880933C01809101
:10CED0003D0180FFFCCF40515109EACFF901C90162
:10CEE000409620913E012193E817F907D1F781E0A0
:10CEF00090E0DF91CF9108950F931F93CF93DF932D
:10CF0000EC018CE70E94CE668CE70E94FF668E01E2
:10CF1000005F1F4F89910E94FF66C017D107D1F7AC
:10CF2000DF91CF911F910F910C94F766813019F426
:10CF300040E050E002C040EC50E060E070E08CE780
:10CF400090E00C948F13813019F44EE050E002C051
:10CF500048E050E060E070E08CE790E00C948F13C4
:10CF600041E050E060E070E08CE790E00E948F13B9
:10CF70006AE67AE080E090E00C94776648E350E05F
:10CF800060E070E08CE790E00E948F1349E350E08E
:10CF900060E070E08CE790E00E948F1344E150E085
:10CFA00060E070E08CE790E00E948F1348E750E06B
:10CFB00060E070E08CE790E00E948F134EE550E057
:10CFC00060E070E08CE790E00E948F134DE650E047
:10CFD00060E070E08CE790E00E948F136CE17AE1F2
:10CFE00086E090E00E9477664CE050E060E070E000
:10CFF0008CE790E00E948F1341E050E060E070E029
:10D000008CE790E00E948F1346E050E060E070E013
:10D010008CE790E00E948F136AE67AE080E090E06F
:10D020000C947766CF93DF93CDB7DEB7A2970FB698
:10D03000F894DEBF0FBECDBF81E1E8EBF9E0DE0181
:10D04000529601900D928A95E1F781E1E9ECF9E0C1
:10D05000DE01119601900D928A95E1F70E94BE675C
:10D06000CE0142960E947C6782E00E9496676AE643
:10D070007AE080E090E00E947766CE0101960E94FF
:10D080007C6760E17EEA88E290E00E94776680E05B
:10D090000E94A36760E17EEA88E290E00E947766E2
:10D0A0004EE050E060E070E08CE790E00E948F136B
:10D0B000A2960FB6F894DEBF0FBECDBFDF91CF9121
:10D0C0000895CF92DF92EF92FF920F931F93CF9329
:10D0D000DF9300D01F92CDB7DEB7042F122F21307F
:10D0E00061F0223031F0243031F0283031F493E017
:10D0F00005C091E003C092E001C090E0E82FF0E0AD
:10D100008160F82E0C3009F4E0C00E3011F4946008
:10D11000DCC0003111F49860D8C0023109F0D5C0EC
:10D12000613009F4B7C09C60623011F4906207C0AE
:10D13000633011F4906403C0643009F49066906821
:10D14000692F70E023E030E0AE014F5F5F4FCF0109
:10D150000E94A61369E07AE180E090E00E94776681
:10D160008F2D0E949A660E94106789830E94106723
:10D170008A83023119F40E9410678B830E94106722
:10D1800087FDF1CF0E941A670E94F76669E07AE195
:10D1900080E090E00E9477668F2D0E949A660E9440
:10D1A000106789830E9410678A83023119F40E94F4
:10D1B0001A678B830E941A670E94F76669812A8129
:10D1C000023139F5862F90E0A0E0B0E04B81DC0120
:10D1D0009927882730E0322F2227820F931FA11D25
:10D1E000B11D61FF09C0840F911DA11DB11DBC01BE
:10D1F000CD018C6F9F6F06C0BC01CD01640F711D06
:10D20000811D911D0E94509020E83FEF4FEF57E4A1
:10D210001FC070E0762F6627620F711D072E000C6D
:10D22000880B990B0E9450900C3029F420E030EECE
:10D230004FEF54E40DC00E3029F420E038EF4FEFEB
:10D2400055E406C0003131F420E03EEF4FEF56E4E4
:10D250000E949C8F2FE632E143E050E40E94489206
:10D260006B017C01612F70E080E090E00E945090A3
:10D270009B01AC01C701B6010E949C8F0F900F90DB
:10D280000F90DF91CF911F910F91FF90EF90DF9062
:10D29000CF9008959C68692F70E023E030E0AE01E4
:10D2A0004F5F5F4FCF010E94A61369E07AE180E0F3
:10D2B00090E00E9477668F2D0E949A660E94106708
:10D2C00089830E9410678A8356CF613009F02CCF82
:10D2D0009068692F70E023E030E0AE014F5F5F4F50
:10D2E000CF010E94A61369E07AE180E090E00E94FD
:10D2F00077668F2D0E949A660E94106789830E942C
:10D3000010678A833BCFE6E4F1E090812081308191
:10D310008081929596959695937022952F70922B79
:10D32000892B232F22952F70822B08950F931F9303
:10D33000CF93DF9300D0CDB7DEB746E06CE080E05E
:10D340000E94C86C89E18093C4001092C50082E0FD
:10D350008093C00080E00E94586D0E94F66B84B7F5
:10D3600084B784B784B784B78AED99E09F938F938D
:10D370008AE692E19F938F930E94499A0E94297BAB
:10D380000E94C85A60E070E080E992E00E94725BFF
:10D390000E94AB5EE0912003F091210309950E9469
:10D3A000836990E00E94657BCE0101960E94246B08
:10D3B0000F900F900F900F90882341F08AE492E134
:10D3C0009F938F930E94499A0F900F90CE010196E0
:10D3D0000E9433590E94326B8C010E942E6BAE0169
:10D3E0004F5F5F4FB8010E942A700E94946A0E94AA
:10D3F0000B700E94366B0E9463718DE392E19F93E4
:10D400008F930E94499A8A811F928F9309E312E1B8
:10D410001F930F930E94499A89811F928F931F93A4
:10D420000F930E94499A87E392E19F938F930E9402
:10D43000499A0E94697BE0915D03F0915E03099532
:10D44000E0914F03F09150030995E0913603F0917C
:10D45000370309950E946A71182F0E9408701F9265
:10D460001F931F928F9380915C038F9380915B0336
:10D470008F9380914E038F9380914D038F938CE116
:10D4800092E19F938F930E94499AE0916703F091F4
:10D4900068030FB6F894DEBF0FBECDBF309791F092
:10D4A0000995BC0180E890E00E9433937F936F93CD
:10D4B00089E092E19F938F930E94499A0F900F9079
:10D4C0000F900F9087E092E19F938F930E94499A6B
:10D4D00060E070E086EE92E00E94725B8AEF92E07C
:10D4E0000E94397A8FEF91E19F938F930E94499A1E
:10D4F0000F900F900F900F900F900F90DF91CF91A2
:10D500001F910F9108957F936F939F938F9389EF4E
:10D5100091E19F938F930E94499A0F900F900F90E3
:10D520000F900F900F900895DF92EF92FF920F935C
:10D530001F93CF93DF93CDB7DEB7A0970FB6F894C4
:10D54000DEBF0FBECDBF83E690E00E94479D182F3F
:10D55000282F35EF380F303108F0982F9095291784
:10D5600009F463C085E892E19F938F930E94499AE2
:10D57000EAECF2E18E010F5F1F4F0F900F90D80180
:10D58000D02EE12EF02E88E0800F94919D9331965D
:10D590008A13FBCFF89448E050E06FE770E0C801D1
:10D5A0000E944D9DECEBF2E1D8018EE08F0D94913D
:10D5B0009D9331968A13FBCF4EE050E061E770E017
:10D5C000C8010E944D9DE2EBF2E12AE02F0D84910B
:10D5D000D8018D938D0131962A13F9CF4AE050E09E
:10D5E00067E670E08D2D9E2D0E944D9D6DEC7BEACF
:10D5F00081E690E00E94659D60E070E08FE590E03C
:10D600000E94659D60E08EE590E00E94579D60E07D
:10D6100070E085E690E00E94659D1AE16AE175EE92
:10D6200083E690E00E94659D7894812FA0960FB6C6
:10D63000F894DEBF0FBECDBFDF91CF911F910F9148
:10D64000FF90EF90DF900895F89442E050E06FE78C
:10D6500070E00E942F9D789480E0089581E690E02C
:10D660000C94479D8FE590E00C94479D8EE590E0EB
:10D670000C943F9D0F931F930091EE341091EF3463
:10D680002091F0343091F134482F50E060E070E0A8
:10D69000DB01CA01800F911FA21FB31F8093EE34DC
:10D6A0009093EF34A093F034B093F1348091EA3446
:10D6B0009091EB34A091EC34B091ED34840F951F30
:10D6C000A61FB71F8093EA349093EB34A093EC34F9
:10D6D000B093ED3480918E368823A1F08091E634AA
:10D6E0009091E734A091E834B091E934480F591F84
:10D6F0006A1F7B1F4093E6345093E7346093E8340D
:10D700007093E9341F910F9108951F920F920FB6F5
:10D710000F9211240BB60F922F933F934F935F9369
:10D720006F937F938F939F93AF93BF93EF93FF93E9
:10D730008091FA139091FB1301969093FB138093C1
:10D74000FA138091F9138F5F8093F9138038A9F44D
:10D750001092F9138091EE349091EF34A091F0344F
:10D76000B091F1340196A11DB11D8093EE349093D8
:10D77000EF34A093F034B093F13480918E36882347
:10D78000E1F08091F8138F5F8093F8138038A9F44B
:10D790001092F8138091E6349091E734A091E83428
:10D7A000B091E9340196A11DB11D8093E6349093A8
:10D7B000E734A093E834B093E9340E94075E892BE4
:10D7C00011F00E941A5DFF91EF91BF91AF919F916F
:10D7D0008F917F916F915F914F913F912F910F901A
:10D7E0000BBE0F900FBE0F901F901895F8941092DB
:10D7F000B60016BC83EF87BD82E084BD94E095BD82
:10D8000095B395BB80936E00789408958091FA1338
:10D810009091FB132091FA133091FB138217930719
:10D82000A9F70895009741F022E330E0000021506D
:10D830003109E1F70197F6CF08950F931F93CF9326
:10D84000DF93EC010E94066C8C010E94066C801B29
:10D85000910B8C179D07C8F3DF91CF911F910F910A
:10D86000089508950F931F936091EE347091EF34F3
:10D870008091F0349091F1340091EE341091EF34B6
:10D880002091F0343091F1346017710782079307CB
:10D8900059F71F910F9108951F920F920FB60F9293
:10D8A00011241092BC020F900FBE0F901F9018957C
:10D8B0001F920F920FB60F9211240BB60F922F9357
:10D8C0003F934F935F936F937F938F939F93AF9308
:10D8D000BF93EF93FF93E091B202F091B302808186
:10D8E000E091BD02F091BE02309709F00995FF91D9
:10D8F000EF91BF91AF919F918F917F916F915F91C8
:10D900004F913F912F910F900BBE0F900FBE0F9034
:10D910001F9018951F920F920FB60F92112410921C
:10D92000C9020F900FBE0F901F9018951F920F9273
:10D930000FB60F9211240BB60F922F933F934F9374
:10D940005F936F937F938F939F93AF93BF93EF9367
:10D95000FF93E091BF02F091C0028081E091CA0282
:10D96000F091CB02309709F00995FF91EF91BF91AB
:10D97000AF919F918F917F916F915F914F913F9167
:10D980002F910F900BBE0F900FBE0F901F90189508
:10D990002DE0829FC0011124FC01EE54FD4FA281B5
:10D9A000B3811C92A481B5816C93A681B78188ED67
:10D9B0008C93A085B1854C931286148613860895A6
:10D9C0002DE0829FC0011124FC01EE54FD4F81E047
:10D9D0008287A081B1816C933A9680818111FDCFBD
:10D9E00008951F93CF93DF93182FEB01FE019491BD
:10D9F000992339F0FE016491812F0E94E06C2196F9
:10DA0000F5CFDF91CF911F9108951F93CF93DF93AF
:10DA1000182FEB019881992369F09A3021F46DE079
:10DA2000812F0E94E06C69916D30A1F3812F0E94DB
:10DA3000E06CF0CFDF91CF911F910895CF93DF93EA
:10DA4000CDB7DEB79E01285F3F4F4E815F8160E416
:10DA500070E08CEF93E10E940E9B6CEF73E18D817F
:10DA60000E94056DDF91CF910895CF93C82F8A3022
:10DA700031F46DE080913C140E94E06C02C08D3066
:10DA800029F06C2F80913C140E94E06C80E090E0C3
:10DA9000CF9108952DE0829FC0011124FC01EE5426
:10DAA000FD4F748763870895682F80E00C94E06CC5
:10DAB00080933C1484EA92E090935B3D80935A3DBE
:10DAC000089584B7877F84BF0FB6F894A895809196
:10DAD0006000886180936000109260000FBE08951E
:10DAE0009FE088E10FB6F894A895809360000FBE80
:10DAF000909360000895A89508950FB6F894A8959E
:10DB000080916000886180936000109260000FBE79
:10DB10000895F89498E088E10FB6F894A89580935A
:10DB200060000FBE90936000FFCF8091F934809128
:10DB3000F93490E0089540E06FE181E491E00C94C5
:10DB4000FE72E9E3F1E0808180818D7F80838DE04A
:10DB500090E00197F1F723E040E06FE182E491E08B
:10DB60000E94097383E090E00197F1F70895909186
:10DB7000390191FD0AC0282F803108F02FE040E0E4
:10DB80006FE085E491E00C94097308958091390168
:10DB900081FD0EC040E06FE181E491E00E94FE72E1
:10DBA000282F2F7E81E090E0213021F080E0089541
:10DBB00080E090E008958091390181FF02C081E00A
:10DBC000089540E06FE181E491E00E94FE728F31A0
:10DBD00021F08F7E8150823090F780E008950E947E
:10DBE000DB6D8823E1F30895CF93DF93C82F0E9464
:10DBF000EF6D0E949B6DD82FC81771F1C83019F4D2
:10DC00000E94A16D25C0C93121F4863189F429E033
:10DC100005C0C63169F4893159F426E040E06FE16E
:10DC200082E491E00E94097383E090E00197F1F7AC
:10DC30002C2F40E06FE182E491E00E940973D8301C
:10DC400019F489E691E002C083E090E00197F1F7D2
:10DC50000E949B6D8C1303C080E490E002C083E4BB
:10DC600090E0DF91CF9108950E94EF6D10928E3673
:10DC70000E94A16D80913901826080933901809169
:10DC800011378823D9F180919400909195004091AB
:10DC900022375091233784179507A0F48091EE36F0
:10DCA0009091EF36A091F036B091F1368C57914EAD
:10DCB000AF4FBF4F8093EE369093EF36A093F03680
:10DCC000B093F1362091940030919500241B350BD0
:10DCD0008091EE369091EF36A091F036B091F1360A
:10DCE000820F931FA11DB11D8093EE369093EF36E6
:10DCF000A093F036B093F13610921137809113371C
:10DD00008823D9F180919400909195004091263715
:10DD10005091273784179507A0F48091F63690919B
:10DD2000F736A091F836B091F9368C57914EAF4F37
:10DD3000BF4F8093F6369093F736A093F836B093A2
:10DD4000F9362091940030919500241B350B809179
:10DD5000F6369091F736A091F836B091F936820FE9
:10DD6000931FA11DB11D8093F6369093F736A093B3
:10DD7000F836B093F93610921337089580918E36A5
:10DD8000882381F08091C014882331F081E0809352
:10DD9000BE1481E090E008950E94DB6D8823B1F30A
:10DDA0000E94346E80E090E00895809194009091FC
:10DDB0009500909327378093263781E0809313371F
:10DDC0009091390191FD08C08091390181FD1AC0FF
:10DDD00086E10E94F46D16C080938D3620919400E8
:10DDE0003091950030932337209322378093113759
:10DDF000809139018D7F8093390180918D36811119
:10DE0000FCCFE2CF81E080938E36089580918E36EC
:10DE100081110AC08091C014882321F081E0809391
:10DE2000BF1402C00E94D56E81E090E008951F9358
:10DE3000CF93DF931F92CDB7DEB78FB789838091E1
:10DE4000C01481111FC0F89480918E36882351F040
:10DE50008091390181FD14C00E94DB6D882381F01F
:10DE600080E003C00E94066F81E0909147019E30E0
:10DE700088F4882351F01FEF0E94BE6E107429F4BD
:10DE800089818FBF80E090E009C089818FBF81E0E8
:10DE900090E004C08823A1F310E0EECF0F90DF9153
:10DEA000CF911F9108958091BF14882321F00E9483
:10DEB000D56E1092BF148091BE14882321F00E9469
:10DEC000346E1092BE141092C01408950F931F93D5
:10DED000AB0121E02093C0140091D2361091D336CB
:10DEE0002091D4363091D5360F5F1F4F2F4F3F4FC3
:10DEF0000093D2361093D3362093D4363093D53650
:10DF000022E0260F27FF0CC080918B3690918C3633
:10DF1000019690938C3680938B360FEF1FEF07C0DE
:10DF2000BC018DE394E10E947A9900E010E00E9428
:10DF3000536FC8011F910F9108958093C2140895E3
:10DF40000E949B6D823021F0823111F081E00895B2
:10DF500080E0089508958FEF80934E0122E044E021
:10DF600060EF8CE691E00E94097325E041E06EE0ED
:10DF70008CE290E00E94097380E880936F018091A9
:10DF8000460180936D0121E045E060E284E491E088
:10DF90000C940973CF93DF93CDEFD3E0CE010197BB
:10DFA000F1F70E94F47210920235109284351092AB
:10DFB00006361092013510920035E9E3F1E08081D8
:10DFC0008E7F808380818D7F80838DE090E00197BC
:10DFD000F1F780818160808323E040E06FE182E49B
:10DFE00091E00E9409732197F1F780915D01809182
:10DFF0005E010E94AB6F60E070E08CEC92E00E94EA
:10E00000725B0E94D56E81E090E0DF91CF91089520
:10E010008091C1140895CF93DF931F92CDB7DEB7DF
:10E0200089830E94EF6D89818093C114282F40E07D
:10E030006FE188E491E00F90DF91CF910C94097328
:10E040000E940B708091390181FD03C086E00C9421
:10E05000F46D0895FA0180936201909363016093D7
:10E060006001709361013097C1F0808180936B01F2
:10E07000818180936A018281809369018381809389
:10E080006801848180936701858180936601868120
:10E090008093650187818093640108958CEC92E000
:10E0A0000E94935B81E08093F9348091FA349091DF
:10E0B000FB3401969093FB348093FA3481E090E036
:10E0C00008958091013592E8899FF0011124EE5F57
:10E0D000FA4C10828F5F833018F48093013502C0B0
:10E0E00010920135E091013582E8E89FF00111249A
:10E0F000EE5FFA4C808181110C944E701092F934CD
:10E1000008951F93CF93DF932091013512E8129F5A
:10E1100090011124F901EE5FFA4C4081411103C0D6
:10E120000E94617092C05091390151FD8EC0509192
:10E130008E36552309F489C047FF16C00E946170CE
:10E140008091C2369091C336A091C436B091C53645
:10E150000196A11DB11D8093C2369093C336A09342
:10E16000C436B093C53671C04330B0F40E946170BC
:10E170008091BE369091BF36A091C036B091C13625
:10E180000196A11DB11D8093BE369093BF36A0931A
:10E19000C036B093C13659C050E0EA0122976C17DF
:10E1A0007D07B0F40E9461708091BA369091BB36C1
:10E1B000A091BC36B091BD360196A11DB11D8093D2
:10E1C000BA369093BB36A093BC36B093BD363DC0F3
:10E1D000B9016D5F7A4C0E947A99E09101351E9FDA
:10E1E000F0011124EE57FA4C80818093F2340E94A2
:10E1F0006170809147018093F3349091F8349923B2
:10E2000011F0891710F48093F8346091F33470E0C2
:10E2100084E00E94FE626091F23470E083E00E942C
:10E22000FE628091D6369091D736A091D836B091C3
:10E23000D9360196A11DB11D8093D6369093D7365D
:10E24000A093D836B093D93602C0C0E0D0E0CE015A
:10E25000DF91CF911F910895CF93DF93EC018881D7
:10E2600099810097E9F08730954021F01982188252
:10E2700083E026C06238C1F41092F9340E948562AE
:10E280000E94EA6160E870E00E9481701816190629
:10E290006CF40E94E561E0916103F09162030995DD
:10E2A00087E095E09983888381E00AC08091F63405
:10E2B0009091F73401969093F7348093F634F0CF31
:10E2C000DF91CF91089591E09093C0140E94B76DB3
:10E2D0000C94536F8091390181FD06C040E06FE0DE
:10E2E00085E491E00C94FE7280E108950F931F93F2
:10E2F000CF93DF93C82F81E08093C014D0918E36E6
:10E300009091390191FF16C02091940030919500B1
:10E3100030932337209322378093113780938D36A3
:10E32000809139018D7F8093390180918D368111E3
:10E33000FCCFD0E00E94EF6D80918E36882309F4E7
:10E340003FC0809113378823D9F180919400909138
:10E350009500409126375091273784179507A0F4F0
:10E360008091F6369091F736A091F836B091F93653
:10E370008C57914EAF4FBF4F8093F6369093F73640
:10E38000A093F836B093F93620919400309195001F
:10E39000241B350B8091F6369091F736A091F83614
:10E3A000B091F936820F931FA11DB11D8093F636EF
:10E3B0009093F736A093F836B093F936109213374E
:10E3C0008091390181FD03C089E10E94F46D86E0EE
:10E3D0000E940963892B51F00E946A71082F86E020
:10E3E0000E94096381500E94B76D02C000E010E0F6
:10E3F00080919400909195009093253780932437D5
:10E4000081E080931237F894809139018260809383
:10E410003901809139018D7F8093390162E06C0F61
:10E420008DE394E10E9439737894809188369091BD
:10E430008936019690938936809388360E94EF6DD5
:10E4400045E060EE82E491E00E94FE72C82F86E013
:10E450000E940963892B19F0802F0E94B76DDD237C
:10E4600019F00E94D56E02C00E94346E809112375E
:10E470008823D9F1809194009091950040912437A0
:10E480005091253784179507A0F48091F23690912A
:10E49000F336A091F436B091F5368C57914EAF4FCC
:10E4A000BF4F8093F2369093F336A093F436B09337
:10E4B000F5362091940030919500241B350B809106
:10E4C000F2369091F336A091F436B091F536820F82
:10E4D000931FA11DB11D8093F2369093F336A09344
:10E4E000F436B093F5361092123780918E36882329
:10E4F00061F08091940090919500909327378093DC
:10E50000263781E08093133707C023E040E06FE1B6
:10E5100082E491E00E9409730E94536FC130E9F0D8
:10E52000C330A9F48091CA369091CB36A091CC36F5
:10E53000B091CD360196A11DB11D8093CA3690933E
:10E54000CB36A093CC36B093CD36C2E009C0C530EF
:10E5500031F0C73029F4C1E003C0C0E001C0C3E01E
:10E560008C2F90E0DF91CF911F910F910895CF9361
:10E57000DF93EB010E94666F009729F4CE010E94A1
:10E580007671009751F020918B3630918C362F5F49
:10E590003F4F30938C3620938B36DF91CF91089587
:10E5A000CF93DF9380918E36811104C00E94066F55
:10E5B000D1E001C0D0E00E949B6D863111F0813125
:10E5C00019F4C091470109C040E06FE186E491E091
:10E5D0000E94FE72C82FCC0FC80FD1110E94BE6ED0
:10E5E0008C2FDF91CF9108951092C4141092C31410
:10E5F000EFE6F0E08081806280830895FC018081F5
:10E600006823862F90E002C0959587954A95E2F79A
:10E610000895FC01922FF8942081362F3095522FC7
:10E620005323292F01C0220F4A95EAF72623252BD1
:10E63000208378940895CF93DF93E0917B01EC01E0
:10E64000E993A0E8B1E020E82E0F3C9139931196B0
:10E650002A13FBCFE150F0E0E058FE4F2181FC018E
:10E66000E058FF4F2083319681E08083DF91CF9186
:10E67000089560938001E1E8F1E06158DC012D919B
:10E68000CD01208331966E13F9CF08951F920F921A
:10E690000FB60F9211240BB60F922F933F934F9307
:10E6A0005F936F937F938F939F93AF93BF93EF93FA
:10E6B000FF93809147018093F3348091003522E8E5
:10E6C000829FC00111248E5F9A4C0E941B7380911F
:10E6D00000358F5F833018F48093003502C01092AC
:10E6E00000350E944E70FF91EF91BF91AF919F91C5
:10E6F0008F917F916F915F914F913F912F910F90EB
:10E700000BBE0F900FBE0F901F9018951F920F9287
:10E710000FB60F9211240F900FBE0F901F901895F7
:10E720001F920F920FB60F9211240F900FBE0F90F1
:10E730001F9018951F920F920FB60F9211240F90F1
:10E740000FBE0F901F9018951F920F920FB60F9249
:10E75000112410928D360F900FBE0F901F901895B8
:10E760001F920F920FB60F92112410928D360F90B8
:10E770000FBE0F901F9018951F920F920FB60F9219
:10E7800011248F9381E08093F9348F910F900FBE05
:10E790000F901F9018951F920F920FB60F92112491
:10E7A00010928D360F900FBE0F901F9018951F92EC
:10E7B0000F920FB60F9211248F939F938091C314E1
:10E7C0009091C41401969093C4148093C3149F91A4
:10E7D0008F910F900FBE0F901F901895CF92DF92E0
:10E7E000EF92FF920F931F93CF93DF937C018B01E6
:10E7F0006A0185EC94E10E94335CEC01892B51F0B5
:10E80000EC81FD81309711F0C8010995CE010E947D
:10E81000DF5CF3CFA601B801C701DF91CF911F9153
:10E820000F91FF90EF90DF90CF900C94B8590F9319
:10E830001F93CF93DF9300D0CDB7DEB7809196368C
:10E8400090919736A0919836B09199360196A11D76
:10E85000B11D8093963690939736A0939836B093D7
:10E8600099360E947E768C0185EC94E10E94335C9F
:10E87000009779F0DC011296ED91FC911397309797
:10E8800029F089839A8309959A8189810E94DF5CA6
:10E89000EFCF0115110549F0C8010F900F90DF91DE
:10E8A000CF911F910F910C94AF590F900F90DF9162
:10E8B000CF911F910F9108950E94697B0E948562FC
:10E8C0000E94A8748DE493E09093913680939036E3
:10E8D0000E947C762FEF31E040E05EE160E074E082
:10E8E00082E090E00C944976BC0185EC94E10C94B4
:10E8F000975CBC0185EC94E10C94785CCF93DF933A
:10E90000EC0140919236509193366091943670911B
:10E9100095364F5F5F4F6F4F7F4F409392365093C6
:10E92000933660939436709395360E949176009753
:10E9300061F00E940362E0915103F0915203BE0125
:10E940008EEE93E7099581E090E0DF91CF910895F5
:10E950008BEC94E10C942F5C0F93CF93DF93EC013D
:10E960007B836A8318865F834E83BC018BEC94E1C2
:10E970000E94975CE091C714F091C814309749F059
:10E980004C815D8101E020E030E068858A819B81D7
:10E990000995DF91CF910F910895BC018BEC94E123
:10E9A0000C94785C0F93FC011086E091C714F091F1
:10E9B000C814309761F0DC0100E020E030E040E076
:10E9C00050E060E012968D919C91139709950F91FC
:10E9D00008950F93DC0114962D913C91159781E0D9
:10E9E00018968C93189715967C936E931497E091D4
:10E9F000C714F091C814309741F0AB0100E061E01A
:10EA000012968D919C91139709950F9108950F93EC
:10EA1000E091C714F091C814309779F0DC01149696
:10EA20004D915C91159701E09A0118966C91189799
:10EA300012968D919C91139709950F910895E091ED
:10EA4000C914F091CA14309709F00994089590936D
:10EA5000CA148093C91408959093C8148093C7145E
:10EA600008958BEC94E10C94335CEF92FF920F933A
:10EA70001F93CF93DF938C01EB017A018BEC94E130
:10EA80000E94335C0097D9F0DC0112962D913C91E5
:10EA900013972C173D0781F41696ED91FC9117976B
:10EAA000309769F09701AE01B801DF91CF911F91C6
:10EAB0000F91FF90EF9009940E94DF5CE3CFDF910C
:10EAC000CF911F910F91FF90EF9008950895CF93EC
:10EAD000DF93CDECD4E169A97AA920E030E046E8E3
:10EAE00055E788EE94E10E94B75E0E94677B69A9B2
:10EAF0007AA90E94339320E030E04AE955E7BC014F
:10EB000088ED94E1DF91CF910C94B75E8091FE1473
:10EB10009091FF142091FC143091FD14880F991FDF
:10EB20002817390708F4C9019093FF148093FE1445
:10EB30000C946775CF93DF930E9485620E94EA610F
:10EB4000EC01198218820E94317528813981009761
:10EB500019F1FC0140854423F9F0FC014281538105
:10EB6000F901EE0FFF1FEE0FFF1FEC0FFD1F538388
:10EB70004283FC01448155812F5F3F4FF901EE0F25
:10EB8000FF1FEE0FFF1FEC0FFD1F518340833983E2
:10EB900028830E94DF5CD9CFC901880F991F880F95
:10EBA000991F02960E94E56188819981892B31F035
:10EBB0008DEC94E1DF91CF910C948559DF91CF9149
:10EBC0000895AF92BF92CF92DF92EF92FF920F9390
:10EBD0001F93CF93DF9300D0CDB7DEB76B010E94B8
:10EBE000EA61FC01E080F180FA82E982FCE0EF1644
:10EBF000F10418F400E010E00DC0FF92EF9288EFEE
:10EC000099E09F938F930E94359A0F900F900F90E9
:10EC10000F9022C00E151F05F9F00E94EA619801BD
:10EC2000220F331F220F331F820F931FFC01A2807C
:10EC3000B3800E94EA610F5F1F4F9801220F331FBC
:10EC4000220F331F820F931FFC0140815181B501B8
:10EC5000C6010E943575DECF0F900F90DF91CF91E6
:10EC60001F910F91FF90EF90DF90CF90BF90AF90EA
:10EC700008950F93013059F48091F8149091F9148C
:10EC80009093FF148093FE140F910C9467750F916D
:10EC90000895EF92FF920F931F93CF93DF937B0121
:10ECA0008A01E9014AE353E0BC018DEC94E10E9442
:10ECB0006859EDECF4E1F4A6E3A616A705A7D0ABDE
:10ECC000C7A789E396E7DF91CF911F910F91FF903E
:10ECD000EF900C942C7588EE94E10E943B5F88EDD8
:10ECE00094E10E943B5F8DEC94E10C9483598091F8
:10ECF000FE149091FF1408950C94C459CF93DF93A0
:10ED0000E0913E03F0913F030995EC01892B29F036
:10ED10006A817B8181E00E94FE62CE01DF91CF910A
:10ED200008950F931F93CF93DF93EC01E09140037D
:10ED3000F091410309958C016A817B8181E00E94F9
:10ED4000FE6281E090E0012B11F480E090E0DF9121
:10ED5000CF911F910F910895E0914203F0914303E9
:10ED6000099420E030E00296FC0132974081442370
:10ED700031F0FC0131974081240F311DF4CFC901DE
:10ED80000895FC01208130E0322F22278181282B39
:10ED900002C0220F331F6A95E2F7232F3327FA01AF
:10EDA000EC5BFC4F808190E08223932328E030E0ED
:10EDB000241B350B02C0969587952A95E2F7089596
:10EDC0006F927F928F929F92AF92BF92CF92DF927B
:10EDD000EF92FF920F931F93CF93DF937C018B01F0
:10EDE0005A01E9012830310544F4A901B501C801EF
:10EDF0000E94C176F701808346C0690183E0D59403
:10EE0000C7948A95E1F7452B21F04701612C712CBD
:10EE100006C0FB01D701CB018C0D9D1D1FC048E032
:10EE200050E0B501C801860D971D0E94C176F4011E
:10EE300081934F01FFEF6F1A7F0A6C147D0479F7FD
:10EE4000AE014770552741155105E9F0E701C60DA0
:10EE5000D71DB501C801860D971D12C0E817F90727
:10EE600019F021912D93FACFAE0147705527411526
:10EE7000510549F0E701CC0DDD1D60E070E0CF01E8
:10EE80000E94C1768883DF91CF911F910F91FF90EF
:10EE9000EF90DF90CF90BF90AF909F908F907F903A
:10EEA0006F9008958F929F92AF92BF92CF92DF9210
:10EEB000EF92FF920F931F93CF93DF9300D0CDB7C4
:10EEC000DEB70E94EA618C0182E090E00E94C86196
:10EED000892B19F480E090E05FC0F801218130E0D7
:10EEE000322F22278081A901480F511DCA010E949B
:10EEF000D5597C01892B71F30E94EA614C01F7011D
:10EF00009681292F26952695269530E0977041E029
:10EF100050E011F440E050E0C901840F951F0E94B9
:10EF2000C861892BB9F2F70104811581A12CB12C9C
:10EF3000F8018081882379F1F801C180D12CA501E5
:10EF400047705527B50193E0759567959A95E1F758
:10EF5000680D791D883168F09601CE0101960E94F6
:10EF6000E076BE016F5F7F4FF80180810E941263DF
:10EF70000DC01A8219829601CE0101960E94E07698
:10EF800069817A81F80180810E94FE62AC0CBD1C0F
:10EF90000E5F1F4FCDCFC7010F900F90DF91CF9124
:10EFA0001F910F91FF90EF90DF90CF90BF90AF90A7
:10EFB0009F908F900895DC0150E0E0E1F0E0CF01F8
:10EFC000861B970B821B930B02C0440F551F8A951B
:10EFD000E2F78C91852B8C9311968C911197482B8D
:10EFE00011964C9308956F927F928F929F92AF9259
:10EFF000BF92CF92DF92EF92FF920F931F93CF9326
:10F00000DF93283031051CF4FA0140815AC05901C0
:10F01000E3E0B594A794EA95E1F76115710541F035
:10F020003901EA018B017C014A01C12CD12C05C0B8
:10F03000EA01FC014A0D5B1D2AC0F40141914F0118
:10F0400028E030E0B801C7018C0D9D1D0E94DB77E0
:10F05000FFEFCF1ADF0ACA14DB0479F79301277098
:10F06000332721153105E9F1CC0DDD1D488150E034
:10F07000021B130B085F1F4F02C0559547950A9559
:10F08000E2F760E070E0C7018C0D9D1D1AC0C41747
:10F09000D50719F069916193FACF277033272115AD
:10F0A0003105F9F0488150E068E070E0621B730BB5
:10F0B00002C0559547956A95E2F760E070E08A0DC9
:10F0C0009B1DDF91CF911F910F91FF90EF90DF90EB
:10F0D000CF90BF90AF909F908F907F906F900C9447
:10F0E000DB77DF91CF911F910F91FF90EF90DF9031
:10F0F000CF90BF90AF909F908F907F906F9008952A
:10F100006F927F928F929F92AF92BF92CF92DF9237
:10F11000EF92FF920F931F93CF93DF9300D0CDB761
:10F12000DEB77C01FC018681082F069506950695C1
:10F13000202F30E0877001E010E011F400E010E0D3
:10F14000020F131FC80102960E944E62009709F435
:10F1500048C00E94F161F7012281FC012083F70180
:10F160002381FC0121830E94F16102965C01A801C8
:10F1700060E070E00E948399F701048115810F5FC0
:10F180001F4F812C912CF80131978081882339F110
:10F19000F801C080D12C3401F7E06F22772474018C
:10F1A00093E0F594E7949A95E1F7EA0CFB1C88311B
:10F1B00028F00E941C639601AC0108C00E940963FC
:10F1C0009A8389839601AE014F5F5F4FB301C701F8
:10F1D0000E94F3778C0C9D1C0E5F1F4FD4CF81E0F3
:10F1E00090E00F900F90DF91CF911F910F91FF90C2
:10F1F000EF90DF90CF90BF90AF909F908F907F90D7
:10F200006F900895E0915F03F09160030994E0919D
:10F210003803F09139030994E0916303F09164039A
:10F220000994E0916503F0916603099480E090E011
:10F2300008950895E0913003F0913103099480E03E
:10F2400090E008950F931F93CF93DF93CDB7DEB770
:10F25000E0970FB6F894DEBF0FBECDBF0E943762B5
:10F260008C010E94EA61AE014F5F5F4F602F0E94E8
:10F27000ED80882309F442C088A99801281B310930
:10F28000C9010E94C861892BC9F18E8181110CC00E
:10F29000BE016A5E7F4F88E10E941263E0915303D2
:10F2A000F091540309952AC02A853B852D3C9BEAA1
:10F2B000390719F02F3F3F4F09F5823019F088E0E8
:10F2C00090E002C082E090E0019710F3E1E0F0E00E
:10F2D000EC0FFD1FE80FF91F23852F3FA9F3BE0197
:10F2E000645F7F4F89E10E94126389E10E941C6381
:10F2F00063EA74E30E942159892B51F6E0960FB618
:10F30000F894DEBF0FBECDBFDF91CF911F910F915B
:10F310000895AF92BF92CF92DF92EF92FF920F9338
:10F320001F93CF93DF93CDB7DEB7E0970FB6F89476
:10F33000DEBF0FBECDBF8C016B01CE0101967C01FB
:10F3400080E3F70111928A95E9F781E089838CE0E7
:10F350000E9409638C831D821F828091021591E0B7
:10F36000980F90930215898783E0B82EB8868DECAC
:10F370009BEA9B878A8789E10E941C636CE073E0AB
:10F380000E942159892B31F082E08E838FEF8C8788
:10F390008D8709C089E10E941C63BC01CE010C96D7
:10F3A0000E941859BE828DEC9BEA9D8B8C8B63EA80
:10F3B00074E3CE0146960E9418590E94EA619FA705
:10F3C0008EA70E94376288ABC7010E94ED7FB82EDE
:10F3D00090E00E944E62892B31F10E94F1614B2D29
:10F3E000BC01C7010E940B80E0902603F090270328
:10F3F0000E9441625C010E94F161B501F70109952B
:10F400000115110581F0009739F0019761F441E091
:10F4100050E064E070E004C041E050E060E070E083
:10F42000C601F8010995E0960FB6F894DEBF0FBE4D
:10F43000CDBFDF91CF911F910F91FF90EF90DF90A3
:10F44000CF90BF90AF9008950E94677B8093021584
:10F45000E0913003F09131030994892B29F0E09178
:10F460003003F091310304C0E0913203F091330393
:10F470000994CF93DF93EC0189919991009729F03A
:10F4800060E070E00E94725BF7CFDF91CF9108954A
:10F49000CF93DF93EC0189919991009719F00E9425
:10F4A000C25AF9CFDF91CF910895CF93DF93EC014A
:10F4B0007B836A830E94066C99838883DF91CF9156
:10F4C0000895FC012081318182819381820F931FF5
:10F4D000918380830895CF93DF93EC010E94066CA3
:10F4E00099838883DF91CF910895CF93DF93EC01C7
:10F4F0000E94066C28813981821B930B9C012F5F2F
:10F500003F4F81E090E04A815B814217530710F042
:10F5100080E090E0DF91CF910895CF93DF93FC01DD
:10F52000C281D38180819181C80FD91F0E94066C4E
:10F530009E01281B390BC901DF91CF910895CF930C
:10F54000DF93E8E1F7E3CAEDD6E3ACE0B7E311926D
:10F55000119219921992199219921D9287E3E03330
:10F56000F807A9F7DF91CF910895CF93DF93FC01BE
:10F57000E45FF84C40819C01220F331F220F331FA0
:10F580004423F9F04091940050919500E901C6524E
:10F59000D94C880F991FFC01E85EF84C808191815D
:10F5A000BA01681B790B88819981AA81BB81860F7A
:10F5B000971FA11DB11D88839983AA83BB835183A3
:10F5C0004083F901E652F94C608171818281938117
:10F5D000DF91CF91089560E070E0CB010895880F2E
:10F5E000991F880F991FFC01E652F94C4083518303
:10F5F000628373830895CF93DF93CCE0D7E3EAED82
:10F60000F6E3A8E1B7E389918823D1F080919400D3
:10F61000909195002D913C911197AC01421B530B99
:10F620009A014081518162817381420F531F611D94
:10F63000711D408351836283738311969C938E93D3
:10F640003496129657E3EA30F507E9F6DF91CF9149
:10F6500008950C947F7F0F931F93FC0180910315F5
:10F66000909104153383228315830483718360830F
:10F67000F0930415E0930315892B19F4CB010E9434
:10F68000997F80E090E01F910F910895809103157C
:10F69000909104150097C1F0109204151092031573
:10F6A000DC0114966D917C9115971296ED91FC9169
:10F6B00013970995E0910315F0910415309721F007
:10F6C000808191810C94997F08950C94F1950C940C
:10F6D000ED958EED92E00E94A95B86ED92E00C9490
:10F6E000A95BCF93DF930E94F761892BA9F086ED88
:10F6F00092E00E94C75BEC01892B21F10E943762E6
:10F70000998388830E9432629B838A83CE01049608
:10F710000E9473618CAB14C08EED92E00E94C75BB7
:10F72000EC01009779F002960E94856199838883A5
:10F73000BE016E547F4FCE018E579F4F0E94DC62F8
:10F74000CE0102C080E090E0DF91CF910895BC012E
:10F750006E547F4F8E579F4F0C94DC62CF93DF9394
:10F76000EC01BC018EED92E00E94125CBE01892B7F
:10F7700019F08EED92E009C086ED92E00E94125CD5
:10F78000892B39F0BE0186ED92E0DF91CF910C9488
:10F79000EC5BDF91CF9108950F931F93CF93DF938D
:10F7A000EC01BC018EED92E00E94125C892B91F07D
:10F7B000FE0161917191CF010E949862BE016E5469
:10F7C0007F4FCE018E579F4FDF91CF911F910F91A9
:10F7D0000C94ED62BE0186ED92E00E94125C892BD2
:10F7E000D1F00E948562688179818A819B810E9423
:10F7F00098628CA990E00E944E620CA910E00E94D1
:10F80000F161BE016C5F7F4FA801DF91CF911F9125
:10F810000F910C947A99DF91CF911F910F910895D8
:10F82000CF93DF93EC01BC018EED92E00E94125C5D
:10F83000892B19F0CE0102960CC0BE0186ED92E034
:10F840000E94125C892B19F08A819B8102C080E0A2
:10F8500090E0DF91CF910895FC018081918108951E
:10F86000860F911D860F911D8E579F4F0895860F0D
:10F87000911D860F911DFC01EE57FF4F80819181F4
:10F880000895089582E69BE10E94F05D892B21F0A6
:10F8900082E69BE10C94DD5D0895E0914E1BF091B2
:10F8A0004F1B309709F0099480E00895EF92FF9282
:10F8B0000F931F93CF93DF938C01EA01FC018081AA
:10F8C0009181009741F08C30934071F1F8011182E1
:10F8D000108283E0F6C080E024E0829FF0011124D2
:10F8E000E05BF44E118210828F5F8430A9F7809321
:10F8F0004D1B80918812909189129093611B809387
:10F90000601B0E94BB5A8093303760E470E082E64F
:10F910009BE10E94C95D0E945A828CE093E0F8014D
:10F920009183808381E0CDC06230D9F480913137FA
:10F9300090913237892B89F380914237863029F4B0
:10F9400080915A3781FD0E94427C81E00E94AF8302
:10F950008091313790913237892BF9F20E946F7E76
:10F96000DCCF633060F5611114C02097B1F2D09301
:10F970003F3CC0933E3C83E00E94AF83809131378F
:10F9800090913237892B11F00E944D7C0E94427C6D
:10F99000C4CF613011F6209709F4BFCFD0933B3C20
:10F9A000C0933A3C85E00E94AF83809131379091BB
:10F9B0003237892B09F4B1CF0E944D7CAECF673826
:10F9C00009F040C010924C1B80E5E82E8BE1F82E28
:10F9D00080914C1B8430C0F4F701828193818C1795
:10F9E0009D0749F4808191810E947A83F7011182F9
:10F9F000108213821282F4E0EF0EF11C80914C1BF6
:10FA00008F5F80934C1BE4CFE9E5FCE38381948115
:10FA10008C179D0719F4148213821082B0962CE380
:10FA2000E93DF20799F7E6EDFCE3818592858C17B5
:10FA30009D0711F4158214823D968DE3E835F80791
:10FA4000A1F76BCF683809F068CFC256DB4109F0E7
:10FA500064CF82E69BE10E94F05D892B09F45DCFC3
:10FA600010924C1BE0914C1BE43008F056CF20E282
:10FA7000E29FF0011124E05CF34C818D8823D9F0E2
:10FA800082E69BE10E94DD5D80914C1BE0E28E9F4F
:10FA9000C0011124805C934C90933F3C80933E3C8A
:10FAA00082E00E94AF838091313790913237892B69
:10FAB00011F00E944D7C80914C1B8F5F80934C1BFA
:10FAC000D1CFDF91CF911F910F91FF90EF900895CB
:10FAD00090934F1B80934E1B08959C014091881278
:10FAE0005091891290E0E0E5FBE19430A1F0608153
:10FAF00071816217730761F46281738164177507FE
:10FB000039F490934B1B11821082C9010C947A83B3
:10FB100034969F5FEACF90934B1B08959C0190E031
:10FB2000E0E5FBE19430B1F081E0890F4081518143
:10FB3000452B69F490934A1B31832083809188126E
:10FB40009091891293838283C9010C949583349692
:10FB5000982FE8CF90934A1B0895209188123091F6
:10FB60008912FC01358F248F778F668F089520913D
:10FB7000881230918912FC0132872187748763874C
:10FB80000895CF93DF93EA010E940983009749F01B
:10FB90002091881230918912FC0132872187D48705
:10FBA000C387DF91CF9108950F931F93CF93DF9376
:10FBB00000D000D0CDB7DEB78C01AB019FEF9983A9
:10FBC0009A839B839C83B801CE0101960E94C17DDC
:10FBD000009719F0FC01158304830F900F900F908C
:10FBE0000F90DF91CF911F910F91089540E050E069
:10FBF00062E086EE92E00E94635B109232371092D0
:10FC000031370895AC0161E086EE92E00C94445BDC
:10FC1000AC0160E086EE92E00C94445B0F931F937E
:10FC2000CF93DF938A010E948682EC01892B59F0E1
:10FC300080918812909189129D8F8C8F1F8F0E8FCB
:10FC4000CE010E94087ECE01DF91CF911F910F91CE
:10FC50000895CF93DF93A0913E3CB0913F3C109725
:10FC600019F0ED016C9605C0C0913A3CD0913B3C37
:10FC700029968091393C86FF23C01092491B80E071
:10FC8000E0E5FBE18430C1F04081518114962D9173
:10FC90003C9115974217530761F422813381211556
:10FCA000310539F08093491B398328831B821A82DE
:10FCB00005C034968F5FE6CF8093491B0E94427C3B
:10FCC00088819981009741F04A815B81609130374A
:10FCD000DF91CF910C94635BDF91CF9108950F93E7
:10FCE0001F93CF93DF9380914237863009F071C024
:10FCF00080913137909132378115954009F069C074
:10FD000004E912E01093323700933137D2E0D093F8
:10FD10003B37C4E9C0933C3710925E3710925D3791
:10FD20000E9454828095909590935E3780935D37C2
:10FD300010924437109243370E94438280959095E9
:10FD400090934437809343370E944D7C1093323711
:10FD500000933137D0933B37C0933C37A0913C3C64
:10FD6000B0913D3CFD01E459FD4F8CE692E00190DD
:10FD70000D920197E1F76CE672E081E597E30E944E
:10FD80000382809135378093513780913637809345
:10FD9000523780913737809353378091383780932B
:10FDA000543710925E3710925D370E9454828095CE
:10FDB000909590935E3780935D3710924437109200
:10FDC00043370E9443828095909590934437809367
:10FDD0004337DF91CF911F910F910C944D7CFC0123
:10FDE000680F791F80E048E1E617F70781F021915D
:10FDF00098E0322F3827532F517030FD8427869595
:10FE0000513009F480682695915099F7EDCF089507
:10FE10001F920F920FB60F9211240BB60F922F93D1
:10FE20003F934F935F936F937F938F939F93AF9382
:10FE3000BF93EF93FF9380919400909195009093DE
:10FE40001D3780931C3781E080930E3780917100BD
:10FE5000807D809371000E94467B80910E378823BD
:10FE6000D9F1809194009091950040911C37509168
:10FE70001D3784179507A0F48091E2369091E33600
:10FE8000A091E436B091E5368C57914EAF4FBF4FFD
:10FE90008093E2369093E336A093E436B093E53650
:10FEA0002091940030919500241B350B8091E2360F
:10FEB0009091E336A091E436B091E536820F931F1E
:10FEC000A11DB11D8093E2369093E336A093E436F2
:10FED000B093E53610920E37FF91EF91BF91AF913D
:10FEE0009F918F917F916F915F914F913F912F9152
:10FEF0000F900BBE0F900FBE0F901F9018959FB7DD
:10FF0000F894E1E7F0E08081807D808388B38F62A0
:10FF100088BB10929000E1E9F0E01082109292000C
:10FF200010929500109294008081856080839FBF1D
:10FF300008959C019FB7F8943093990020939800FE
:10FF400088B38F6288BBE1E7F0E0808182608083C4
:10FF50009FBF0895CF93DF93FC01DB0185E0EB01A8
:10FF600019928A95E9F78581837011F082E08C936C
:10FF70008781837021F082E012968C93129785819D
:10FF8000837081F08781837069F02389348981854A
:10FF900092852817390731F481E0848312961C92E8
:10FFA000129701C0148285818370823029F08330DA
:10FFB00011F488E001C080E011968C93119787813D
:10FFC0008370823029F0833011F488E001C080E032
:10FFD00013968C93DF91CF910895CF93DF9300D048
:10FFE00000D01F92CDB7DEB7BE016F5F7F4F0E947A
:10FFF000AA7F99818A81890F8D5F9B81890F9C815E
:020000021000EC
:10000000890F9D81890F0F900F900F900F900F9087
:10001000DF91CF9108954F925F926F927F928F926E
:100020009F92AF92BF92CF92DF92EF92FF920F9387
:100030001F93CF93DF9300D000D000D0CDB7DEB7B1
:100040008C017B01BE016F5F7F4F4E830E94AA7FB0
:10005000B9815A80652D70E0AB814C80242D30E051
:100060008B2F90E00396860F971F8A0F911D820FAA
:10007000931F5D81850F911D4E8150E048175907F0
:100080000CF493C0F801818180FB882480F8912CC6
:1000900083E0880C991C8A95E1F7828180FBAA2471
:1000A000A0F8B12C94E0AA0CBB1C9A95E1F78A2821
:1000B00080818770882A838180FBCC24C0F8D12C72
:1000C00045E0CC0CDD1C4A95E1F7C828848180FB13
:1000D000662460F8712C56E0660C771C5A95E1F79F
:1000E0006C28F7016082F80185818370F4E08F9FAE
:1000F000A0011124F80196819370F0E19F9FC00147
:100100001124842BF8014781F0E44F9FA0011124B2
:10011000842BF7018183F8018085F7018283B23057
:1001200051F4F8018185F7018383F8018285F70195
:10013000848385E001C083E0580E852D952D961BA4
:100140006115710561F061507109A801460F571FD3
:10015000FA014385F701E90FF11D4083EECFA2308C
:1001600089F4F701E50DF11DD80153969C91539741
:10017000908391E0950DF701E90FF11D8E5F549684
:100180009C919083B42DB80F8B2F9B2F921B211520
:10019000310561F021503109F801E20FF31F858923
:1001A000F701E90FF11D8083EFCF80E026960FB6AF
:1001B000F894DEBF0FBECDBFDF91CF911F910F919D
:1001C000FF90EF90DF90CF90BF90AF909F908F9077
:1001D0007F906F905F904F900895BF92CF92DF9283
:1001E000EF92FF920F931F93CF93DF93633008F446
:1001F000AEC0EA01D62E7C01FC01908196FBBB24A7
:10020000B0F88181282F269526952370C82EC29498
:10021000C694C69453E0C522392F3770388393FBB8
:10022000332730F9398394FB332730F93A8395FB30
:10023000992790F99B83BC822D83829583708E834E
:10024000CF8282818887222379F13381848190E073
:10025000982F8827830F911D9A87898787010B5FC5
:100260001F4F223071F46CE073E0CE010B960E94B8
:100270001859F70186818B8785818C870E5F1F4F08
:100280001EC02330E1F4F7013D96DE011B969E016E
:100290002D5E3F4F9E2F8F2F42914D93A217B30794
:1002A000D9F7092F182F0BC087010D5F1F4F6CE086
:1002B00073E0CE010B960E9418591A861986CC203D
:1002C000A1F1B1100DC0F8012081818190E0982F3B
:1002D0008827820F911D9C8B8B8B0E5F1F4F04C054
:1002E00089859A859C8B8B8BF2E0CF120EC06CE0D7
:1002F00073E0CE0145960E941859F80181818D8BDB
:1003000080818E8B0E5F1F4F18C0F3E0CF1215C097
:10031000085F1F4FD801FE017596CE014D962E91B4
:100320002193E817F907D9F708C06CE073E0CE0114
:1003300045960E9418591C8A1B8AC8018E199F096C
:100340002D2D281B2FA71EA70DA7D81608F480E077
:10035000DF91CF911F910F91FF90EF90DF90CF90A1
:10036000BF900895FB0141505109460F571FE417F4
:10037000F50778F4208130E0322F22276181260FA3
:10038000311D820F931F8217930708F4019632964E
:10039000EECFE417F50751F4208130E0322F222709
:1003A000820F931F8217930708F401960895CF9345
:1003B000DF93C0913C37D0E0649720913B3730E029
:1003C000322F2227C20FD31F48E050E065E477E3C5
:1003D0009E01280F311DC9010E94B281AE016DE45A
:1003E00077E30E94B281009721F098278927982708
:1003F00002C08FEF9FEFDF91CF91089590937B1B09
:1004000080937A1B0895FC012381260F20933837AF
:10041000A72FBB2792819A0F909337373181309362
:100420003637408140933537E92FF0E0EA17FB0774
:1004300048F481E0830F80933637811103C04F5F0A
:100440004093353730E077272617370788F49F5FCA
:100450009093373791110CC0809136378F5F80931E
:100460003637811105C0809135378F5F80933537DE
:100470000895AB01BC0180E090E00E94B281982712
:1004800089279827089544E150E069E377E380E005
:1004900090E00E94B281009721F098278927982741
:1004A00008958FEF9FEF089586E00C94D78181E146
:1004B0000C94D78180E0E82FF0E0EE0FFF1FE054AE
:1004C000F34C118210828F5F8430A9F780E090E2B4
:1004D000899FF0011124E05CF34C118E8F5F843012
:1004E000B1F780E094E09093751B8093741B80E0DB
:1004F0009DE0989FF0011124EA52F34C158214827A
:100500008F5F8A30B1F78093731B0895CF93DF9389
:10051000EC012091741B3091751B2F5F3F4F21150B
:100520008DE7380710F020E030E1522F432FE0E450
:10053000FCE390E0943059F0818D882329F0A48168
:10054000B581A417B50749F39F5FB096F3CF3093F9
:10055000751B2093741B1092731B90E0E0E0F0E099
:100560009430E9F080E2989FD0011124A05CB34C54
:1005700059968C915997811104C09093731BFD017A
:1005800010C0873041F4309739F05A962C915A9721
:10059000828D821708F0DF019F5FFD01E1CF90930C
:1005A000731B309791F182E0818F8091761B848755
:1005B0008091771B85878091781B86878091791B36
:1005C000878788ED94E0938B828B958B848B81E079
:1005D00090E0918B808B138E828F83E0808F168AC0
:1005E00080E1878B2091741B3091751B3227232764
:1005F0003227358324837783668388819981AA8112
:10060000BB8180839183A283B383CF01DF91CF919C
:1006100008950F931F93CF93DF93DC012091741BF8
:100620003091751B2F5F3F4F21158DE7380710F074
:1006300020E030E1522F432FE6EDFCE390E09A30CA
:1006400041F0C481D5819F5F3D96C417D507B9F7A6
:10065000E9CF3093751B2093741B90E08DE09A30A6
:10066000D1F0492F50E021E0290F849FF001859FB0
:10067000F00D1124EA52F34CEF0124960481158108
:10068000012B39F49093731B309741F480E090E094
:100690002CC0922FE4CF9093731BF8CF2091741B42
:1006A0003091751B3227232732273983288377839C
:1006B0006683109729F4108211821282138209C076
:1006C0008D919D910D90BC91A02D80839183A283EB
:1006D000B3838DE0849FD001859FB00D1124AA5271
:1006E000B34C80E418968C93CF01DF91CF911F918A
:1006F0000F9108959C0190E09430A1F0E92FF0E073
:1007000081E0890FEE0FFF1FE054F34C40815181CF
:100710004217530729F49093731B11821082089596
:10072000982FEACF9093731B08959C0190E094302A
:1007300099F0E92FF0E081E0890FEE0FFF1FE05400
:10074000F34C40815181452B29F49093731B3183E5
:1007500020830895982FEBCF9093731B0895AF9249
:10076000BF92CF92DF92EF92FF920F931F93CF939E
:10077000DF93C0913E3CD0913F3C843009F4DBC113
:1007800021E637E330933D3C20933C3C30933437B3
:1007900020933337833059F4898D8F70833009F07B
:1007A0006AC088899989892B09F0D5C67EC08230B4
:1007B00009F07FC08091791B8F5F8093791B811135
:1007C00013C08091781B8F5F8093781B81110CC0C0
:1007D0008091771B8F5F8093771B811105C080917B
:1007E000761B8F5F8093761B1092323710923137D1
:1007F0001092D53C1092D43C898D982F9D7F9530D6
:1008000041F48A8D8F5F8A8F843109F0A4C6198ED6
:10081000A2C6882309F49FC628893989232B09F4A5
:1008200040C09A8D2FEF290F2A8F911194C69B8D6E
:10083000983031F02FEF280F223048F4953039F4FA
:10084000198E80E88093393C0E94297E3DC5953001
:1008500038F423E0092E01C0220F0A94EAF701C000
:1008600020E32A8F9F5F9B8F8F708330A1F048F425
:10087000813009F445C3823009F06DC610925A37B1
:1008800042C3863009F4BCC4883009F4B9C484304A
:1008900009F061C6B5C484E08093393C0E94297E8A
:1008A00045C58F70833009F056C688E08093393C87
:1008B00000C5853019F5E0913A3CF0913B3C8481CC
:1008C0009581892B09F447C610923F3C10923E3C1B
:1008D00085E597E390933D3C80933C3C909334377F
:1008E000809333371092D53C1092D43C109232371B
:1008F0001092313788E08093393C1BC180913937A1
:10090000853409F028C600913B3710E0102F0027EE
:1009100080913C37080F111D80913137909132370B
:100920008017910708F417C61093323700933137B8
:1009300080913F378F7309F00EC6F0904037F11069
:100940000AC68091D03C9091D13CC0916903D0916E
:100950006A038C179D0759F44091D23C5091D33CC7
:1009600020916B0330916C0342175307A1F0209143
:10097000493730914A372817390709F0ECC52091DB
:100980004B3730914C378091D23C9091D33C281713
:10099000390709F0E0C50E944382019609F0DBC5E2
:1009A00080914237863009F429C18131E9F18130E3
:1009B00009F0D1C580914D37883009F0CCC510922F
:1009C0004D3780914F3790915037873F6FEF9607A3
:1009D00010F0099601C008969093503780934F37D6
:1009E0008091453790914637A0914737B09148376D
:1009F0008093493790934A37A0934B37B0934C3745
:100A00008091D03C9091D13CA091D23CB091D33C0C
:100A10008093453790934637A0934737B093483734
:100A200080E48093413774C50C511109109332371B
:100A30000093313785E597E390933D3C80933C3CB0
:100A40008091533790915437892B29F00E94578217
:100A5000019609F080C520914F373091503721150C
:100A6000310509F478C586ED9CE390933B3C809377
:100A70003A3CA0904D37B0904E3740916D03509165
:100A80006E0360916F0370917003A0914537B09130
:100A900046370091473710914837E0906B03F0904C
:100AA0006C03E0913A3CF0913B3C8DE3E835F8076C
:100AB00008F051C584819581009721F128173907E5
:100AC00009F586819781009719F0A816B906D1F427
:100AD000808191818C179D0729F4C280D380CE1428
:100AE000DF04B1F08417950729F4C280D380C616BD
:100AF000D70671F0A817B90729F4828193810817E6
:100B0000190731F03D96F0933B3CE0933A3CC9CF56
:100B100010923F3C10923E3C82E08093393C85E548
:100B200097E390933437809333371092D53C1092EB
:100B3000D43C0E94297E8091D43C9091D53C009772
:100B400009F409C59C01245E3F4F3093323720934E
:100B5000313730933B3720933C37E0913A3CF0916A
:100B60003B3C20852093413721E120934237089672
:100B7000982789279827909352378093513710925E
:100B80005437109253378481958190934E378093D8
:100B90004D37868197819093503780934F3780915E
:100BA000D03C9091D13CA091D23CB091D33C809369
:100BB000453790934637A0934737B09348378081A5
:100BC0009181A281B3818093493790934A37A09352
:100BD0004B37B0934C3781E697E390933D3C80933D
:100BE0003C3C0E94578280959095009711F48FEFBE
:100BF0009FEF90935437809353378AC40E94548256
:100C0000019609F0A8C440914F37509150374115D3
:100C1000510509F4A0C480914D3790914E3700974B
:100C200009F499C46091453770914637E091473790
:100C3000F0914837C0E4DCE3298D2223A9F0AC8190
:100C4000BD814A175B0781F4AE81BF818A179B077C
:100C500059F4A881B9816A177B0731F4AA81BB8155
:100C6000EA17FB0709F467C1A0962CE3C03CD20742
:100C700019F780915A378F738230D9F45093711BD2
:100C80004093701B80E0843091F0E82FF0E0EE0F8D
:100C9000FF1FE054F34C208131818F5F42175307CF
:100CA00091F71092731B80E0C0E0D0E07CC080938D
:100CB000731B80915A3782FD4EC484E180935A376A
:100CC00088E290E0909332378093313780E58093CB
:100CD0005937309154378091583780935437209149
:100CE00053378091573780935337209357379091DC
:100CF0005237809156378093523790935637809170
:100D000051378093731B40915537409351378093EF
:100D100055373F5F3093583731110DC02F5F209307
:100D20005737211108C09F5F90935637911103C028
:100D30008F5F8093553780914D3790914E379093C8
:100D4000711B8093701B20914F3730915037309337
:100D50004E3720934D379093503780934F37809183
:100D6000453790914637A0914737B09148378093E7
:100D7000493790934A37A0934B37B0934C378091C3
:100D8000D03C9091D13CA091D23CB091D33C809387
:100D9000453790934637A0934737B09348379DC364
:100DA000973089F08F5F8430C1F060E2869F9001B8
:100DB0001124F901E05CF34C918D9111F1CF8093F6
:100DC000731BEF010CC0209721F0428D9A8D941770
:100DD00048F7E901C05CD34CE5CF8093731B2097A3
:100DE00009F4B9C3D0933F3CC0933E3C83E08A8F63
:100DF000888F1E8A84E08F8B1B8E80914F37909155
:100E000050379D838C8380914D3790914E379F83CF
:100E10008E838091453790914637A0914737B091A6
:100E2000483788839983AA83BB8381E0898F809127
:100E3000761B8C878091771B8D878091781B8E879E
:100E40008091791B8F8781E090E0998B888B8091CE
:100E500054378B87809153378A878091523789879F
:100E600080915137888781E090E00E94F68A8091D6
:100E70005937982F907F913508F442C082958F7032
:100E800090E00597880F991F880F991F2091721B7A
:100E9000EF2DF0E0E817F9077CF5E75CF84C20A5AA
:100EA000211103C01092721B29C0213011F4F39458
:100EB000EFCF2230E1F431A53430C9F42093721B16
:100EC000F092731B82A590E0982F882723A5822B90
:100ED0009093711B8093701B893D74E0970710F00D
:100EE00088ED94E09B8B8A8B9D8B8C8B09C031A500
:100EF000332311F0F30ECCCF2093721BF092731BAF
:100F000080E180935A3780915A37826080935A37B4
:100F100082E08093613784E0809362378093633707
:100F200088ED809364378CE290E090933237809321
:100F3000313780E67FC2D0933F3CC0933E3C109255
:100F4000393C80915A37982F9470F92E82FF03C054
:100F5000198E80E218C29091593792959F70990F1F
:100F6000990F9093731B091B1109045111091093D8
:100F7000323700933137922F9F70923029F4982F97
:100F80009F73923139F41FC0913021F4982F9F73D1
:100F90009230C9F0012B19F4982F9370A1F0209191
:100FA0005137988529133CC22091523799852913CE
:100FB00037C2209153379A85291332C22091543772
:100FC0009B8529132DC284FF49C0688979896115E1
:100FD000710509F443C0CE010C960E940382309142
:100FE000553780913537381339C020915637809165
:100FF0003637281333C0909157378091373798137D
:101000002DC08091583740913837841327C03C87D2
:101010002D879E878F878B8D811119C09E89888D22
:101020002A8D821B292F269526952695821B980F9F
:101030009E8B87FD81952F89322F36953695231B00
:10104000820F8F8B969596959695890F888F81E064
:101050008093393C888D8A8F198A188A298DE22FCE
:10106000EF708E2F90E0FC013197E830F10508F029
:1010700072C2E057FF4F0C949C938091393C80FFE3
:1010800014C083E0898F80E48093393C198A188AE0
:101090008091313790913237009709F406C122E4EC
:1010A0002093393C0E94F68A00C180915A378F7391
:1010B000823009F050C224CF8091393C80FF6BC050
:1010C00080915A378F73823109F065C0809159370A
:1010D000982F907F913508F442C082958F7090E0F0
:1010E0000597880F991F880F991F2091721BEF2D6C
:1010F000F0E0E817F9077CF5E75CF84C20A5211132
:1011000003C01092721B29C0213011F4F394EFCF69
:101110002230E1F431A53430C9F42093721BF092EF
:10112000731B82A590E0982F882723A5822B90938C
:10113000711B8093701B893D24E0920710F088EDAD
:1011400094E09B8B8A8B9D8B8C8B09C031A53323BC
:1011500011F0F30ECCCF2093721BF092731B83E03F
:10116000898F809151378887809152378987809104
:1011700053378A87809154378B8781E090E00E94B3
:10118000F68A82E48093393C198A188A10923237A1
:10119000109231378AC080E28093393C0E94297EC8
:1011A000E0913E3CF0913F3C118E83CD80915A37C7
:1011B00080FF28C024FD26C088899989892B09F0E1
:1011C000CAC1809131379091323701960E94F68AD8
:1011D0008091393C982F90619093393C2091313720
:1011E00030913237232B19F082618093393C0E9471
:1011F000297E81E090E0998B888B88E0898F1B8E17
:1012000081E10FC185FF1DC080915F3790E0982F6D
:10121000882730916037832B40913C3C50913D3C76
:10122000480F591F50933D3C40933C3C409131370F
:1012300050913237BA01681B790B70933237609343
:10124000313740913137509132374115510551F0C6
:1012500024FD08C09091393C92609093393CCA01BA
:101260000E94F68A80915B3790E0982F8827209122
:101270005C37820F911D9093711B8093701B2C899A
:101280003D892817390710F0892B21F43093711B01
:101290002093701B8091701B9091711B9B8B8A8B8C
:1012A0008091393C837009F456C11092D53C10925C
:1012B000D43C0E94297E8091393C85FF07C0109262
:1012C000D53C1092D43C198E84E1ABC084FF0AC097
:1012D0001092D53C1092D43C81E090E0998B888BA1
:1012E00084E08CCF2091D43C3091D53C2115310540
:1012F000E1F080FF02C0198A188A888999890097CD
:1013000081F48A899B898217930720F49093D53CB6
:101310008093D43C8091D43C9091D53C998B888B20
:1013200004C09093D53C8093D43C1B8E809133377E
:101330009091343790933D3C80933C3C8091D43CD9
:101340009091D53C892B59F088899989009739F07B
:101350008896909332378093313788E10BC0809123
:10136000393C81FFF8C088E290E090933237809357
:10137000313780E180935A375CC08091393C80FFDF
:10138000EAC0198E80E18093393C0E94297EE3C037
:101390008091313790913237009711F00E94F68A90
:1013A00090915A378091393C90FF0BC080FF06C066
:1013B00087E0898F1A8E198A188A19C086E0898F6A
:1013C00016C080FF1EC085E0898F198A188AC3C0A5
:1013D0008091313790913237009711F00E94F68A50
:1013E00080915A3780FF0DC087E0898F1A8E81E087
:1013F00090E00E94F68A80E18093393C0E94297E29
:101400000FC08091313790913237892B49F4A3C0B6
:101410008091393C80FF9FC087E0898F1A8E9BC0E6
:1014200080E180935A3788E290E09093323780933E
:10143000313780E580935937888580935537898582
:10144000809356378A85809357378B85809358379A
:101450008C85809351378D85809352378E8580930C
:1014600053378F858093543786E0809342378C8141
:101470009D8190934E3780934D378E819F819093BD
:10148000503780934F378091D03C9091D13CA091C0
:10149000D23CB091D33C8093453790934637A0938C
:1014A0004737B093483788819981AA81BB8180935F
:1014B000493790934A37A0934B37B0934C37898D77
:1014C00084FF05C010925C3710925B3706C084E041
:1014D00080935B3788ED80935C3780E4809341375D
:1014E000809131379091323790933B3780933C37DE
:1014F0001092603710925F3710925E3710925D370E
:101500000E9454828095909590935E3780935D37CA
:1015100085E48093393710923A3710924037109211
:101520003F3780917A1B90917B1B019690937B1B98
:1015300080937A1B90933D3780933E3710924437C7
:10154000109243370E944382809590959093443740
:101550008093433704C01092323710923137109283
:10156000393CDF91CF911F910F91FF90EF90DF9069
:10157000CF90BF90AF900895982789279827089516
:101580000E94A5930895FC018091333790913437E0
:1015900029E33CE3281B390BAB01261737070CF472
:1015A000A9011416150654F45093D53C4093D43C2D
:1015B000E817F90719F0BF010C947A99089580E8AB
:1015C00080936100109261000E9496690E94D85A2F
:1015D0000E947B6D8091E4349091E5340097B1F3E3
:1015E00001979093E5348093E434F0CF20913E3C12
:1015F00030913F3CBC01C90108960E940382E091F2
:101600003E3CF0913F3CA5E3B7E38C918087119677
:101610008C911197818712968C91129782871396DD
:101620008C91838708952F923F924F925F926F9291
:101630007F928F929F92AF92BF92CF92DF92EF9262
:10164000FF920F931F93CF93DF93CDB7DEB76397CE
:101650000FB6F894DEBF0FBECDBF6C014B012A015F
:10166000FC0117821682838181FF43C3AE014F5F65
:101670005F4F3A01F6019381F40193FD859193FF49
:1016800081914F01882309F430C3853239F493FDE9
:10169000859193FF81914F01853239F4B60190E035
:1016A0000E94FD9952012501E5CF10E0F12C20E0C8
:1016B0002032A0F48B3269F030F4803259F083325A
:1016C00069F420612CC08D3239F0803339F4216007
:1016D00026C02260246023C0286021C027FD27C0C7
:1016E00030ED380F3A3078F426FF06C0FAE01F9F3D
:1016F000300D1124132F13C04AE0F49E300D112435
:10170000F32E20620CC08E3221F426FDEEC220643E
:1017100006C08C3611F4206802C0883641F4F4010A
:1017200093FD859193FF81914F018111C1CF9BEB77
:10173000980F933018F42061805E06C09BE9980FE3
:10174000933008F071C12F7E26FF16E02F73322EE2
:10175000853619F42064322E08C0863621F4F22F23
:10176000F0683F2E02C01111115037FE07C01C3324
:1017700050F4EE24E394E10E27E00BC0183038F06B
:1017800027E017E005C027E04CE3E42E02C0212F3C
:10179000E12C520144E0A40EB11CF2016081718180
:1017A000828193810E2DA3010E9481982C010981D1
:1017B00000FF02C003FF07C031FC08C032FE09C0B1
:1017C00030E2232E07C02DE2222E04C09BE2292EF8
:1017D00001C0212C802F8C7019F0211068C2A8C282
:1017E00037FE0FC0E40C04FF04C08A81813309F482
:1017F000EA941E1474F5F8E0FE1578F588E0E82EFA
:101800002CC036FC2AC0812F90E0841595059CF0F1
:101810002CEF42162FEF520674F0432D4068342E01
:101820000AC0E2E0F0E0EC0FFD1FE10FF11D808146
:10183000803319F411501111F4CF37FE0EC0EE248D
:10184000E394E10E812F90E0481659062CF4141908
:1018500004C0EE24E39401C010E037FE06C0141467
:10186000150434F4C201019605C085E090E002C081
:1018700081E090E021100196112331F0212F30E01A
:101880002F5F3F4F820F931F2F2D30E0821793075A
:1018900014F4F81A01C0F12C832D897049F4FF204B
:1018A00039F0B60180E290E00E94FD99FA94F7CFFA
:1018B000222029F0B601822D90E00E94FD9933FC90
:1018C00009C0FF2039F0B60180E390E00E94FD9945
:1018D000FA94F7CF37FE5AC0942D852D57FE02C0DB
:1018E00090E080E0292E382E20E030E0A2014E1951
:1018F00051095D874C87A201421953095F874E87C2
:10190000612F70E044275527461B570B598B488B96
:101910005FEF2516350649F4B6018EE290E02A8B7A
:101920003B8B0E94FD993B892A89421453046CF039
:101930004C855D854215530544F4EE85FF85E20F25
:10194000F31FE60DF71D818101C080E351E0251AE8
:1019500031082F5F3F4F48895989241635064CF0CE
:10196000B60190E02A8B3B8B0E94FD992A893B8926
:10197000CFCF2414350439F49A81963318F4953373
:1019800011F404FF81E3B60190E04BC08A818133FA
:1019900009F00F7EB60190E00E94FD99111105C07B
:1019A00034FC18C085E690E017C0B6018EE290E0E6
:1019B0000E94FD9982E0EE24E394E80EF301E80F23
:1019C000F11D8081B60190E00E94FD9911508E2D8D
:1019D00091F7E6CF85E490E0B6010E94FD9957FCAF
:1019E00005C04114510439F404FF05C051944194D9
:1019F00051088DE201C08BE2B60190E00E94FD9992
:101A000080E39AE0491651042CF08F5F5AE0451AA2
:101A10005108F7CFB60190E00E94FD99B601C201CE
:101A2000C0960E94FD9957C1833631F0833779F013
:101A3000833509F058C021C05201E2E0AE0EB11C5E
:101A4000F2018081898301E010E0230114C052017A
:101A5000F2E0AF0EB11CF2014080518026FF03C0BE
:101A6000612F70E002C06FEF7FEFC2012A8B0E94EE
:101A7000A9998C012A892F7715C05201F2E0AF0E87
:101A8000B11CF2014080518026FF03C0612F70E03D
:101A900002C06FEF7FEFC2012A8B0E946B998C010D
:101AA0002A892068322E23FD1AC08F2D90E0081756
:101AB0001907A8F4B60180E290E00E94FD99FA941B
:101AC000F4CFF20137FC859137FE81912F01B601E9
:101AD00090E00E94FD99F110FA940150110901154E
:101AE000110579F7F8C0843611F0893659F552019D
:101AF00027FF09C0F4E0AF0EB11CF20160817181D3
:101B0000828193810AC0F2E0AF0EB11CF2016081C4
:101B10007181072E000C880B990B2F76322E97FFC0
:101B200009C090958095709561957F4F8F4F9F4F1D
:101B30002068322E2AE030E0A3010E94479BE82E65
:101B4000E6183FC0022F853721F40F7E2AE030E0EF
:101B50001DC0097F8F3691F018F4883559F0C5C043
:101B6000803719F0883711F0C0C0006104FF09C048
:101B7000046007C024FF08C0066006C028E030E00B
:101B800005C020E130E002C020E132E0520107FF51
:101B900009C0F4E0AF0EB11CF20160817181828155
:101BA000938108C0F2E0AF0EB11CF2016081718137
:101BB00080E090E0A3010E94479BE82EE6180F7793
:101BC000302E36FE0BC0332D3E7FE11650F434FE2E
:101BD0000AC032FC08C0332D3E7E05C00E2D332DC9
:101BE00003C00E2D01C0012F34FF0CC0FE01EE0D0D
:101BF000F11D8081803311F4397E08C032FF05C0A9
:101C00000E5F04C0832F867809F00F5F33FD13C089
